:020000021000EC
:108000007804012041BF0100697902002DBF010001
:108010002DBF01002DBF01002DBF01002DBF0100AC
:10802000000000000000000000000000F9C0010096
:108030002DBF010000000000B1C001002DBF0100F4
:108040007DC201007DC201007DC201007DC2010030
:108050007DC201007DC201007DC201007DC2010020
:108060007DC201007DC201007DC201007DC2010010
:108070007DC201007DC201007DC201007DC2010000
:108080007DC201007DC201007DC201007DC20100F0
:108090007DC201007DC201007DC201007DC20100E0
:1080A0007DC201007DC201007DC201007DC20100D0
:1080B0007DC201007DC201007DC201007DC20100C0
:1080C0007DC201007DC201007DC201007DC20100B0
:1080D0007DC201007DC201007DC201007DC20100A0
:1080E0007DC201007DC201007DC201007DC2010090
:1080F0007DC201007DC201007DC201007DC2010080
:108100007DC201007DC201007DC201007DC201006F
:108110007DC201007DC201007DC201007DC201005F
:108120007DC201007DC201007DC201007DC201004F
:108130007DC201007DC201007DC201007DC201003F
:048140007DC20100FB
:04814400FFFFFFFF3B
:108148004FF0FF0C1CEAD0521EBF1CEAD15392EA32
:108158000C0F93EA0C0F6FD01A4480EA010C40020E
:1081680018BF5FEA41211ED04FF0006343EA501068
:1081780043EA5111A0FB01310CF00040B1F5000FAA
:108188003EBF490041EAD3715B0040EA010062F159
:108198007F02FD2A1DD8B3F1004F40EBC25008BF43
:1081A80020F00100704790F0000F0CF0004C08BF61
:1081B80049024CEA502040EA51207F3AC2BFD2F12E
:1081C800FF0340EAC250704740F400004FF000033C
:1081D800013A5DDC12F1190FDCBF00F00040704776
:1081E800C2F10002410021FA02F1C2F1200200FAB4
:1081F80002FC5FEA310040F1000053EA4C0308BF7B
:1082080020EADC70704792F0000F00F0004C02BFCB
:10821800400010F4000F013AF9D040EA0C0093F046
:10822800000F01F0004C02BF490011F4000F013BA0
:10823800F9D041EA0C018FE70CEAD15392EA0C0F0E
:1082480018BF93EA0C0F0AD030F0004C18BF31F079
:10825800004CD8D180EA010000F00040704790F04F
:10826800000F17BF90F0004F084691F0000F91F0F3
:10827800004F14D092EA0C0F01D142020FD193EAB9
:108288000C0F03D14B0218BF084608D180EA010041
:1082980000F0004040F0FE4040F40000704740F01D
:1082A800FE4040F44000704781F0004102E000BF0A
:1082B80083F0004330B54FEA41044FEA430594EA9E
:1082C800050F08BF90EA020F1FBF54EA000C55EAD9
:1082D800020C7FEA645C7FEA655C00F0E2804FEAAA
:1082E8005454D4EB5555B8BF6D420CDD2C4480EA8C
:1082F800020281EA030382EA000083EA010180EABC
:10830800020281EA0303362D88BF30BD11F0004F09
:108318004FEA01314FF4801C4CEA113102D040423F
:1083280061EB410113F0004F4FEA03334CEA13337A
:1083380002D0524263EB430394EA050F00F0A78092
:10834800A4F10104D5F1200E0DDB02FA0EFC22FA8D
:1083580005F2801841F1000103FA0EF2801843FA81
:1083680005F359410EE0A5F120050EF1200E012A72
:1083780003FA0EFC28BF4CF0020C43FA05F3C018B0
:1083880051EBE37101F0004507D54FF0000EDCF129
:10839800000C7EEB00006EEB0101B1F5801F1BD3D2
:1083A800B1F5001F0CD349085FEA30004FEA3C0CD6
:1083B80004F101044FEA445212F5800F80F09A80CC
:1083C800BCF1004F08BF5FEA500C50F1000041EBD0
:1083D800045141EA050130BD5FEA4C0C404141EBD4
:1083E8000101013C28BFB1F5801FE9D291F0000FCF
:1083F80004BF01460020B1FA81F308BF2033A3F17E
:108408000B03B3F120020CDA0C3208DD02F1140C74
:10841800C2F10C0201FA0CF021FA02F10CE002F1AF
:108428001402D8BFC2F1200C01FA02F120FA0CFCA8
:10843800DCBF41EA0C019040E41AA2BF01EB0451F1
:10844800294330BD6FEA04041F3C1CDA0C340EDCEF
:1084580004F11404C4F1200220FA04F001FA02F332
:1084680040EA030021FA04F345EA030130BDC4F1F0
:108478000C04C4F1200220FA02F001FA04F340EAE5
:108488000300294630BD21FA04F0294630BD94F096
:10849800000F83F4801306BF81F480110134013D7D
:1084A8004EE77FEA645C18BF7FEA655C29D094EAEE
:1084B800050F08BF90EA020F05D054EA000C04BF6C
:1084C8001946104630BD91EA030F1EBF0021002057
:1084D80030BD5FEA545C05D14000494128BF41F0F6
:1084E800004130BD14F580043CBF01F5801130BD5A
:1084F80001F0004545F0FE4141F470014FF00000E5
:1085080030BD7FEA645C1ABF194610467FEA655C95
:108518001CBF0B46024650EA013406BF52EA033537
:1085280091EA030F41F4002130BD00BF90F0000F25
:1085380004BF0021704730B54FF4806404F1320461
:108548004FF000054FF0000150E700BF90F0000F1A
:1085580004BF0021704730B54FF4806404F1320441
:1085680010F0004548BF40424FF000013EE700BF11
:1085780042004FEAE2014FEA31014FEA02701FBFA1
:1085880012F07F4393F07F4F81F06051704732F0D3
:108598007F4208BF704793F07F4F04BF41F400212A
:1085A800704730B54FF4607401F0004521F0004188
:1085B8001CE700BF50EA010208BF704730B54FF012
:1085C80000050AE050EA010208BF704730B511F013
:1085D800004502D5404261EB41014FF4806404F14B
:1085E80032045FEA915C3FF4D8AE4FF003025FEAD1
:1085F800DC0C18BF03325FEADC0C18BF033202EB55
:10860800DC02C2F1200300FA03FC20FA02F001FAAE
:1086180003FE40EA0E0021FA02F11444BDE600BF51
:1086280070B54FF0FF0C4CF4E06C1CEA11541DBF00
:108638001CEA135594EA0C0F95EA0C0F00F0DEF8CB
:108648002C4481EA030621EA4C5123EA4C5350EAB0
:10865800013518BF52EA033541F4801143F4801301
:1086680038D0A0FB02CE4FF00005E1FB02E506F092
:108678000042E0FB03E54FF00006E1FB03569CF0E7
:10868800000F18BF4EF0010EA4F1FF04B6F5007FED
:1086980064F5407404D25FEA4E0E6D4146EB06065F
:1086A80042EAC62141EA55514FEAC52040EA5E50E8
:1086B8004FEACE2EB4F1FD0C88BFBCF5E06F1ED892
:1086C800BEF1004F08BF5FEA500E50F1000041EBC9
:1086D800045170BD06F0004646EA010140EA020076
:1086E80081EA0301B4EB5C04C2BFD4EB0C0541EA98
:1086F800045170BD41F480114FF0000E013C00F3AD
:10870800AB8014F1360FDEBF002001F0004170BDD0
:10871800C4F10004203C35DA0C341BDC04F11404E9
:10872800C4F1200500FA05F320FA04F001FA05F275
:1087380040EA020001F0004221F0004110EBD37042
:1087480021FA04F642EB06015EEA430E08BF20EA6E
:10875800D37070BDC4F10C04C4F1200500FA04F311
:1087680020FA05F001FA04F240EA020001F00041A3
:1087780010EBD37041F100015EEA430E08BF20EA16
:10878800D37070BDC4F1200500FA05F24EEA020E5E
:1087980020FA04F301FA05F243EA020321FA04F08D
:1087A80001F0004121FA04F220EA020000EBD37044
:1087B8005EEA430E08BF20EAD37070BD94F0000F44
:1087C8000FD101F00046400041EB010111F4801F78
:1087D80008BF013CF7D041EA060195F0000F18BF29
:1087E800704703F00046520043EB030313F4801F65
:1087F80008BF013DF7D043EA0603704794EA0C0F1F
:108808000CEA135518BF95EA0C0F0CD050EA410634
:1088180018BF52EA4306D1D181EA030101F00041B1
:108828004FF0000070BD50EA410606BF10461946D9
:1088380052EA430619D094EA0C0F02D150EA0136E5
:1088480013D195EA0C0F05D152EA03361CBF104626
:1088580019460AD181EA030101F0004141F0FE41C5
:1088680041F470014FF0000070BD41F0FE4141F449
:10887800780170BD70B54FF0FF0C4CF4E06C1CEA49
:1088880011541DBF1CEA135594EA0C0F95EA0C0FFE
:1088980000F0A7F8A4EB050481EA030E52EA0335B9
:1088A8004FEA013100F088804FEA03334FF08055DA
:1088B80045EA131343EA12634FEA022245EA111507
:1088C80045EA10654FEA00260EF000419D4208BFB8
:1088D800964244F1FD0404F5407402D25B084FEA65
:1088E8003202B61A65EB03055B084FEA32024FF411
:1088F80080104FF4002CB6EB020E75EB030E22BF6E
:10890800B61A754640EA0C005B084FEA3202B6EB2D
:10891800020E75EB030E22BFB61A754640EA5C00DC
:108928005B084FEA3202B6EB020E75EB030E22BF6C
:10893800B61A754640EA9C005B084FEA3202B6EB6D
:10894800020E75EB030E22BFB61A754640EADC002C
:1089580055EA060E18D04FEA051545EA16754FEA8E
:1089680006164FEAC30343EA52734FEAC2025FEAAC
:108978001C1CC0D111F4801F0BD141EA00014FF03B
:1089880000004FF0004CB6E711F4801F04BF01430C
:108998000020B4F1FD0C88BFBCF5E06F3FF6AFAE28
:1089A800B5EB030C04BFB6EB020C5FEA500C50F1B8
:1089B800000041EB045170BD0EF0004E4EEA11313B
:1089C80014EB5C04C2BFD4EB0C0541EA045170BD42
:1089D80041F480114FF0000E013C90E645EA060E86
:1089E8008DE60CEA135594EA0C0F08BF95EA0C0FB4
:1089F8003FF43BAF94EA0C0F0AD150EA01347FF4FC
:108A080034AF95EA0C0F7FF425AF104619462CE7D2
:108A180095EA0C0F06D152EA03353FF4FDAE104635
:108A2800194622E750EA410618BF52EA43067FF486
:108A3800C5AE50EA41047FF40DAF52EA43057FF416
:108A4800EBAE12E74FEA4102B2F1E04324BFB3F5BF
:108A5800001CDCF1FE5C0DD901F0004C4FEAC002AD
:108A68004CEA5070B2F1004F40EB830008BF20F091
:108A78000100704711F0804F21D113F13872BCBF4B
:108A880001F00040704741F480114FEA5252C2F1A0
:108A98001802C2F1200C10FA0CF320FA02F018BFE9
:108AA80040F001004FEAC1234FEAD32303FA0CFC3C
:108AB80040EA0C0023FA02F34FEA4303CCE77FEACB
:108AC800625307D150EA01331EBF4FF0FE4040F415
:108AD8004000704701F0004040F0FE4040F40000C4
:108AE800704700BF80F0004002E000BF81F0004105
:108AF80042001FBF5FEA410392EA030F7FEA226C3C
:108B08007FEA236C6AD04FEA1262D2EB1363C1BFCB
:108B1800D218414048404140B8BF5B42192B88BF3A
:108B2800704710F0004F40F4000020F07F4018BF5D
:108B3800404211F0004F41F4000121F07F4118BF7D
:108B4800494292EA030F3FD0A2F1010241FA03FC25
:108B580010EB0C00C3F1200301FA03F100F000430D
:108B680002D5494260EB4000B0F5000F13D3B0F1D5
:108B7800807F06D340084FEA310102F10102FE2A44
:108B880051D2B1F1004F40EBC25008BF20F00100B4
:108B980040EA03007047490040EB0000013A28BF53
:108BA800B0F5000FEDD2B0FA80FCACF1080CB2EBD6
:108BB8000C0200FA0CF0AABF00EBC2505242184354
:108BC800BCBFD0401843704792F0000F81F40001F9
:108BD80006BF80F400000132013BB5E74FEA4103CC
:108BE8007FEA226C18BF7FEA236C21D092EA030F38
:108BF80004D092F0000F08BF0846704790EA010FB2
:108C08001CBF0020704712F07F4F04D1400028BFDE
:108C180040F00040704712F100723CBF00F50000C0
:108C2800704700F0004343F0FE4040F400007047F6
:108C38007FEA226216BF08467FEA236301464202A2
:108C480006BF5FEA412390EA010F40F480007047B5
:108C58004FF0000304E000BF10F0004348BF40425B
:108C68005FEA000C08BF704743F0964301464FF097
:108C780000001CE050EA010208BF70474FF00003F3
:108C88000AE000BF50EA010208BF704711F0004334
:108C980002D5404261EB41015FEA010C02BF844604
:108CA8000146002043F0B64308BFA3F18053A3F563
:108CB8000003BCFA8CF2083AA3EBC25310DB01FAAA
:108CC80002FC634400FA02FCC2F12002BCF1004F2E
:108CD80020FA02F243EB020008BF20F001007047BF
:108CE80002F1200201FA02FCC2F1200250EA4C0013
:108CF80021FA02F243EB020008BF20EADC70704759
:108D08007BB972B90029BEBF00204FF0004106E0D0
:108D180008BF00281CBF6FF000414FF0FF3000F083
:108D280057B8ADF1080C6DE904CE002909DB002B1A
:108D38001ADB00F04FF8DDF804E0DDE9022304B0A7
:108D48007047404261EB4101002B1BDB00F042F809
:108D5800DDF804E0DDE9022304B0404261EB4101A3
:108D6800524263EB43037047524263EB430300F004
:108D780031F8DDF804E0DDE9022304B0404261EB9C
:108D880041017047524263EB430300F023F8DDF8DA
:108D980004E0DDE9022304B0524263EB4303704769
:108DA80053B94AB9002908BF00281CBF4FF0FF314A
:108DB8004FF0FF3000F00CB8ADF1080C6DE904CEAF
:108DC80000F008F8DDF804E0DDE9022304B070479C
:108DD800704700BF2DE9F04786468C460846089E36
:108DE800154674461946002B40F0C1808542B2FAF8
:108DF80082F245D94AB1C2F1200300FA02FC95403B
:108E080094402EFA03F343EA0C0C4FEA154EA8B22D
:108E1800230CBCFBFEF80EFB18CC08FB00F943EA58
:108E28000C43994528D9EB1808F1FF3704D2994526
:108E380002D9A8F102072B44A3EB0903A4B2B3FBA0
:108E4800FEFC0EFB1C330CFB00F044EA0344A0427A
:108E580014D92C190CF1FF3304D2A04202D9ACF179
:108E680002032C44241A43EA07401EB1D4400023CD
:108E780034607360BDE8F0874746DDE76346F1E795
:108E880092BB431B01214FEA154EAFB2200CB3FB36
:108E9800FEFC0EFB1C330CFB07F840EA0343984525
:108EA80061D9EB180CF1FF3004D2984502D9ACF126
:108EB80002002B44A3EB0803A4B2B3FBFEFC0EFB99
:108EC8001C330CFB07F744EA0344A7424DD92C197D
:108ED8000CF1FF3304D2A74202D9ACF102032C44AF
:108EE800E41B43EA0040C0E7C2F1200395409440E8
:108EF80020FA03F12EFA03F34FEA154E9040AFB271
:108F08000343B1FBFEFC0EFB1C10190C0CFB07F80D
:108F180041EA0041884522D969180CF1FF3004D292
:108F2800884502D9ACF102002944A1EB08019BB2A3
:108F3800B1FBFEFC0EFB1C110CFB07F743EA0143D7
:108F48009F420ED9EB180CF1FF3104D29F4202D98F
:108F5800ACF102012B44DB1B41EA004193E7604678
:108F6800E3E76146F7E76046A4E76346B8E783426C
:108F780006D916B9002108467CE7C6E900E0F9E7FA
:108F8800B3FA83F78FB9834201D3724508D8BEEB91
:108F9800020460EB030301209C461EB9002169E727
:108FA8003846FAE7C6E9004CF8E7C7F1200CBB40A1
:108FB8000EFA07F522FA0CF42EFA0CF1BA401C430B
:108FC80020FA0CF3B8404FEA144901431FFA84FE13
:108FD800B3FBF9F809FB18300B0C08FB0EFA43EA4F
:108FE80000439A4540D9E31808F1FF3004D29A4566
:108FF80002D9A8F102002344A3EB0A0389B2B3FB08
:10900800F9F809FB183308FB0EFE41EA03418E45C7
:109018002CD9611808F1FF3304D28E4502D9A8F182
:109028000203214443EA0040A1EB0E01A0FB029891
:109038004145CE46434602D306D14D4504D20138B8
:10904800B9EB020E68EB0403002EA7D0B5EB0E02B5
:1090580061EB030101FA0CFC22FA07F3F9404CEA30
:109068000303C6E9003199E74046C5E74346D9E717
:1090780010F8012B11F8013B012A28BF9A42F7D0BA
:10908800D01A7047034613F8012B002AFBD1181A8F
:1090980001387047000000002DE9F0419846002390
:1090A80086B0CDE9043304230D46174606460193DE
:1090B800002800F0B580002900F0B280062104A83D
:1090C80010F060F8044648B103460121584A59484F
:1090D80010F0B8F9204606B0BDE8F081014604AAB0
:1090E800304610F02AF8044648B10346524A012196
:1090F800504810F0A7F904A810F06EF8EAE76A469D
:10910800012104A810F01AF9044610B103464B4A8D
:10911800EDE7009BB3B1042B1AD0052B0CBF092334
:10912800FF232B70032101AB02AA04A810F032F927
:10913800064678B10346424A01213E4810F082F9BA
:109148003446D8E7002300202B706860A860D2E777
:109158000723E6E7019B002BF4D018336B4403F890
:10916800100C02A9384612F03EF90222314602A834
:109178000CF096FE2B78C0B2092B06D10F2824D903
:109188006FF0150423462F4AB1E70F28F8D8072BAC
:1091980022D12D4B2D4F33F81000D8B1FFF7D6F957
:1091A80021A3D3E90023FFF73BFAFFF74BFC042187
:1091B80068600DEB010302AA04A8019110F0EAF817
:1091C800064660B10346224AB6E7224B224F33F8DF
:1091D8001000E2E72148EAE76FF07F04D2E7019B3D
:1091E80002A918336B4403F8100C404612F0FBF840
:1091F8000222314602A80CF053FEC3B20F2B07D946
:109208000121174A0B4810F01DF96FF0150472E799
:10921800581CC0B2FFF720FD3946FEF791FF95E7CD
:109228006FF0150456E700BF7B14AE47E17A24407F
:109238004FDB0200F0BB020078DB0200A1DB02007A
:10924800C3DB0200EFDB020018C302000AD7A33F0A
:1092580013DC0200F8C202000AD723400AD7A34051
:109268003EDC0200F8B502F1080323F0070300AF63
:10927800ADEB030D05466846144612F090F800233E
:109288006E460DF804308AB06A460849D661C2E9CC
:10929800051507491162074942F8101F4FF4235179
:1092A800054802F0D5F8BD46F8BD00BF3EC3020030
:1092B800000201030400000208BC02002DE9F0438B
:1092C80089B00B7806460C4602AF092B00F2D6800F
:1092D800DFE813F00A0040004400C000D400D400C6
:1092E800D400C700D400CE00CD6935B12B46644AFE
:1092F800012164480DF021FB28E00321624A6148FE
:109308000EF067FA614B07F10C0493E80700604B15
:1093180084E807007C606C468AB0BB6002AA5D4B9B
:1093280053615D4B93610523D3614FF4007313843C
:109338005A4B42F8103F4FF4135152482B4602F053
:1093480087F83046A546391D0FF048FA1C37BD4648
:10935800BDE8F083CB69524A0321CAE74A69CB6961
:109368000321009247484F4A0EF046FAD4F8148079
:10937800B8F1800F12D9DFF8309149463046A8F18C
:1093880080020FF0D8FA051E27D028DBA8EB0508C5
:10939800B8F1800FF1D86FF0790901E04FF00009BA
:1093A8004246304640490FF0C9FA0546B8B9237B12
:1093B800012B06D1238B3046BB8107F10C010FF03E
:1093C800BFF9B9F1000F16D063698022012100921C
:1093D8002C48364A0EF010FAB8E76FF00405237BE4
:1093E800012B06D1238B3046BB8107F10C010FF00E
:1093F800A7F9002D17DB62692B492D48FFF732FFCB
:1094080005222C49284811F0F6FF10B90FF06CFE20
:109418009CE706222849244811F0EDFF002895D141
:109428000FF065FE92E715F17A0FCDD02B4601219A
:10943800224A14480DF081FA0321214A11480EF0FE
:10944800C8F930460FF0A2F9034600283FF47EAF72
:109458001C4A4DE7CB690BB11B4A49E78B881B4A6D
:109468007AE7CB690BB11A4A42E78B88194A73E746
:10947800CB69002B3FF46AAF174A39E7174A6BE705
:1094880043C3020008BC02005BC3020050BC0200D8
:109498000100D20471C302008BC302000400000162
:1094A80091C30200AEC3020052DC0020CCC302000C
:1094B8001BC4020026C402002CC4020033C40200EC
:1094C80053C4020070C4020089C402009FC4020091
:1094D800B4C40200CAC40200DFC40200F7C4020018
:1094E8002DE9F0434FF0050889B0DFF8749000AF1C
:1094F800064614461D46C7E905233974C7F808907F
:10950800C7F80C800421781803F000F97B682A4614
:10951800BB83BB7F214623F0030312486C46BB770D
:10952800FFF7A0FE8AB06A460F4BC2F81C80C2E95A
:1095380005394FF4007313840C4B42F8103F002395
:109548004FF413510A4801F083FF07F10801A546BB
:1095580030460FF0B1F82437BD46BDE8F08300BFB0
:1095680015C502001BC5020028C502000400000141
:1095780008BC02002DE9F04F01269DB002AF07F1AB
:10958800140804460FF03FF854220021404611F019
:1095980013FF3B4642460021C7E9076645480EF0DF
:1095A80048FA054688B103463146434A43480DF018
:1095B800C4F9434A314641480EF00BF96FF00905EA
:1095C80028466C37BD46BDE8F08F4FF0080A3E6864
:1095D800DFF8F09039482EB3B369082B4AD1F36904
:1095E80039495B6801204B6045F6073308804B809A
:1095F8003E1D10233246043103F08CFAE94688B048
:1096080002AB324AC3E905264FF400729A831A4620
:109618002F4B42F8103F00234FF4E651274801F042
:1096280017FFCD4638680EF006FA274B17216363FB
:10963800284B4046A364284A09F0F2F8034668B369
:109648000121264A1D480DF078F92548E062FFF708
:1096580019FD042284F85E20224A0023E264802255
:109668002149C4E90E33C4E915122063226584F840
:109678002430A5E7EB468AB002AAC2E9059318236D
:1096880013620523C2F81CA042F8103F00234FF4D0
:10969800215101F0DDFEDD4636689BE787F823009F
:1096A8000F231421114ACDF800800D480CF00AFA56
:1096B800CBE700BF3DC502004BC5020008BC020055
:1096C80062C502009FC5020020DC002089C5020097
:1096D80003000001C5920100C2C50200CAC502000C
:1096E8003EDC002052DD0020D2DC0020EBC5020069
:1096F8002123012110B5074A0748FFF7F1FE034669
:1097080030B1BDE810400321044A05480DF025B9E1
:1097180010BD00BFF4C5020018D3002016C6020011
:1097280008BC020098B504460321224A224800AF2B
:109738000DF011F923781BB1032B20D0BD4698BD3D
:10974800237A012B19D0052BF8D11C4B6C4688B015
:109758006A461B49C2E905134FF400739383194BFA
:1097680042F8103F00234FF4E651134801F070FE11
:10977800A54615480BF082F8E0E7144BE6E7217A96
:10978800134A144B6C4688B0012908BF13466A4631
:109798001149C2E905134FF400739383094B42F84A
:1097A800103F00234FF4E651034801F051FEA5464F
:1097B800C4E700BF6DC6020008BC02004AC602002A
:1097C80079C602000300000120C9002031C602004A
:1097D8005EC6020068C6020099C602002DE9F0477D
:1097E800002582B0624C0321624A634802AF0DF043
:1097F800B2F82E46A146DFF88481DFF87CA194F800
:10980800543053B1B4F85230B4F8562003210092C2
:10981800504642460DF0F0FF013501360C2E04F19A
:109828000C04ECD12B460321554A53480DF095F80A
:109838000122E8214E480AF0B3F9804640B10346B8
:109848000121504A4C480DF088F8BD46BDE8F08724
:1098580099F85030DB07F8D50FF046FCD9E900013C
:1098680000220023FEF726FD6D4688B002AC0426D0
:10987800A246454BC4E9060163614AF8106F4FF4EC
:109888000351434652463C4801F0E2FDD9E9020142
:10989800AD4600220023FEF70DFD88B03B4BC4E91E
:1098A8000601636126614FF403514346524632482C
:1098B80001F0CEFDAD460021D9F81000FFF718F9E8
:1098C80088B0334B6361FEF753FE2661C4E9060195
:1098D8004FF4035143465246274801F0B9FDAD46BF
:1098E8008AB099F8384099F8390099F83A10B9F8D7
:1098F8003C3002AA53620623DFF898C0C2E9070188
:10990800C2E905C442F8103F234C43464FF4435183
:10991800194801F09DFD94F80080AD46B8F1000F9C
:1099280093D111F030FB88B00DF108094FF47A7229
:109938001A4BC9F81430A0FB020302FB0131C00B1B
:109948004FF47A72002340EA4140C90BFFF7D8F977
:109958004A46C9E9060142F8106F4FF403514346DD
:10996800054801F075FD0123AD4623706DE700BF82
:10997800D8C90020A6C6020008BC0200B3C602006F
:10998800C3C60200E4C6020007C702001DC70200E2
:1099980033C702004BC70200D2DD00206FC70200A8
:1099A800072805D0092808D0012808D1FFF716BFD5
:1099B800034A032103480CF0CEBF034AF9E7704776
:1099C8008CC7020008BC02009EC70200F8B500AFB1
:1099D8006C4688B06A46724B5361724B93614FF480
:1099E80000739383704B42F8103F00234FF4E65105
:1099F8006E4801F02DFDA54605F0E8F820B10121DB
:109A08006B4A6A480CF0A7FF03216A4A67480CF0C2
:109A1800A2FF04F0F3F9034660B1674A01216348E5
:109A28000CF09BFF0121654A60480CF094FF002070
:109A3800BD46F8BD0321624A5C480CF08CFF6148C2
:109A48000FF0E4FC034608B15F4AE7E74FF0FF3246
:109A58004FF0FF335D480AF035FF544803215C4A54
:109A68000CF079FF5B480AF02BFAC8B15A4A012179
:109A78004E480CF070FF594805F0D8F820B1012184
:109A8800574A4A480CF067FF5648FFF773FD0346EC
:109A9800002838D0544A012144480CF05EFFC6E73C
:109AA8000321524A41480CF056FF0AF099F904463E
:109AB80008B14F4ADBE70FF017FB00214FF4803065
:109AC8000BF0E6FB20460FF012FBD4E701340AD076
:109AD8003C230321474A35480CF03FFF4FF4F01070
:109AE80000210BF0D5FB0321434A30480CF033FF2B
:109AF8003C480EF09FFD034640B1404A01212B48E7
:109B08000CF02BFFE2E704463D4DECE729463548CB
:109B18000CF015FF0346F8B9324E30460EF0D3FE6E
:109B28000246012128460EF07DF8002816DA0DF0CD
:109B38007EFF344A036801211C480CF00EFF032104
:109B4800314A1A480CF007FF26480EF01FFE03465C
:109B58000028BBD02D4AD1E72D4A9CE730460EF0AD
:109B68008DFE034620B110F10B0F01D0294AE2E720
:109B7800EB88D90706D530460EF0BCFE034608B17F
:109B8800254AD8E7B5F906301A0705D5234A012131
:109B980006480CF0E0FED2E79B06BED5204AF6E761
:109BA800B9C70200D5C702000300000108BC0200C3
:109BB800DFC7020004C802001FC80200F1C8020083
:109BC80051C802002D9701006BC8020020C900206F
:109BD80094C80200A9990100ADC802006769020093
:109BE8000FC9020018D3002038C90200CEC80200ED
:109BF800DCC802005DC902007BC90200A3C90200DB
:109C080010D30020D3C9020027CA020041CA0200AB
:109C1800BDC90200E7C90200FEC9020016CA020057
:109C28001ECA02002DE9F04F91B0009302F0040320
:109C38000293C2F3C2030133840705460E46DDF8DA
:109C480068900392059340F0BB81041D30B1072949
:109C580009D86FF01B0011B0BDE8F08F01F00706BE
:109C6800341DC6F10806009B4FF000084FF0040AA7
:109C7800591E4FF0FF3347460193C3465346CDF86C
:109C880010800DB1009A22600598002800F3E88042
:109C98009848009A824203D397488242C0F0E080F5
:109CA800039AA4EB050E92074FEA9E0000F1038188
:109CB8000F2F00F2B180002D00F0058107F140025E
:109CC8000DEB020C019A0CF8200C0CF8102C0498DF
:109CD80001300490E7E07A285DD84B280ED8472851
:109CE80059D829282DD8252852D054D820287AD0B8
:109CF8002338D0F1000B4BEB000B74E04C382E28C6
:109D080049D8DFE800F0704848484848484848487B
:109D180048484B484848484848484859484B4B5990
:109D28005959704B6D487048184B184848827F4BFA
:109D380048484B487F0000204FF0000B4FF0040AC2
:109D480038E001222A38C0B202FA00F010EA0E0FF9
:109D580049D110F0625C2FD110EA020B43D0604663
:109D6800013C5444B4FBFAF40AFB04F4002D61D01E
:109D7800A3EB050CA444B4453FF66BAF002868D1AB
:109D8800042B47D159F8043B2360042304342AE008
:109D9800019A013A01924FF0000B24E011F8010CEE
:109DA8006C2834D1002011F8023C83466C2BC5D1B5
:109DB8004FF0080A5346D3E709F1070929F00709C4
:109DC800073424F00704F9E802AB35B106982044BB
:109DD800B0423FF63EAFC4E900AB4FF0000B083489
:109DE8004FF0080A534611F8010F002878D0BBF14C
:109DF800000F7FF470AF2528F5D14FF0010B019BC0
:109E0800013301934FF0040AECE7584694E7002029
:109E18008346A5E7082B02D06FF015001BE709F170
:109E2800070929F00709F9E80223C4E900230823F0
:109E38000834D8E768B9042B02D109F10409A4E76A
:109E4800082BE9D109F1070929F0070909F10809DF
:109E5800EDE7059A013A059259F8042B009210E7AC
:109E6800039A900720D54FF0010CA4EB050E4FEA9A
:109E78009E00BEF5007FCFD20F2FCDD8F5B107F1E8
:109E880040020DEB020E019AC0B20EF8200C0EF83B
:109E9800102CBCF1000F3FF41AAF60F07F000EF8F1
:109EA800200C08F101080137C5F108024FF6DA7EE7
:109EB8000434069297E74FF0000CDAE7BCF1000F84
:109EC80001D00136EFE7029802360028EBD100985E
:109ED800CDE90631FFF7D6F8DDE906310644E2E7B9
:109EE800631BB3F5806F97D245B9A6F10804E01853
:109EF800B1E600BFACB802004CEA0200029A9B0827
:109F080028602B709DF81030C2B1EB7085F8028084
:109F1800B8F1000F05D0002208A8C5F1010C97423E
:109F28000ED14FF0000AC5F101030DF1200901938C
:109F38000DF1300B574512D1601B8CE66B70E5E7CD
:109F480010F8013B190608D504EB0C0EB64503F0D2
:109F58007F033FF67EAE04F8013B0132DFE7B8F13C
:109F6800000F03D099F90020002A17DB029BD3B118
:109F78001AF80B2004F8012B0022019B98182044A2
:109F8800B0423FF666AE99F80000009904F8010B5C
:109F98002046039211F003FA039A14440AF1010AC5
:109FA80009F10109C6E799F8002055F82230009315
:109FB800029B009845F82230FFF764F8421CDCE762
:109FC8006FF00D0047E600BF2DE9F04F97B000AFE6
:109FD800D7F880B03B62CBF3C0030446894690F8BB
:109FE80002A0FA62BB6141B9457800780AEB8000AB
:109FF80020444D4517D8A0EB0409E378FB61BAF17A
:10A00800000F02D01BF0010F16D1FB6953BBFB6A8E
:10A018001BB1494620463A6A98474D4628465C3760
:10A02800BD46BDE8F08F461C3046FFF72BF80130DF
:10A03800304409F10109DCE7626823787A62FA6A38
:10A048009900796104EB8301002A40F001810E46F2
:10A058004FF000084D4601EB0A094E454CD101EB83
:10A068000A0610E01BF0020FD1D023789A007A611B
:10A07800626804EB83017A62FA6A002A77D14D4656
:10A08800904601EB0A061BF0050F0CBF02230123C3
:10A09800FB62FB6906EB430A0BF00203BB62564501
:10A0A800BCD016F8021B16F8013C54F82390AF4BAD
:10A0B800994502D3AE4B994536D3BB69002B40D0A6
:10A0C800786A0CF031FF00283BD0E9468AB06A462E
:10A0D800A84B53617B6AC2E906314FF400731384BD
:10A0E800A54B42F8103F00234FF41251A34801F04A
:10A0F800AFF9023DCD46D2E716F8013BF96254F8B4
:10A108002300FEF7BFFFD7F88430F96A01304BB15E
:10A11800D7F8883098453EBFD7F8843023F8180020
:10A1280008F10108054498E7BB6923B1786A0CF087
:10A13800FBFE0028C9D11BF0010F05D1FB6AED1AFF
:10A14800ADE7BB6A002BAAD04846FEF79BFFD7F8BD
:10A15800843053B1D7F8883098453FBFD7F884206A
:10A16800431C22F8183008F10108054497E7BAF1B2
:10A17800000F73D01BF0040673D0D046002607F1F9
:10A18800480052463B61B96211F009F9B96A3B6966
:10A1980001EB0A02BA62FA69F9695200FA60BA6A0E
:10A1A80002EB41023A610BF00202BA603A69B96AFD
:10A1B8008A4258D162781BF0020F18BF00217A62D8
:10A1C80008BF4FEA5801B2181BF0010FD2B240F095
:10A1D8009F801BF0040F14BF40460020BB616270D3
:10A1E800A070E17020463A6A7969FB6A9847051EB3
:10A1F800FFF614AFBB69414623707B6A3A6A637005
:10A20800FB6984F802A0E37007F14800FB6A9847ED
:10A21800B0F10008C0F2B4807B69A9EB0A01C91A41
:10A22800FB683A6AC91AD7E90A0398470028C0F2B6
:10A23800A9804FF0000BA84408EB000507F1380A85
:10A24800B34567D300213A6A0846FB6A9847E5E6B2
:10A2580056464FF0000807F1380092E75646D046B8
:10A2680096E7B04694E7BA6A12F8021B12F8015C46
:10A27800BA6254F825003D4A904202D33C4A9042C3
:10A288001ED3BA6932B1786A7B600CF04DFE7B68E8
:10A2980000288BD1BA6802BB08F1280207F1300CFC
:10A2A80008F10100944407F1580208F1020852FA33
:10A2B80080F00CF8101C5FFA88F800F8105C75E75D
:10A2C800BA693AB1786A7B600CF02EFE7B68002888
:10A2D8007FF46CAF1BF0010F09D006F1280207F1DB
:10A2E8003000711C161806F8205CCEB25EE71BF031
:10A2F800040F3FF45BAF08F1280207F1300008F1C2
:10A30800010102EB000808F8105C5FFA81F84DE7DC
:10A31800002063E71BF80A3054F8239087F8373099
:10A32800D7F88430FBB133F81B8001213A6AFB6A05
:10A3380007F137009847002824DB0544B8F1000FDF
:10A3480006D14846FEF79EFE00F101081FFA88F87C
:10A35800414648463A6AFB6A9847002812DB05449A
:10A368000BF1010B6CE7D7F88480DEE7ACB802008C
:10A378004CEA02006FCA020004000001C0BB0200E0
:10A3880045464BE6054649E6014B1860704700BF55
:10A3980080C5002030B5002587B0CDE9030104460B
:10A3A800009503A90548059500F010F9DDE904308A
:10A3B8009842B8BF255407B030BD00BF7F6F020078
:10A3C800032808B506D90DF032FB092303604FF0C6
:10A3D800FF3008BD2822044B02FB0033D3E8AF3F0F
:10A3E800002BF0D00020F4E788D3002070B5044695
:10A3F8000E461546FFF7E4FF00280DDB28236343CC
:10A40800064AD1184968316015B10C3313442B60E2
:10A4180028235C43105970BD0020FCE780D300203E
:10A4280070B500254FF0FF334FF0FF3217480AF0A0
:10A438003FF9174BD3E8AF2F7AB10135042D03F15B
:10A448002803F7D10DF0F3FA17234FF0FF35036017
:10A458000E480AF0A5F9284670BD28246C43D3E8B5
:10A46800EF0F0130C3E8E10F0029F8D1094E331985
:10A4780032515A6004F10C00304410F01BFB04F117
:10A488002000304410F017FCE2E700BF78C8002035
:10A4980088D3002080D3002010B404461046282218
:10A4A8005443084B1A191951506040B1C26832B16F
:10A4B8000C34234440F2051210BC0CF093BD10BCC0
:10A4C800704700BF80D300202823434330B50D498F
:10A4D80008330B44D3E8AF2F92B1541ED3E8EF5F93
:10A4E800954204D1C3E8EC4FBCF1000FF6D1F1D18D
:10A4F800012A05D12823584300230A180B5053601A
:10A5080030BD00BF80D30020F0B5024601680A279D
:10A518000020074E0B461C780131355D6D0701D4CC
:10A528001360F0BD07FB0043A3F13000F2E700BF62
:10A53800D0E802002DE9F84F15469A46D378224A0A
:10A548006F2B12F803B080460F460BF0030B29D08F
:10A5580024D8582B0CBF10260A26DDF8289032463E
:10A56800002340463946FEF71BFC092AD4B21ED800
:10A578003034B045E4B277F1000709F8014D01D352
:10A58800D14511D82B789B0605D5082E15D1AB7867
:10A5980043F00803AB704846BDE8F88F03F0F703B3
:10A5A800702BD7E70826D8E780460F46D7E7BBF1D8
:10A5B800010F0CBF37345734DBE7102EEBD1AB78E3
:10A5C80043F01003E6E700BFD0E802002DE9F04FA2
:10A5D8008A4616461C46002597B00390307808B97D
:10A5E80028464AE3731C2528049307D05146039B49
:10A5F80098470028C0F241830135F0E11822002174
:10A6080010A810F0D9FE7378252B00F0A380002342
:10A6180098469E469C461846711C0F4611F8012B19
:10A628002B2A00F0C68000F2BD80202A00F0C480EA
:10A63800232A00F0C4802BB19DF8483043F0400332
:10A648008DF84830B8F1000F05D09DF8483043F038
:10A6580020038DF84830BEF1000F05D09DF8483032
:10A6680043F010038DF84830BCF1000F05D09DF879
:10A67800483043F008038DF8483028B19DF8483039
:10A6880043F004038DF848309DF8483003F0440146
:10A69800442903D16FF386138DF848309DF848306C
:10A6A8002A2A43F0800309978DF8483040F08C80BF
:10A6B8009DF8493043F001038DF849307B1C1A7826
:10A6C8002E2A0CBF012100219DF8492061F3410287
:10A6D8008DF849200CD15A1C09925A782A2A40F040
:10A6E80083809DF84920023342F004028DF8492006
:10A6F8001A786C2A00F0A48000F28680682A00F09C
:10A708008C806A2A00F0A5804C2A00F0AA801A469C
:10A7180012F8013B782B04928DF84B309DF84920B4
:10A7280000F217816D2B00F2A980692B00F21181CC
:10A73800572B00F2BE80412B03D0453B022B00F281
:10A74800088104229DF84A3062F302038DF84A30EA
:10A758000123CAE0B21C04928DF84B309DF84930B1
:10A76800D90740F1FD8054F8048BB8F1000F07DADF
:10A778009DF84820C8F1000842F004028DF84820EE
:10A788005A0740F1F68054F804BBBBF1000F80F281
:10A79800F5809DF849306FF341038DF849304FF04B
:10A7A800FF3BEBE02D2A0DD0302A7FF444AF012384
:10A7B80033E74FF0010C30E74FF0010E2DE74FF073
:10A7C80001082AE7012028E709A8FFF79DFE099B51
:10A7D800BB423FF474AF9DF848201390C00F60F35C
:10A7E80041028DF848206AE709A8FFF78DFE9DF819
:10A7F80048301490C3F3400242EAD07262F3410336
:10A808008DF84830099B73E7742A26D07A2A7FF49A
:10A818007EAF06219DF849200CE05A78682A9DF8F9
:10A82800492006D1012161F3C6028DF8492002337F
:10A838006DE7022161F3C6028DF84920013366E70E
:10A848005A786C2A9DF8492001D10421EBE70321AD
:10A85800F0E705219DF84920ECE707219DF84920FC
:10A86800E8E7BDF8482022F4F04222F0020242F460
:10A87800804242F00202ADF84820DFE76E3BD9B2D1
:10A8880001238B4040F282410B4238D113F0240F50
:10A8980052D1DF075DD503219DF84A3061F30203E9
:10A8A8008DF84A3002F07803A3F140004342434157
:10A8B8001BE00120A3F15801C9B200FA01F111F41B
:10A8C800624F7FF43EAF40F6010739421DD111F4C3
:10A8D800043F3ED09DF84A3060F3020302F078024C
:10A8E800402A8DF84A3034D000239DF84820C2F31E
:10A8F80040010B4363F341028DF848202EE7022103
:10A908009DF84A3061F30203E8E702209DF84A10F7
:10A9180002F0780260F30201402A8DF84A1002BF63
:10A928009DF8481041F001018DF84810632BDBD1E8
:10A93800131E18BF0123D8E703219DF84A3012F0EF
:10A94800780F61F302038DF84A3014BF0123002306
:10A95800CBE79DF8483043F001038DF84830C3E752
:10A968009DF94820002AACBF4FF0FF38DDF84C8035
:10A9780006E79F077FF513AFDDF850B00023CDE958
:10A9880013339DF84A309DF8491003F00703012B53
:10A99800C1F3C30133D1CB1E042B04D8DFE803F085
:10A9A800214646212100236801294FEAE372CDE9B7
:10A9B80010321CD19DF94030DA17CDE91032043439
:10A9C8009DF8483013F0030750D032465146049B97
:10A9D80003980CF016FB0028C0F24F810544049E32
:10A9E800FCE554F8043BDA17CDE91032E8E7022910
:10A9F800E5D11AB243F3C033CDE91023DFE7022BC8
:10AA080024D1CB1E042B04D8DFE803F0181010184B
:10AA1800180001294FF0000254F8043B14D0022911
:10AA2800CDE91032CCD19BB21093C9E7073424F09A
:10AA38000704F4E80223CDE91023C1E754F8043BE6
:10AA4800109300231193BBE7DBB2CDE7042B08D1A9
:10AA5800073424F00704D4E900230834CDE910238F
:10AA6800AEE7032BACD154F8043BDDE79DF84B006F
:10AA78007828B4D862281DD825283FF4B7AD5828BF
:10AA8800ADD1DDE910010DF13E03009312AA0AAB26
:10AA9800FFF750FDBBF1000F814680F29880B9F1B5
:10AAA800000F9CD00DF13E06A6EB0903002F50D0F5
:10AAB80001334EE06338152891D801A252F820F0EE
:10AAC80049AB0100ADAB0100E7A90100E7A901000E
:10AAD800E7A90100E7A90100ADAB0100E7A9010062
:10AAE800E7A90100E7A90100E7A9010037AC0100C7
:10AAF800D1AB0100F9AB0100E7A90100E7A901000A
:10AB080021AB0100E7A90100D1AB0100E7A90100D1
:10AB1800E7A90100D1AB0100BBF1000FDDF84090BF
:10AB28000ADB5946484610F08BFCB9F1000F3FF498
:10AB380056AF09EB000676E04846FEF7A3FAF8E7B9
:10AB4800109B00278DF8283001230DF129060DF1FF
:10AB580028099DF84A1011F01002069200F0818031
:10AB68000233139A134405924A0644BF14995B189A
:10AB7800B8F1000F40F38E80A8EB03089DF8483029
:10AB88005807C3F3800B00F18580590678D53FB18B
:10AB980051463846039B984700286EDB5F460135CF
:10ABA80030236EE01E075ABFC3F300135F012B2743
:10ABB800DDE91023002BBFF664AF524263EB430379
:10ABC8002D27CDE910235CE700275AE700279DF8D9
:10ABD80048100DF13E03A3EB09036FF386119B4563
:10ABE8008DF848107FF65BAFABEB0303139356E782
:10ABF800109880B30DF13E060AAB0021009612AA08
:10AC0800FFF798FCBDF84A30BBF1000F03F0EF03E3
:10AC180043F4F04343F010038146ADF84A30D5DAE7
:10AC280000283FF4DCAE0027A6EB090391E7109B50
:10AC380007293FF6D4AEDFE801F00C04060C08083B
:10AC48000C0C1D70CBE61D80C9E6EA17C3E900525B
:10AC5800C5E61D60C3E6314E07460523A6F1050982
:10AC680077E7080748BF01337BE718460793514643
:10AC7800039B98470028079B04DA17B0BDE8F08FBC
:10AC88002023C346594600290BF1FF3BEDDC454420
:10AC9800D8466D1A37B151463846039B9847002865
:10ACA800EBDB01359DF84A30DA0601D41B0706D5DF
:10ACB80051463020039B98470028DEDB0135069B70
:10ACC8003BB151469DF84B00039B98470028D4DBC5
:10ACD8000135059F2F4406E051463020039B9847D5
:10ACE8000028CADB01357B1B002BF5DC33464A46BE
:10ACF800514603980CF085F90028BEDB0544A844AA
:10AD0800A8EB0503002B7FF76AAE51462020039B72
:10AD180098470028B1DB0135F2E700BF28CB0200D5
:10AD28002DE9F047058B04462807904611D40229DF
:10AD380005F0070540F0CC8020460CF0CDFB78B13B
:10AD48000138218B042811D8DFE800F0C2106D8586
:10AD5800950001290CBF45F0100545F02005258315
:10AD680088F31188BFF36F8FBDE8F08701F0070AF9
:10AD7800AA4500F0A5800027B9463E46A368002BE7
:10AD880000F0BC8041F00801218388F31188BFF3EB
:10AD98006F8FA168002900F0BA800D68002900F0C3
:10ADA800B680334652462046D1F80480C047002D6D
:10ADB80076D02B6829461D46F0E701F007035A1F95
:10ADC800012A1BD8002221F00701062B276889B227
:10ADD800C4E9002209D13B4603E0628B0132628359
:10ADE8001B68002BF9D141F00201204621830CF0A9
:10ADF80073FB00287AD041F0200176E0042B0AD1B9
:10AE080021F0070189B2204621830CF065FB10B1BF
:10AE180041F020012183218B01F0070AAA454FD078
:10AE28000027B946AAE7236921F0070141F0060186
:10AE3800062DD3F8009021832DD1B9F1000F3FD012
:10AE480041F00801218388F31188BFF36F8F2046F2
:10AE58003949C84729E021F00701236941F0040175
:10AE680089B2042DD3F804902183E6D000274FF04F
:10AE7800040A3E4682E721F00701236941F00501F3
:10AE880089B2052DD3F808902183D6D000274FF03A
:10AE9800050A3E4672E700274FF0060A3E466DE770
:10AEA8002B4687E7B9F1000FD1D1EFF311882023A2
:10AEB80083F31288BFF36F8F238B23F00803238358
:10AEC800258BEA062ED525F01003238305F0070508
:10AED8006669218B002EBFF670AF00232768C4E98E
:10AEE800003321F0070141F001012183218B4FF04C
:10AEF800000901F0070AAA457FF440AF002F9CD053
:10AF080041F00801218388F31188BFF36F8F002F68
:10AF1800C8D03D6839463346524620460CF008FBF7
:10AF28002F46F4E7AB067FF51BAF25F020032383FC
:10AF380005F0070500E700BF657502002DE9F04739
:10AF4800044607464FF00109DFF8508014B9384627
:10AF5800BDE8F08794FAA4F5B5FA85F509FA05F382
:10AF68002E0108EB05156FEA030A24EA03042B7B7C
:10AF7800002BEBD058F806301B694BB94644736870
:10AF880004222846196807EA0A0700F04DFADDE7A7
:10AF9800284698470028D9D1F0E700BF40BC0200F6
:10AFA80030B5002289B00F490F4810F033F800225D
:10AFB80000230024CDE906230E230C4DCDE90334EC
:10AFC8004FF440722846CDE90144094B09490094E1
:10AFD80009F0AEFE084928460FF077FE204609B072
:10AFE80030BD00BF05B0010050CF0020C0CA00200E
:10AFF800DDB2010038E3002029CB0200014809F046
:10B008003DBC00BF08C900202DE9F04780461F4815
:10B018000F460CF05CFB0646002830D00025284679
:10B02800BDE8F087237B6BB12368DB680BB1204652
:10B03800984723681B69D3B96368042220461968B6
:10B0480000F0F2F9013610344C45EBD3B8F1000F9B
:10B05800E5D0002DE2D02846FFF770FF0546002F07
:10B06800F7D000214FF4A4700AF012F9F1E7204656
:10B0780098470028E0D00AFA06F31D43E2E70546A0
:10B088004FF0010A024CDFF80C90DDE730D40020C5
:10B0980040BC020050BC0200014B53F8200070472E
:10B0A800BCBC020008B5034608462BB1044A13602D
:10B0B80000F05EFC002008BD6FF01500FBE700BF44
:10B0C80084C5002010B5044C237813B9034809F04F
:10B0D800D5FB0123237010BDD3DD002008C9002053
:10B0E80010B5044606480CF0F2FA3CB1054BD3E81B
:10B0F800EF1F0139C3E8E21F002AF8D110BD00BFD5
:10B1080028D400202CD4002000200146034BD3E88B
:10B11800EF0FC3E8E21F002AF9D1704728D40020B6
:10B1280070B5FFF7F1FF0546074C084EB44200D34F
:10B1380070BD63685B792BB123685B6813B12946DE
:10B14800204698471034F1E740BC020050BC02008A
:10B1580010B5044C044920460CF066F8034B1C60FB
:10B1680010BD00BFE4C70020A8BC020020D4002006
:10B1780008B50023074A4FF400411370064A0748F0
:10B188001360074A1360FFF78DFFBDE80840FFF71B
:10B19800DFBF00BFD4DD002028D40020D376020012
:10B1A8002CD4002001460022002301480CF05DB891
:10B1B800E4C7002001480CF0F3B800BFE4C7002042
:10B1C800024B014618680CF03FB900BF20D400209C
:10B1D80001480CF074B900BFE4C7002070B5264BD5
:10B1E8001878002847D0FFF7E5FF054670B1234BD4
:10B1F800D3E8EF1F0139C3E8E21F002AF8D1204C39
:10B20800204EB4422DD32846FFF7DAFF1E4B1F4CC1
:10B218001B68002B19DD0FF0B6FE4FF47A72A0FB05
:10B22800020302FB0131C30B43EA4143D4E9002086
:10B238009B1A40F2E9324FEAD13161EB00019342A7
:10B2480071F1000101D3FFF76BFFD4E9003213F568
:10B258007A7342F10002C4E90032BDE87040FFF79A
:10B26800B7BF63685B7923B12368294620461B680A
:10B2780098471034C5E770BDD3DD00202CD40020DA
:10B2880040BC020050BC020028D4002048CF002057
:10B2980070B50D4D297861B90120FFF7B5FE0B4C4B
:10B2A8000B4EB44206D3FFF799FF0028FBD10123C8
:10B2B8002B7070BD63685B791BB1236820469B685F
:10B2C80098471034EDE700BFD4DD002040BC0200F1
:10B2D80050BC020000212DE9F0470846FFF794FE14
:10B2E800044648B340F267684FF0000909F0EEFFE2
:10B2F8001A4B186030B11A4B1B68092B02DD19482C
:10B3080009F0BCFA0025184FDFF858A044B12046D0
:10B31800FFF714FE044618B94FF0FF384FF0FF3915
:10B32800FFF75CFF064628B9B5B942464B4650467A
:10B3380009F0C8FA3546E9E74FF0FF384FF0FF3912
:10B34800D4E72B689B691BB1002228461146984711
:10B358001035BD42F5D3E8E7044DFAE724D40020C0
:10B368002CD4002008C9002050BC020040BC0200B8
:10B3780013B518480CF0ABF9174B1B7873B1EFF302
:10B388001184202383F31288BFF36F8FFFF726FF02
:10B3980084F31188BFF36F8F02B010BD0F4B1B6889
:10B3A800002BF9D050B9002200230D48CDE9002325
:10B3B8004FF4004200230AF0F1F9EDE70928EBD138
:10B3C80007480FF033FE074802B0BDE8104009F007
:10B3D80055BA00BF2CD40020D4DD002024D400208E
:10B3E80050CF002008C9002010B5064B04461B6842
:10B3F80098472146A06004480BF0B3FFBDE8104011
:10B40800FFF7B6BF84C50020E4C70020044A054BF7
:10B418009B1AB1EBD30F34BF52F8310000207047AC
:10B42800B8BB020040BC0200084B10B4C31A446801
:10B438001B110133237143689A7101224368196013
:10B4480043685A7110BCFFF73DBE00BF40BC020004
:10B458002DE9F04F8FB0C1F34A2804AF0D4691464D
:10B46800B8607B600C0DB8F1000F63D000264FF078
:10B47800040B4FF00A0A07F11403C7F80C80C7E958
:10B4880007667E620193CDF808B0CDF800A007F1F9
:10B498001C0332464846F968FEF796FDB0F5006F82
:10B4A80003461CD36C468AB0D9F8041004AB26486E
:10B4B8001A46C3E9050140F2FF71D9614FF40071E2
:10B4C8001984224B42F8103F4FF41251334620485A
:10B4D800FFF7BEFFA5462C37BD46BDE8F08FC0F389
:10B4E8000A0804F11700184420F0070080083B60A0
:10B4F800FFF758FE68F35325044690B13B6800F106
:10B508001001C7E9083607F11403F961CDE900A372
:10B51800CDF808B048460F4AF96807F11C03FEF752
:10B5280053FD68F353252A4620467B68B9680CF01A
:10B5380000F9D0E704F1170020F007008008FFF7B2
:10B5480031FE0446EDE700BF3ECB020004000001D7
:10B55800D8BB02000F7702002DE9F04F87B00446F0
:10B56800DDE9105ADDE912690F4693469846A6B3FD
:10B578001021334652460020CDF80090CDF81490A3
:10B58800FEF750FB014605F117000844144B04F080
:10B5980007040BF0070BE40020F0070003EA41233F
:10B5A80044EA8B1480081C430391FFF7FBFD44EA2F
:10B5B8000554054640B13EB1334652460399CDF88D
:10B5C80000901030FEF72EFB4346224639462846A7
:10B5D80007B0BDE8F04F0CF0ACB83146D3E700BF78
:10B5E80000FE0F00406820B1034BC01A40F3CF00A3
:10B5F80070474FF0FF307047B8BB02000EB403B578
:10B6080003AB53F8042B0146044801930CF00EF9E0
:10B6180002B05DF804EB03B0704700BF5D7802002C
:10B62800CA0605D48B064CBF02490349FFF7E6BF9B
:10B63800704700BF64E4020063E402002DE9F04FA4
:10B6480089B09A46149B9DF84CB00693159B044606
:10B658000593169B0D469046179E0493BBF1000F69
:10B6680000F09D8006F4807307930CF04AF806F00A
:10B678000209024600283ED020469249FFF7BEFF45
:10B688000746B9F1000F08D016F0440F35D12A4605
:10B6980020468D49FFF7B2FF074406F0010353B176
:10B6A8008A4B204653F82B20894B8A49002A08BF29
:10B6B8001A46FFF7A3FF06F48073002B49D006F063
:10B6C8000803002B63D1B8F1000F66D0424620462C
:10B6D8008149FFF793FF0546069B3D44002B6DD13A
:10B6E800049B002B73D1F30700F1E5803146204617
:10B6F800FFF796FFD9E00746C3E7784B186800289C
:10B70800CAD0774B4FF47A791B684FF46161B5FB67
:10B71800F3F5B5FBF0F300FB135509FB05F5B3FB97
:10B72800F1F2B5FBF0FE4FF03C0C01FB123100FBCF
:10B738001E55B1FBFCF309FB05F5B5FBF0F50CFB59
:10B74800131120460091CDE901E56649FFF756FF40
:10B75800A2E706F00803EBB1634B204653F82B2011
:10B768006249FFF74BFF0546B8F1000F05D0424686
:10B7780020465949FFF742FF0544BAF1000FABD004
:10B78800524620465A49FFF739FF0544A4E74FF0CF
:10B79800000AE1E706F00805E6E745469CE7BAF146
:10B7A800010F069B06D1002B65D1049B002B7CD092
:10B7B80000250CE0002BF8D04E485DE04E48069B73
:10B7C80022464E490BF07FFB049B002B69D0DFF823
:10B7D8003081DFF83091049F3146102F204628BF72
:10B7E80010274FF0000AFFF71BFF554546DC059B65
:10B7F800494620461A78FFF701FF4FF0010A1AF070
:10B80800070F03D141462046FFF7F8FE57453CD9BC
:10B81800059B4946204613F80A20FFF7EFFE0AF178
:10B82800010ABAF1100FEAD14FF0000A2046364952
:10B83800FFF7E4FE5246059B20469A5C334B995C21
:10B8480011F0970F08BF2E223149FFF7D7FE0AF1F2
:10B85800010ABAF1100F1DD01AF0070F03D14146A3
:10B868002046FFF7CBFE57455246E4D841462046CE
:10B87800FFF7C4FEEBE720485D46A0E741462046B7
:10B88800FFF7BCFE0AF1010AAFE720462149FFF79E
:10B89800B5FEC4E7059B3B440593049BDB1B04935F
:10B8A80099D1BBF1000F7FF41EAF204609B0BDE867
:10B8B800F04F0BF0C2BF2046054A0649FFF79EFE2F
:10B8C80014E700BF82CB020086CB0200CCBC02008A
:10B8D8007DCB020003D60200ABCB020038D4002097
:10B8E80034D400208FCB0200E0BC0200AFCB0200B2
:10B8F800B5CB02008B7802005D7802003578020033
:10B90800C2CB0200BACB0200C4CB0200D0E80200CE
:10B918005ED90200C0CB020042F20F7373B58B42AE
:10B9280028BF0B4605680446052168460D4A0BF0FA
:10B9380042FB0646636828460B225B680A490BF0FF
:10B9480067FF63683246694628465B680BF060FF0C
:10B9580063681B2228465B6804490BF059FF02B054
:10B9680070BD00BF2EC60200E2CB0200C6CB0200AB
:10B9780000210123064A904206D8064A01B901234C
:10B988001360054B18607047012140085B00F2E71F
:10B9980040420F0034D4002038D40020F8B50D46BA
:10B9A8000446064F4618B44201D12846F8BD14F89B
:10B9B800011BBB6801485B689847F4E78CB9020033
:10B9C800014B03600020704728BD020008B50448F9
:10B9D8000BF0E4FABDE8084002480BF0DFBA00BFFC
:10B9E80028CC02005DCC02002DE9F04706460C4643
:10B9F80000AF002936D0D1E90012E9468AB06D4679
:10BA0800A3684FF0050AA8461F48C5E90723C5E9FA
:10BA1800050148F810AF002342464FF421511B4856
:10BA2800FFF716FDD4E90312CD466369AD46184801
:10BA3800C5E90723C5E90501C5F810A0002342465A
:10BA48004FF421511148FFF703FDCD46E369012169
:10BA5800104A0E480BF0C6FEA36901210E4A0B4896
:10BA68000BF0C0FE012E07D1EFF305830B4A3146D8
:10BA78000648103B0BF0B6FE2146304608F06AFC3B
:10BA8800BD46BDE8F08700BF8BCC020028BC020091
:10BA9800BACC0200E9CC0200F8CC020026CD0200A4
:10BAA80030BFFFF7FDBF00BF074A936893F90E1038
:10BAB800002907DB526993421FBF044A536843F0C9
:10BAC80080535360704700BFDCDB002000ED00E0CE
:10BAD80070B52A4C06460D4629482A490BF047FFFF
:10BAE800A36ADB0647D5264827490BF040FF1120FB
:10BAF800A36A1C0704D5224824490BF038FF1220FA
:10BB08001E4CA36A990712D521491D480BF02FFF37
:10BB1800636BA26A120609D501211E4A18480BF068
:10BB280061FE1EB1A36A23F08003A3621320134CA5
:10BB3800A36ADE0704D5124817490BF018FF142032
:10BB4800A36A9C0604D50E4814490BF010FF152073
:10BB58000A4B9A6AD10658BF9A6A9A6A920642BFF5
:10BB68005A6A22F400525A629A6A42F0FF029A62B2
:10BB780000232B7070BD1020BAE700BF00ED00E075
:10BB880028BC020039CD02004FCD020082CD020050
:10BB980095CD0200ADCD0200C3CD0200E2CD02007A
:10BBA80010B5244C244925480BF0E1FEA36A9901FD
:10BBB8003ED5224822490BF0DAFE1E20A36ADA019C
:10BBC80004D51E481F490BF0D2FE1F20194CA36A4A
:10BBD800DB0204D519481C490BF0C9FE0220A36AF0
:10BBE8001C0304D5154819490BF0C1FE2120114C3E
:10BBF800A36A590304D5114815490BF0B8FE222051
:10BC0800A36A9A0304D50D4812490BF0B0FE23200D
:10BC1800084CA36ADB0304D508480F490BF0A7FEBC
:10BC28002420A36A6FEA03436FEA1343A36210BD9B
:10BC38001D20C3E700ED00E011CE020028BC020081
:10BC480029CE02003CCE020056CE020080CE020071
:10BC58009ECE0200C3CE0200DDCE020070B5294C94
:10BC680006460D46284829490BF081FEA36AD904E7
:10BC78003CD5254826490BF07AFE1720A36A1A05F9
:10BC880004D5214823490BF072FE18201D4CA36AE5
:10BC98009B0512D51C4820490BF069FEA36BA26ACC
:10BCA800100409D501211D4A17480BF09BFD1EB150
:10BCB800A36A23F40043A3621920124CA36A59050E
:10BCC80004D5114816490BF052FE1A20A36ADA056A
:10BCD8000ED50D4813490BF04AFE1B20094A936AFA
:10BCE80043F47F43936200232B7070BD1620C5E791
:10BCF800A36A9B04F2D504480B490BF038FE1C20BC
:10BD0800ECE700BF00ED00E028BC020008CF02000D
:10BD18001ECF020082CD02002FCF020048CF0200C2
:10BD28005DCF020078CF0200E2CD02002DE9F04796
:10BD38008AB0694B0446D3F804A089461646002504
:10BD480000AFCAF3080885F31188BFF36F8F02F0BC
:10BD58007F43B3F17F4F1ED1D3071CD4500603D4C1
:10BD6800110708D4012508E05C495D480BF0FFFD88
:10BD780016F0040600D04C4600250023FB71A8F1FC
:10BD88000303092B00F28680DFE803F0077C7F7944
:10BD98008484848484822C46EFE7524950480BF00F
:10BDA800E6FD00234C4EFB71F36A9A0705D54E4910
:10BDB8004B480BF0DCFD002329E0F36A002B01DA85
:10BDC8004A49F5E7F36A5B00F5D5494944480BF061
:10BDD800CEFD7369A26943F480737361BFF34F8F1B
:10BDE800BFF36F8F736932F8022C23F48073736189
:10BDF800BFF34F8FBFF36F8F4DF602739A4228D16E
:10BE0800236801213B4A36480BF0ECFC2368FA7999
:10BE1800DAB907F1080604F1200C32462068616897
:10BE2800083403C264451646F7D17A6A002D4ED00D
:10BE3800C2F3080121B96FEA52226FEA42227A62FC
:10BE4800184607F10801FFF7CFFD2837BD46BDE8C2
:10BE5800F087B36ADBB22BB10120F91DFFF738FE7A
:10BE68000346D4E7B36A13F47F4F04D00120F91DC9
:10BE7800FFF7F4FEF4E7B36AB3F5803F9BD3FFF70F
:10BE88008FFEEDE70020F91DE8E70020F91DEFE738
:10BE980019498DE7194A6E461AF4F87F8AB0184B8B
:10BEA80018BF13466A461749C2E90513A8F11003DB
:10BEB800D3614FF400731384134B42F8103F0023EF
:10BEC8004FF411510648FFF7C3FAB54673E722F459
:10BED800FF7222F00102B2E700ED00E0BECF0200DF
:10BEE80028BC0200E1CF0200F8CF020019D00200FE
:10BEF80027D0020046D0020062D00200A5CF02007F
:10BF080090CF020086D0020004000001044B5A6959
:10BF180042F010025A615A6942F480625A617047CD
:10BF280000ED00E0EFF30880EFF3098101B57246F8
:10BF3800FFF7FCFE01BD00BF002080F31488BFF3AB
:10BF48006F8F002080F30A8880F30B880DF0F9FAD0
:10BF580000200E490860BFF34F8F0D4880F3088812
:10BF680000F02CF8202080F311880A484FF4006173
:10BF7800401880F30988EFF314800221084380F306
:10BF88001488BFF36F8F00F009F9000094ED00E00A
:10BF98007804012038EB0020002318460649D1F820
:10BFA8009020C2F30722934200DB7047C1F8983013
:10BFB800C1F8A0000133F6E700ED00E010B572B655
:10BFC800002484F31388FFF7E7FF23464FF0FF3080
:10BFD8000C4A03F120010133102B42F82100F8D15B
:10BFE80000234FF0FF30074A03F160010133102BA3
:10BFF80042F82100F8D162B6BFF34F8FBFF36F8FBD
:10C0080010BD00BF00E100E0084B9B6883420BD1E4
:10C01800EFF3058343B1064B5A6842F080525A60E9
:10C028005A6A22F400425A620EF050BFDCDB00204C
:10C0380000ED00E06FF00A01084A9368D9670849E3
:10C0480098674B6843F080534B60002383F3118853
:10C05800BFF36F8F9368D86F704700BFDCDB002099
:10C0680000ED00E00E4A936883F88100EFF3118336
:10C07800202383F31288BFF36F8F4FF00061536959
:10C0880020F0FF009360074A5160002193F8812057
:10C0980010439A6F996782F31188BFF36F8F7047C7
:10C0A800DCDB002000ED00E010498A6882F881E0BE
:10C0B8004FF030001044EFF3098C80E8F01F74460D
:10C0C8007046FFF7CFFFA64608498A68864602F100
:10C0D800300090E8F01F8CF3098802F1000004B5E5
:10C0E8000BF04FFCBDE8044070470000DCDB00208B
:10C0F8001EF0040F0CBFEFF30880EFF3098081698D
:10C1080011F8021C0229FFD001B50BF025FC01BD76
:10C1180040B2002807DB01234109034A00F01F0051
:10C12800834042F82130704700E100E040B2002827
:10C138000CDB01220649430900F01F00824020332E
:10C1480041F82320BFF34F8FBFF36F8F704700BFB5
:10C1580000E100E0054B420953F82220012300F0DA
:10C168001F0003FA00F01040704700BF00E100E034
:10C1780040B2002801F10101ACBF00F16040064B5C
:10C188004FEA4111C9B2ABBF00F5614000F00F00A2
:10C1980080F800131954704714ED00E00B4A08B5F5
:10C1A8000B4B22F07F029A60BFF34F8FBFF36F8F64
:10C1B800D3F8882022F47002C3F8882008F0B4F974
:10C1C80009F022F900F04AF808F0EEF900800100C1
:10C1D80000ED00E042F8203C009B0D4942F81C3C71
:10C1E800019B21F0010142F8183C029B42F8081C0F
:10C1F80042F8143C4FF0807342F8043C00238367F4
:10C208004FF43C43203A0265C0F88030704700BFC5
:10C21800D96F02000B4B0E4698601546836E83F368
:10C228000B882C4686F309884FF00000064B984788
:10C2380020464FF000014FF000024FF00003034C7E
:10C24800204700BFDCDB002093790200D96F020091
:10C258001022014B1A61704700ED00E000232021F5
:10C268000348C2180133412B82F80013F9D17047F3
:10C2780000E100E008B5EFF30583064A103B02EB46
:10C28800C30152F8330049688847BDE80840FFF702
:10C298000BBC00BFA0B902001FB5094C094A2346D0
:10C2A8000121094800F012F900230393074B0121EB
:10C2B800E41A01A80193029400F012F904B010BD29
:10C2C8000000042080C5002028BD0200D8C9002035
:10C2D80010B50C7A0B6804F01F0223F01F031A43F1
:10C2E800CB68640923F01F03054943EA440343F07C
:10C2F8000103C1F89800C1F89C20C1F8A03010BD16
:10C3080000ED00E010B50A4BD3F89030C3F30723D3
:10C31800013B984208D901210346064A06480BF01A
:10C3280061FA6FF0150010BDFFF7D2FFFBE700BF01
:10C3380000ED00E09DD0020000BC02002DE9F04FA6
:10C348008946144606464FF00008514D85B0C84549
:10C3580027DAD6F804A0BAF1000F44D0BAF11F0FBB
:10C3680017D91AF01F0F14D1D6F800B01BF01F0F01
:10C378000FD158460BF02CFB07460AEB0B0001388F
:10C388000BF026FB874210D06FF01507414A3B4659
:10C3980001E04346404A012140480BF023FA6FF080
:10C3A8001504204605B0BDE8F08F17F1160FEDD043
:10C3B800BC42EBDDC5F89870D5F89C10C5F89870AC
:10C3C800D5F8A03021F01F0143F01F0BD6E9003249
:10C3D8001A44994202F1FF3A1DD1D34507D131469B
:10C3E800F8B20BF0FEFA08F101080C36AFE7314657
:10C3F800C5F89870D5F89C3022F01F0203F01F038F
:10C408001343C5F89C30E0B20BF0EBFA10F1160FAD
:10C41800C5D0441CE7E7C5F89870D5F8A020013BC3
:10C4280023F01F0302F01F021343D3453146E0B245
:10C43800C5F8A030E8D00BF0D4FA10F1160FAED042
:10C44800C5F89870D5F89C209DF808300BF1FF3B93
:10C4580062F304038DF80830D5F8A0309DF8082061
:10C468005B0863F347128DF80820D6E900321344BD
:10C47800009323F01F035B44A3EB0A03013023F06E
:10C488001F036946C0B20393FFF73CFFBEE700BF36
:10C4980000ED00E0E6D00200C3D0020000BC0200BC
:10C4A8000522044BC3F89420BFF34F8FBFF36F8F5F
:10C4B800704700BF00ED00E0BFF35F8F0022024B22
:10C4C800C3F89420704700BF00ED00E010B5034C9E
:10C4D8002278FFF733FF207010BD00BFD6DD0020A3
:10C4E8002DE9F74F294D8A4606464FF00008AB461E
:10C4F800274FD0451BDAD6F80490B9F1000F3FD08A
:10C508003168084601910BF063FA0199044609EB7A
:10C51800010001380BF05CFA84424FF014021D4B05
:10C5280008D002FB08F36FF015024BF8032003B0A4
:10C53800BDE8F08F14F1160F2C60F8D01978A142DD
:10C54800F5DD02FB08B0C7F89840C7F89840D7F85F
:10C558009C4000F10801007B64F304000871D7F8DF
:10C56800A0000C79400860F347140C71D7F89C10B0
:10C5780021F01F016960D7F8A01021F01F0129617F
:10C5880008F1010814350C36B3E700BF68D4002061
:10C5980000ED00E0D6DD0020F0B54149414CD1F86E
:10C5A80090302568C3F307239D4287B075D80020D3
:10C5B800FFF782FF3C4BC1F8C030854216D13B4C97
:10C5C80001A82570FFF7FCF900250646384FAE4252
:10C5D80013D1002023783249D1F89020C2F30722E2
:10C5E800934254DBFFF75CFF00202FE0616801EB0A
:10C5F8000011FFF76DFE0130DFE70199280101EB1B
:10C608000513DA683A40B2F5001F21D0B2F5800F61
:10C618002BD0B2F5801F38D15A689B680958013B66
:10C6280022F01F0003440120844623F01F0340EA40
:10C638004C10CDE902218DF8100002A9207805934D
:10C64800FFF760FE00281DDA6FF0150007B0F0BD97
:10C658005A689B680958013B22F01F0003444FF0B9
:10C66800020C012023F01F03E1E75A689B68095870
:10C67800013B22F01F0003444FF0000C062023F07A
:10C688001F03D4E723780133237001359FE7C1F8EE
:10C698009830C1F8A00001339EE74FF0FF30D5E78E
:10C6A80000ED00E034BD0200AAFF4400D6DD002002
:10C6B8000000F0FF014B1860704700BF90C50020D4
:10C6C80010B5074C2368C2180648C0F1005101F59F
:10C6D80080218A4236BF22604FF0FF30C01810BD5B
:10C6E8007CD40020F81001200122024B0020C3F85E
:10C6F800402570470090034020B1034B800143F070
:10C7080001031847704700BFA0BC0200F7B50646F2
:10C718000D460D488AB2836831461B689847002841
:10C7280010DA00240CE02F1B042F28BF04270CF07C
:10C7380074FA3A46019001A930190EF030FE3C44D3
:10C74800A542F0D803B0F0BD78B902002DE9F04158
:10C7580005460E461746104CDFF84080444507D37F
:10C768000BF065F96A2303604FF0FF30BDE8F081F4
:10C778002368AB4200D063B93A4631462846A368DD
:10C78800984730B13A4631462846E368BDE8F0415B
:10C7980018471034E2E700BFA8BB0200B8BB02008C
:10C7A8002DE9F04F4FF0000846469DB0CDE906014F
:10C7B80008A814461D460EF0E8FBDDE90823DDE96C
:10C7C800069BCDE904230DAB0A93CDF80C80BBF191
:10C7D800000F22D1002E6ED0B5F1FF3F08BFB4F193
:10C7E800FF3F17BF4FF47A724FF0FF34A4FB0243A8
:10C7F80002FB05331CBFE40B44EA4344079B4FF498
:10C80800827200934146069B039801940BF015F938
:10C81800074638461DB0BDE8F08FD9F8000000285B
:10C8280029DB0CAA0BA9FDF7E1FD074618B34FF069
:10C83800FF324FF0FF330C980BF00EF91CAB01934D
:10C848000AAB00934FF481724B4639460B980BF0B4
:10C85800F4F810F1780F824612D10022002308A8BC
:10C868000EF093FBDDE90834CDE9043400240C987C
:10C878000BF0F4F8254609F108090BF1FF3BA6E790
:10C888001AF1120F0C980BD1039B1BB10BF0E6F8B1
:10C898000126F0E70B9BB84603930BF0DFF8F7E7A8
:10C8A8000BF0DCF8BAF1000FE5DA0BF0C0F8CAF1CA
:10C8B8000003036021E0DDE9042308A80EF089FBEA
:10C8C800DDE9084522462B46DFF8C8800A990DACF9
:10C8D800091B891008FB01F1204608F099FF00F1B7
:10C8E8000B030B2B054604D82B4F1F4117F00107EC
:10C8F80006D00BF09CF86D4205604FF0FF3788E7D3
:10C90800B9460A94DDE906458DB9B9F1000F80D022
:10C91800002F7FF47EAFDDE9042308A80EF059FB51
:10C92800DDE908452B4625432246CFD171E720682B
:10C93800E680002827DB0CAA0BA9FDF757FD8246E5
:10C9480018B92023E38001371DE04FF0FF324FF084
:10C95800FF330C980BF080F80AAB514640F20312F3
:10C9680000930B9823460BF068F882460C980BF05E
:10C9780075F81AF10B0F09D0BAF1000F95D1B4F977
:10C988000630002BDFD10834013DBDE74FF0010927
:10C99800F9E700BFCDCCCCCC7EF7FFFF014B186088
:10C9A800704700BF80D4002010B4034C246824686A
:10C9B800A44610BC604700BF80D40020014B1B6810
:10C9C8005B68184780D400202DE9F0410D460646E3
:10C9D800E8B1E1B10846FCF755FB08281AD8104F12
:10C9E800DFF84080441C474507D322462946301DBE
:10C9F8000EF0D5FC0020BDE8F081B74205D02246F4
:10CA08002946381D0EF0BBFC38B13C37EBE76FF018
:10CA18001500F0E76FF05A00EDE76FF07700EAE7EE
:10CA280068C90020A4C90020F0B54FF0FF324FF0CC
:10CA3800FF33274885B00BF047F90025254C264ED3
:10CA4800B44205D3224805B0BDE8F0400BF05AB90E
:10CA5800C4E90155236825731B689F6897B13B6833
:10CA680083B104F110000EF025F804F124000EF053
:10CA780021F83B682046984794F8383023F00303A0
:10CA880084F83830237903BB2046CDE901338DF88B
:10CA98000C300BF0B2F940B1104A01A81368591CC8
:10CAA800116008210E4A0AF086FA9DF8043043B94D
:10CAB8000C4A01A81368591C116008210A4A0AF097
:10CAC8007AFA204601A9FFF77FFF3C34B8E700BF98
:10CAD800B4C8002068C90020A4C9002088D4002058
:10CAE80033D1020084D400203AD1020038B5074C73
:10CAF800074DAC4200D338BD032120460BF0EDF8BA
:10CB080010B920460BF047F93C34F2E768C9002019
:10CB1800A4C900202DE9F04F002489B002288346DB
:10CB28000E46CDE9064402925FD10B6804913BB9E9
:10CB38004A6852B94FF6FF734C89E11A4C424C418E
:10CB480006A801460022134608E01C46F8E70D78BF
:10CB5800013301350D70DDB2082D03D036F81350BE
:10CB6800002DF4D00132082A01F10101EBD14FF078
:10CB7800FF374FF0010A002310F8012B524588BFF8
:10CB88005FB203F10103DBB288BF9246082BF3D1F1
:10CB980099463A220023BAF1010F08BF4FF0FF3738
:10CBA800CDE900230022029800252B46B9F1040F95
:10CBB8005ED10199C95C034641BB302103F8021BD1
:10CBC8000099417018460135EDB24D452B46EDDB15
:10CBD800029B98420BD0BBF1010F4FF0000340F0CD
:10CBE8009C8000F8013C029802E0012803D0002054
:10CBF80009B0BDE8F08F2E234FF004094FF0FF373E
:10CC080082462646019100930494CBE74FF0000C2E
:10CC18004FF00908CDF814C0DFF804C1B1FBFCFEE1
:10CC280003910CFB1E11DDF814E0C64503DCDDF8AA
:10CC38000CE0E64509D3DDF80CE0CDF81480BEFB26
:10CC4800FCFE0EF1300E03F801EB4FF00A0E08F16E
:10CC5800FF38B8F1FF3FBCFBFEFCDFD14FF000010D
:10CC680019701B1A50FA83F0009B00F8013BAAE7E1
:10CC780074B1052D0CD906F10C0301933A2300F881
:10CC8800013B2E234FF004094FF0010B00938BE773
:10CC98009F420DD102B915B93A2300F8013B3A2356
:10CCA80000F8013B0AF1FF332B440022DDB28AE78A
:10CCB80012B13A2300F8013B049B33F8152052BA0D
:10CCC80012F47F4FC2F307235FFA82F816D00F2BB6
:10CCD800D9B20AD9002361220BF09CF80123612202
:10CCE80041460BF097F801226DE7092B04D8303143
:10CCF800C9B200F8011BF1E75731F9E7B8F10F0F96
:10CD0800EDD8B8F1090F94BF08F1300808F15708B9
:10CD18005FFA88F800F8018BE5E7037063E700BF66
:10CD280000CA9A3B2DE9F0470F6890F860503C4BD9
:10CD38003C4A064690F85E000537042814BF1046A2
:10CD480018460F600C460BF048F9C5F3400503463A
:10CD580038B9D4E90020904296F85E1004D16FF0FB
:10CD68000B031846BDE8F087501C20601170D4E909
:10CD780000829045F3D008F10102226088F8003063
:10CD88002146B6F85C000BF016F903460028E8D1F6
:10CD980006F12C000BF021F903460028E1D1306C94
:10CDA8006D00E8B1214696F860A090F808900BF065
:10CDB80014F90AF0010A03460028D2D1736C2146FF
:10CDC8005BB318460BF009F903460028C9D145F0B2
:10CDD80004054FEAC90345EA4A1503F018031D4341
:10CDE800B06B38B121460BF0F8F803460028B8D1EB
:10CDF80045F08005F06B38B121460BF0EEF803469C
:10CE08000028AED145F0400588F800502246394642
:10CE1800BDE8F04710200BF0FBB80BF0CCF8D3E7D7
:10CE28005CBD020064BD0200D0E900239B1A012BFF
:10CE380081BF054B1B881380036883BF023343609F
:10CE480000206FF00B00704740D10200D0E90023AA
:10CE58009B1A012B81BF054B1B881380036883BF76
:10CE68000233436000206FF00B00704742D102008C
:10CE7800142290F824305343014AD358184700BF6E
:10CE88006CBD020030B4142590F82440024B05FB19
:10CE9800043330BC5B6818476CBD020010B414241E
:10CEA80090F82420024B04FB023310BC9B681847FF
:10CEB8006CBD020070B4142690F82450034C06FB95
:10CEC8000544E468A44670BC604700BF6CBD02001E
:10CED800084B70B5C31A0D4607499B1004465943C1
:10CEE800402206480BF048FD2B4601462046BDE887
:10CEF80070401847A0D40020B76DDBB650B90200C7
:10CF0800402373B50B4C0093041B0B460D460A498E
:10CF1800A41061430646094A09480BF058FD011E52
:10CF280005DA30462B4602B0BDE87040184702B01B
:10CF380070BD00BFA0D40020B76DDBB63F8A0200E9
:10CF480050B9020010B5EFF31184202383F312883F
:10CF5800BFF36F8F074A136823F00201DB071160E4
:10CF680002D401200CF0F8FA84F31188BFF36F8F14
:10CF780010BD00BFF0D4002070B500220121044686
:10CF88000520FFF7F5F80F4804F0D0FA0E4B984249
:10CF980015D104F0DBFA26690C4930460AF0EBFAA1
:10CFA80000280BDB012535642469084904F11C00BD
:10CFB8000AF0E1FA002801DB0020E56470BD6FF09B
:10CFC8000400FBE7DDD001000000AD0B80BD0200CE
:10CFD8007FB500220123CDE9022304ABCDE9043358
:10CFE800094A6B46CDF800D0CDF804D00BF01CFDF3
:10CFF800002805DB4FF480420023684607F062FCF6
:10D0080007B05DF804FB00BF5D8A02000C22104BDC
:10D01800014602FB0033002030B4D3E90E52986376
:10D02800EFF31180202484F31288BFF36F8F1C6CF8
:10D0380004F0C00444F002041C6480F31188BFF3B8
:10D048006F8F1DB12B4630BC0248184730BC704763
:10D05800A0D4002050B9020010B4EFF311822023AD
:10D0680083F31288BFF36F8F1748016841F00204F9
:10D078000460C80707D482F31188BFF36F8F0120BB
:10D0880010BC04F077BA1149D1F80C04D1F80C148B
:10D09800C907F0D5EFF3118083F31288BFF36F8FC0
:10D0A8000B490B6C03F0C00343F002030B6480F3DD
:10D0B8001188BFF36F8F82F31188BFF36F8F002041
:10D0C80010BCFFF7A3BF00BFF0D400200050004001
:10D0D800A0D4002010B1012804D07047034B1B6C6A
:10D0E8005B0701D1FFF792BF704700BFA0D40020B3
:10D0F8002DE9F041012207463449D1E8EF3FC1E864
:10D10800E02F0028F9D133B9314932484B60CB6060
:10D118008A600AF043FA7B1E012B28D8012F06D11A
:10D128002D4BD3F81C3403F00303022B1FD00DF052
:10D13800C6FD0546E8B9294B1B78D3B1022206463D
:10D14800254BC3F80823244CDFF89480D4F818241E
:10D15800D4F81834D20315D503F00303022B01D0F9
:10D16800012F0FD16DB386F31188BFF36F8FBDE820
:10D17800F081EFF31186202383F31288BFF36F8FBA
:10D188000125E0E7C5B130460AF013FCD4F818359C
:10D19800DBB2012BDAD1D4F80421002AD6D0002240
:10D1A800C4F80421D4F804210222C4F81825202246
:10D1B800C8F88021A360C9E70021212008F068F899
:10D1C800E4E70222044BC3F80423D0E79CD40020F0
:10D1D8008CD40020BCD400200050004030E3002054
:10D1E80000E100E008B507480DF0B3FB38B1064888
:10D1F800FFF760FA0448FDF7C7F8002008BD6FF094
:10D208001200FBE78CB9020015D201000A2838B5D4
:10D218000446074D04D1AB680D2128465B68984742
:10D22800AB6803485B68E1B29847204638BD00BF49
:10D238008CB9020038B545682B69B3B1103528465A
:10D2480004F0CCFD044680B90146284604F08AFD66
:10D25800084B98420BD122462846074904F058FD4E
:10D26800224605213120FEF783FF002038BD6FF0EC
:10D278000400FBE70000AD0B85D20100430970B53F
:10D2880007D10B4B596821B101250C68094E85401F
:10D2980001B970BD8A682A4002D030464B68984769
:10D2A8001CB1236821461C46F2E72346FAE700BF73
:10D2B800F4D4002064B902002DE9F04340F20635A9
:10D2C8004668D00648BF0320337B02EA050558BFED
:10D2D800C2F3401087B001F01F07B5F5837F1446ED
:10D2E80047EA43178DF8030041D00FD8062D18D010
:10D2F80007D8B5B1022D3CD06FF0150007B0BDE8D6
:10D30800F083B5F5807FF7D101250AE040F20222CB
:10D31800954230D0B5F5407F2FD0B5F5007FEBD1E1
:10D32800022522032BD5012372688B409360326952
:10D3380062BB07F01F037F0975D13D4A84F4803131
:10D3480002EB8302D2F80032C1F30041C4F3404437
:10D3580023F4E16344EA410423F007031C4344EA4D
:10D36800800444EA0524C2F800420020C6E70725E5
:10D37800D7E70425D5E70525D3E70325D1E76303D8
:10D3880041BF012372688B40D360D0E7103639461D
:10D3980030460DF1020204F0C9FC14F4403F804607
:10D3A8000CD1394630460CF075F9224B9845DCD142
:10D3B80030469DF8021004F01FFDD6E74FF0000933
:10D3C80001AB3946304603AACDE90439CDE90199C4
:10D3D800CDF80C9004F008FB164B98428CD114F44D
:10D3E800003315D09DF8033084F48034C4F300442E
:10D3F8008DF80E3039464B46304603AA8DF80C504E
:10D408008DF80D4004F0ECFB0A4B9842CDD073E741
:10D41800CDE9043339460DF10303304603AA0393DB
:10D4280004F0E2FAF0E7803352F82330FFDE00BF61
:10D43800002584400000AD0BF0B5406801F01F04E2
:10D44800057B87B044EA45140569002D5FD0B2F525
:10D45800001F00F1100506D1214628460CF01CF9E2
:10D46800002007B0F0BD0027B2F5800F01AE01978C
:10D47800776037D1B3F1007F14BF052304238DF8FB
:10D4880004300023CDE904630393836823FA01F190
:10D4980011F0010118D1B2F1A07F15D104F01F03DA
:10D4A800620903F1800338D11D4A52F82330DB07A3
:10D4B8000AD40DF1030632462146284604F036FC0C
:10D4C800184B984219D002962146284603AA04F020
:10D4D8008BFA154B98421DD101222146284604F0AB
:10D4E800A3FCBDE7B3F1C06F05D0B3F1007F14BF53
:10D4F80001230223C3E70323C1E73146284604F08A
:10D5080087FC094B9842DED06FF00B00A9E76FF05B
:10D518008500A6E76FF01500A3E751F82330FFDE7A
:10D52800002584400400AD0B0000AD0B2DE9F04749
:10D5380040F2FF16594FDFF868C1DFF868E100EBE9
:10D548008101814202D10020BDE8F087046814F40B
:10D55800804FC4F3C325C4F3080340F08C80640CE7
:10D56800B34208BF4FF0FF337D5D192C00F286806F
:10D57800DFE804F00D13191C1F251C8484848436ED
:10D588006084848484848484848463787B7EC2F801
:10D598000C355C1C5BD10430D3E7C2F814355C1C35
:10D5A800F9D000245CE0C2F80835F2E7C2F810357B
:10D5B800F5E75C1CC2F80835EDD0002404E05C1CDB
:10D5C800C2F80C35E7D001245FEA531859D14FF05F
:10D5D8000109DFF8CC8009FA03FAC8F80CA008E0C2
:10D5E800C2F80835002DDAD15C1CD4D000240625F9
:10D5F800A146D0F800A00AF40048B8F1000F1CBFFB
:10D608004FF00009012403F01F085B093FD10CEB20
:10D618008808D8F80032CAF3412A03EA0E0343EA1D
:10D628008A0343EA052343EA090343EA4403C8F8A3
:10D638000032B0E7C2F80C35D4E7C2F86035B3F170
:10D64800FF3F0468A7D0C4F30044002CBBD05C099A
:10D658001AD10124DFF8488004FA03F9C8F80890C1
:10D66800A146C6E7C2F86435E9E7C2F86835E6E7D7
:10D67800C2F86C35E3E76FF0150065E76FF08500D9
:10D6880062E70023DB60FFDE00239B60FBE70023EB
:10D6980008F1800853F82830F5E700BF89D1020067
:10D6A80000258440F0F8FCFF2DE9F74306464FF0CB
:10D6B8000008002201210820FEF75AFD0820FEF785
:10D6C80027FD776835693C684146C4F800852E60B7
:10D6D800D7F80C9001AA48460BF01EFA002837DB51
:10D6E800019BD9F8002019791868FFF71FFF002857
:10D6F8002EDB6B7A3169012B03D0032B26D14FF037
:10D708001008AB7A032B21D195F80BC0BCF1000FA0
:10D7180002D0BCF1010F19D12A7A12B1022A15D10F
:10D728000E226B687068B3F5164F00687BD02DD851
:10D73800B3F5165F7AD016D8B3F5966F78D00AD8B5
:10D74800B3F5967F77D0B3F5167F77D06FF0850065
:10D7580003B0BDE8F083B3F5166F72D0B3F5965FEA
:10D76800F4D15C4B3EE0B3F5E14F6DD007D8B3F58B
:10D77800615F6BD0B3F5964FE8D1574B32E047F66F
:10D78800122E7345E2D14FF400032BE0B3F5613F4D
:10D798005ED013D8B3F5963F5DD009D84DF6C02EAC
:10D7A80073455AD0B3F5614FD0D14FF46B0319E0EC
:10D7B800B3F5E13FCAD14FF0EB7313E0B3F5612F36
:10D7C8004ED009D8DFF814E173454CD0B3F5E12FFA
:10D7D800BCD14FF0E86305E0DFF804E17345B5D14B
:10D7E8004FF08053C0F82435736848EA0C081B686A
:10D7F80042EA0802C3F86C250B1DD5E9010183E84C
:10D8080003007B6899073DD505F1180003F040FF38
:10D81800344B98422AD034480121344A09F0D9FFC0
:10D828006FF0040094E74FF41D03DBE7304BD9E7B2
:10D838004FF49E23D6E74FF4A033D3E74FF41C33BD
:10D84800D0E74FF41D23CDE72A4BCBE72A4BC9E796
:10D858004FF06C73C6E7294BC4E74FF46503C1E783
:10D868004FF07063BEE74FF08063BBE7287E04F19A
:10D878000C0204F590710BF068FE01202B7E984095
:10D8880003F0F6FD0823C4F800353B7A53B9C4F811
:10D898001031D4F810316B69C4F834350123C4F859
:10D8A800383523607B6800209A075CBF4FF480738B
:10D8B800C4F804337B68DB0644BF4FF48003C4F824
:10D8C80004332B69C4F844350123C4F84805A36020
:10D8D800E3603DE700B0130000A04E0090D00300C5
:10D8E80040420F000000AD0B38BC020091D102008D
:10D8F8000050270000C0750000F03A0000903A017F
:10D908002DE9F04104460D4607690DF0D8F94FF0AE
:10D918002008B0B92C4B1B789BB1642660680BF0CB
:10D9280029F9F0B901200BF00EFE013EF6D10021D5
:10D93800212007F0ADFCF0E786F31188BFF36F8F65
:10D94800F5E7EFF31186314688F31288BFF36F8F3E
:10D9580060680BF00FF980B986F31188BFF36F8FF9
:10D96800EFE7EFF31186314688F31288BFF36F8F24
:10D9780060680BF0FFF80028DED03B691D70626814
:10D9880038691368C3F844050120C3F84805002026
:10D99800C3F82001D3F82051C3F858015268D3F8CE
:10D9A8005801D20608D5082062681268C2F8000536
:10D9B8004FF48002C3F8042301229A6081F311888E
:10D9C800BFF36F8FBDE8F08130E30020012383406F
:10D9D80070B5DC430B4AD2E8EF1F01EA0405C2E840
:10D9E800E65F002EF7D14FF4803282400648C0F837
:10D9F8000823BFF35F8FBFF36F8F0B4214BF012063
:10DA0800002070BD04D500200050014070B40E49BC
:10DA180022F07F46D1E90034D01AC31844F100043B
:10DA2800C1E90034A6F50013B3F5400F09D2074B3E
:10DA38001B681A0A1B069C19054B42F10005C3E92D
:10DA4800004570BC07F0BABD98CF002008D500206B
:10DA5800A0CF0020D9B101230D4A8340D2E8EFCFEF
:10DA68004CEA030CC2E8E1CF0029F7D14FF4803328
:10DA7800084A8340C2F80433074BD3E8AF3FC3409A
:10DA8800DB0742BF4FF40012044BC3F80021704774
:10DA980004D500200050014000D5002000E100E03E
:10DAA8000D4B1868010A0006BFF35F8F0B4BD3F8C4
:10DAB8000435181841F10001B3F5801F0AD2084B4C
:10DAC800D3E90023904271EB030303D210F1807075
:10DAD80041F10001704700BF08D500200050014007
:10DAE800A0CF00202DE9F04F85B016461F4604460A
:10DAF8009DF840A0FFF76AFF0190FFF7D1FFB04201
:10DB080071EB070352D23B4B301A67EB0101984285
:10DB180071F100014DD2384B03EB0413D3E9022312
:10DB28009F4208BF964258D04FF48038334908FACC
:10DB380004F8204626F07F4BC1F848830BF061F8C3
:10DB48004FF00309584604F15005AD00ADB205F198
:10DB5800804504F5A87305F5A8350293029A20F0CC
:10DB68007F4341F82230C1F84483D1F80435244A70
:10DB7800C01A033820F07F4090422ED9286868B137
:10DB8800D1F80435A3EB0B0020F07F40B0F5000F6F
:10DB9800039322D920460BF034F8039BBAF1000F07
:10DBA80007D109EB030009F10109D7E7BAF1000F22
:10DBB80009D06FF0150520460199FFF74BFF28465D
:10DBC80005B0BDE8F08F01230E4AA340D2E8EF0F5D
:10DBD8001843C2E8E10F0029F8D107490E9823013C
:10DBE800C8500F9B01EB04120025C2E9026753607D
:10DBF800E1E700BF0100800088CF0020005001400D
:10DC0800FDFF7F0000D500207FB500254FF0FF30D5
:10DC18004FF0FF31194C1A4B0226C4F80833C4F8E8
:10DC28004833184BC4F80855C3E902014FF4803350
:10DC38004FF40012C4F80433134B0121C4F80463F1
:10DC48001520C3F880212A46FEF792FA1520FEF720
:10DC58005FFA01230D4AA360236013600C4B0D4A41
:10DC6800009328460023CDE90155FFF73BFF3046D6
:10DC7800FFF73EFA284604B070BD00BF00500140CF
:10DC880003000F0088CF002000E100E004D5002049
:10DC980015DA0100FFFF7F002DE9F7432E4BD3F87B
:10DCA800042390070BD5D3F8042142B10022C3F80E
:10DCB80004212A4AD3F80431136801331360264A31
:10DCC800D2F80433D90326D5254BD3E8EF1F21F02A
:10DCD8000100C3E8E40F002CF7D1CB0702D4D2F837
:10DCE8004031C3B100251C4CC4F84051D4F8403130
:10DCF800FFF7D6FEEFF31182202383F31288BFF3D8
:10DD08006F8F184BD3E90267B042B94106D282F34C
:10DD18001188BFF36F8F03B0BDE8F0834FF0FF3871
:10DD2800D3E900104FF0FF391D60C3E902894FF4B1
:10DD38008033C4F84833C4F84051D4F8403182F3F2
:10DD48001188BFF36F8F0029E5D0009032463B461B
:10DD580028468847DFE700BF0050014008D500206B
:10DD680000D5002088CF002030B5431C124C85B068
:10DD780005D08442A8BF0446012CB8BF0124FFF790
:10DD88008FFE0E4B0C4DD3E90013401AB0F5000F6F
:10DD98000FD22218AA4228BF2A4600205218084942
:10DDA800CDE90100009143F10003FFF79BFE05B0A8
:10DDB80030BD2A46F1E700BFFFFF7F0098CF002063
:10DDC80015DA010008B5FFF76BFE024B1B68C01A95
:10DDD80008BD00BF98CF002070B50546054C064E1B
:10DDE800B44200D370BDD4E90031284698470834BE
:10DDF800F6E700BF2CEA02002CEA020070B5002208
:10DE080001212A20FEF7B4F90B4806F089F90446E7
:10DE180028B101210346094A094809F0E3FC094DE4
:10DE2800094EB54201D3204670BDD5E900312046E0
:10DE380098470835F5E700BF44BE0200CAD1020082
:10DE480020BC02002CEA020044EA0200F0B50F4BA5
:10DE580001461A680E4B0B25002618461F46B84285
:10DE680001D3013D04D11846013A19605A60F0BD4A
:10DE780004688C42FBD03CB14468141BA642BCBF6A
:10DE8800034626460830EAE70346ECE7C8D50020F3
:10DE9800D4D500200020054BC3E90000044BD3E88B
:10DEA800EF2FC3E8E10F0029F9D17047CCD5002046
:10DEB800C8D500202DE9F04788B005460E460CF07D
:10DEC80041FD20B96FF06D0008B0BDE8F0870DF096
:10DED8005AF833680446002B0F4604D107F056F968
:10DEE8006FF00A00F0E7BCBF4FF0FF333360012248
:10DEF800002101A80CF061FEE8460795EFF3118AAE
:10DF0800202383F31288BFF36F8F07F0DFF9FFF741
:10DF18009DFFDFF818914268D9F800309A426CD119
:10DF28000023434D00936B68002B6DD1C5E9008831
:10DF38008AF31188BFF36F8F33685A1C69D04FF486
:10DF4800004E40F2E730002123EAE37C4FF47A7276
:10DF58000023CCFB0E01FAF723FF02460B4601A86B
:10DF680006F0B0FCEFF3118A202383F31288BFF385
:10DF78006F8F00222B685BB1434554D10099002A6A
:10DF88004BD16A6829609A4200D1696000230093E6
:10DF980007F09CF9FFF75AFFD9F8003043608AF37D
:10DFA8001188BFF36F8F0CF0CDFC00288AD035683C
:10DFB8006B1C27D00CF0E7FF4FF47A7EA0FB0E32E3
:10DFC8000EFB0121A4FB0E420EFB0722DB0BE40B28
:10DFD80043EA414344EA42441B1B4FEAD1314FEA2A
:10DFE800E57C61EBD231ED1A6CEB010CBCF1000F52
:10DFF800B8BF002535602DB972E743608AF31188F0
:10E00800BFF36F8F00205FE7C3F80080C5F8048076
:10E018008EE74FF0FF321346A1E711606968994215
:10E0280008BF6A60B2E71A461B68A4E7C8D5002093
:10E03800CCD5002030B404682CB10D4B9C4202D3DF
:10E04800A8339C420BD30B4C2378062B0BD85D1CB2
:10E058002570074C03EB430304EBC303036000681C
:10E0680030BC0CF0AABD6FF00B0030BC704700BF8D
:10E0780020D50020DADD002002682AB1094B9A4237
:10E0880002D314339A4206D3074B1A7832B90122C5
:10E098001A70044B036000680CF00CBD6FF00B00A5
:10E0A800704700BF0CD50020D9DD002038B50546E3
:10E0B8000A4BD3E8EF1F0131C3E8E21F002AF8D169
:10E0C800074B1C6804B938BDE369AB4201D005B100
:10E0D80013B9201D06F0D2FB2468F3E7C8D5002049
:10E0E800CCD5002001460022002301480CF0A9BC31
:10E0F80024D60020014601480CF0ADBC24D60020EF
:10E1080001460022002301480CF09BBC38D60020B1
:10E11800014601480CF09FBC38D6002008B54FF4E2
:10E128008062064906480CF043FCBDE808404FF4FD
:10E138000252044904480CF03BBC00BFDBDD002060
:10E1480024D60020E884002038D6002010B5044BDF
:10E158001C6804B910BD201D06F090FB2468F8E780
:10E16800CCD5002070B50546054C064EB44200D308
:10E1780070BDD4E90031284698470834F6E700BF57
:10E188001CEA02002CEA0200014804F0DFBA00BFD2
:10E198006DE10100292800F099800ADC01284FD0A0
:10E1A800062800F09580002800F08E804FF0FF30A0
:10E1B8007047B0F58D7F04D0B0F5007FF6D11E29E9
:10E1C80048E04B1E142BF1D801A050F823F000BFF3
:10E1D8002FE201002FE201002FE201002FE20100EF
:10E1E8002FE201002FE20100B5E10100B5E10100D5
:10E1F800B5E10100B5E10100B5E101002FE2010040
:10E208002FE2010035E2010039E20100B5E1010029
:10E21800B5E101002DE201003DE2010041E201000B
:10E2280045E201000E210020116070470F21FAE736
:10E238001021F8E71121F6E71221F4E71321F2E79C
:10E2480036293FDC202907DC1429ECD038DC0229E8
:10E25800E9D00429E7D0A9E7A1F12103152BA5D816
:10E2680001A050F823F000BF2FE201002FE20100C7
:10E27800B5E10100B5E10100B5E10100B5E101003A
:10E28800B5E101002FE20100B5E10100B5E10100AF
:10E29800B5E10100B5E10100B5E10100B5E101001A
:10E2A800B5E10100B5E10100B5E101002FE201008F
:10E2B8002FE201002FE201002FE201002FE201000E
:10E2C8001529C7E73D29C5E71F29C3E72029C1E765
:10E2D8003729BFE74FF0FF32064B00201A609A61DA
:10E2E8001A639A641A669A67C3F89020C3F8A8203C
:10E2F800704700BF50D600200B490346087880B904
:10E308000A49097839B1A2F5807102290AD9A2F51A
:10E318008872012A06D9013B022B8CBF00200120FC
:10E3280070470020704700BF5CE200205BE20020DD
:10E3380070B4002318250168084C05FB03F2A658A1
:10E34800B14206D1B0F906100832A01870BC07F027
:10E35800B7BA0133082BF0D170BC704750D60020F3
:10E368002DE9F347074690460C4679B300231A4631
:10E37800C868834234D1802A71D800254FF0FF3213
:10E388004FF0FF3338480AF041FDA946374EE3689D
:10E39800AB422CD800263546DFF8D0A0B14511DDB8
:10E3A80085B96368384601932368A9EB0602009390
:10E3B8000AEB060143460AF02DFD051EEEDD2E444C
:10E3C800B145EEDC28480AF023FD05E009F02FFBF3
:10E3D80016234FF0FF350360284602B0BDE8F087EA
:10E3E800A16801EBC301496801330A44C1E7A36886
:10E3F80006EB090003EBC50253F8351052680CF020
:10E40800CEFFA3684FEAC50A53445B6801359944B7
:10E41800BDE7A3684FEAC60A03EBC6035B683BB1D6
:10E428004FF00009A36803EB0A025268914504D330
:10E438000136E368B342ECD8CEE753F80A106368B4
:10E4480049440193236838460093A2EB09024346E6
:10E458000AF0E0FC011E05DB89440D44E2E70026D2
:10E468003546E6E70D46B7E7C8C80020DBE10020DF
:10E478004FF0FF324FF0FF3370B505460B480AF0F6
:10E48800C5FC002318200A4A00FB03F156588C18D3
:10E49800013605D1555005480AF0BAFC204670BD32
:10E4A8000133082BF0D10024F5E700BF64C8002031
:10E4B80050D6002038B5094D04464FF0FF322846A3
:10E4C8004FF0FF330AF0A2FC00234FF0FF32C4E9FB
:10E4D80000232846BDE838400AF09ABC64C80020EA
:10E4E80010B50446094B0A4A186003680948DA61FE
:10E4F800FEF754FA23680C33D3E8EF1F41F0080104
:10E50800C3E8E21F002AF7D110BD00BF4CD6002097
:10E518002DE6010070BE0200F0B5A1F58173046814
:10E5280087B0032B57D8DFE803F002407753012761
:10E53800D2E9016113683A4AB3F904300492ADF89C
:10E5480014308DF816703368994204D109F06FFAC7
:10E558000C23036014E000F1080528460CF0C8FEFF
:10E568002B460022394630680CF099FE08232046D5
:10E5780000933C22394604AB04F01AFF044610B15C
:10E588004FF0FF340EE0336814333360CDE90200F6
:10E59800284602AA03A90CF0B0FE039B002B18BF63
:10E5A8006FF07704204607B0F0BDD2E90042136847
:10E5B800143313600023CDE9033303AA04A90830F8
:10E5C8000CF09BFE049B0BB1039BE3800024E9E75E
:10E5D80013684360FAE7032912D0042918D1156893
:10E5E80035F4804303D009F022FA1623036004218E
:10E5F8002046C5F3803207B0BDE8F0400BF06CBF91
:10E60800204600220BF068FF840304F48044C9E725
:10E6180009F00DFA16239CE76FF05E04C2E700BF0D
:10E6280039E301002DE9F0410D1E0746904612DA44
:10E6380006F070FD1C4E012333704246384625F023
:10E648004041FEF783F800233370044606F076FD58
:10E658002046BDE8F0816B0003D506F05BFD134E44
:10E66800E9E7FBF7DDFE041E09DB2946424638468A
:10E678000BF0B1FA051E05DA2046FBF725FF4FF02F
:10E68800FF34E5E7FFF7F4FE014638B909F0CFF9A2
:10E698000C230360284604F059FEEDE72046044A9F
:10E6A800FBF7FAFED4E700BF5CE200205BE2002043
:10E6B80078BE02002DE9F04F14460E4600218BB0BB
:10E6C8000546202202A81F4601910CF075FE5CB198
:10E6D80063680293E3680493A3680393236905932B
:10E6E800236A03B1089302AC4FF0FF324FF0FF33B7
:10E6F8003B480AF08BFB31462246284601AB04F022
:10E7080039FB064648B9804681464FF0180A019DF4
:10E7180038604DB901980BF040FA31480AF078FB9F
:10E7280030460BB0BDE8F08F54200CF005FE0446CF
:10E7380000284FD0C0F80090C0F820902B684360A4
:10E74800AB68C3606B688360EB680361D5F804B09D
:10E75800BBF1010F15D108200CF0EEFDE061002897
:10E7680035D00823A3616B695A88A0F800B04280AD
:10E778005B684360B8F1000F2FD13C60A046ED699B
:10E78800C7E7BBF1020F09D00CF0CFFD6FF005060B
:10E7980038680AF02EFB00233B60BBE718200CF01A
:10E7A800CBFDE06198B1C4F818A06A695388111DBF
:10E7B8004380034602F1140C23F804BB51F804EB20
:10E7C800614543F804EBF9D1137D0375D2E7204680
:10E7D8000CF0ABFD6FF00906DAE7C8F80040CDE7AA
:10E7E8008CC800202DE9F04389B007460C46154631
:10E7F800FBF716FE0646002E38681DDBFCB10DB38C
:10E808002B6801AA082B18BF16230DF108090193DC
:10E8180049460BF05AFBB0F100080ADBFFF728FE67
:10E82800074690B909F003F90C230360404604F049
:10E838008DFD3046FBF748FE4FF0FF3618E02246C4
:10E84800A146E5E72A46A946E2E764B15DB1B9F811
:10E858000020012A10D108232B60BDF80A3022803D
:10E868006380039B636039463046164AFBF714FE03
:10E87800304609B0BDE8F083022A17D118232B606F
:10E88800BDF80A3003AD638023460DF11C0C23F854
:10E89800042B2A4603CA624518605960154603F1DD
:10E8A8000803F6D19DF81C302375DCE709F0BFF8A2
:10E8B80086230360404604F049FD3846FFF7FAFD19
:10E8C800B7E700BF78BE020007B5D0E900320121E2
:10E8D80000920348034A08F08FFF03B05DF804FB79
:10E8E80020BC02000DD2020008B5034903480AF013
:10E8F800F7FB6FF0150008BD36D20200D0BB02004E
:10E9080008B5034903480AF0EBFB002008BD00BF27
:10E9180051D20200D0BB02002DE9F74300244FF08A
:10E9280001082546124E30683779D0F81090836870
:10E9380001A95B68984700280CD014DB08FA05F396
:10E948001C430135042D06F10806ECD1204603B01E
:10E95800BDE8F083D9F80020019B08FA07F7534077
:10E968003B42EED0EAE703B0BDE8F043FFF7C8BF8B
:10E97800DCBE02002DE9F041074688460025104E0E
:10E9880027FA05F212F0010210D128FA05F3DB0785
:10E998000ED5317930680AF093FB044640B1094935
:10E9A80009480AF09DFB2046BDE8F0810122F0E706
:10E9B8000135042D06F10806E2D10024F3E700BF73
:10E9C800BCBE020066D20200D0BB02002DE9F843AB
:10E9D800074600264FF001091E4DDFF87C802868A5
:10E9E80047B3404529D0002814BF4FF0E8624FF0E4
:10E9F800986229798368D0F810C09C6904B313021F
:10EA080008D5DCF800C009FA01F313EA0C0F18BFA7
:10EA180082F0C06202F0B05302F0B072A047044620
:10EA280088B1012123460D4A0D4808F0DBFE204637
:10EA3800BDE8F8834FF40012DBE74FF09862D8E79F
:10EA48006FF05704EDE70136042E05F10805C6D12D
:10EA5800EDE700BFDCBE020064B902007CD2020010
:10EA6800D0BB020038B5EFF31185202383F3128859
:10EA7800BFF36F8F0E4C2378ABB90E4B984200D082
:10EA880050B90020FFF7A2FF18B10B490B480AF054
:10EA980027FB00220A4B1A70012321222370094800
:10EAA800002306F00FF985F31188BFF36F8F38BD87
:10EAB8005EE2002064B902009CD20200D0BB0200D2
:10EAC8005DE20020A8CF00202DE9F041334F3B78CC
:10EAD80053B10020FFF77AFF28B131493148BDE82A
:10EAE800F0410AF0FDBA3870FFF716FF04462E4BC6
:10EAF800D3E8EF2FC3E8E14F0029F9D12B4BDFF81A
:10EB0800B0801A7842BBD8F80060A64219D0294BC9
:10EB180066401B680BB1314698474FF0FF334FF002
:10EB2800FF32254805F0C4FD244B1D6835B1043D6E
:10EB38002B683146204698476D68F7E71E4805F070
:10EB48002FFEC8F8004054B1BDE8F0414FF4A4725C
:10EB580000231B4806F0B6B800221A70F1E7EFF35D
:10EB68001186202383F31288BFF36F8F154B1D780E
:10EB7800012D05D086F31188BFF36F8FBDE8F081B2
:10EB880028461C70FFF722FF3D7086F31188BFF3FB
:10EB98006F8F0028F2D00C49A0E700BF5DE200208B
:10EBA800B8D20200D0BB020040D7002064C70020C2
:10EBB80014D7002044D7002018D700202CD70020D5
:10EBC800A8CF00205EE20020D1D2020070B5002557
:10EBD8000B4E4FF4003130460AF05DFA044648B94E
:10EBE8000135042D06F10806F3D1BDE870400F2168
:10EBF800FFF7C0BE034904480AF072FA204670BD08
:10EC0800BCBE0200E9D20200D0BB0200054BD3E82B
:10EC1800AF3F00B10360044811B102685A400A606E
:10EC28000360704740D7002010D700202DE9F84333
:10EC3800384B1860384D39480BF03CFF2E460027FA
:10EC4800A846F388304613F0010F0CBF202110218D
:10EC580041F480310AF01FFA044630B13049314896
:10EC68000AF03EFA2046BDE8F8830137042F06F182
:10EC78000806E6D1064607464FF0010928682979B3
:10EC880083689C693CB100234FF40012A0470446F6
:10EC980020B12549E3E76FF05704FAE72B790136ED
:10ECA80009FA03F3042E47EA030705F10805E5D13D
:10ECB80005461E4E1E4BC6E9013758F835008368D5
:10ECC800DB6933B1012231469847044620B119491E
:10ECD800C5E76FF05704FAE70135042DEDD1164961
:10ECE80016480BF0DCFF0122154B14481A7000235C
:10ECF800002205F0B3FF21462046FFF787FFFFF704
:10ED08000BFE104BD3E8EF2FC3E8E10F0029A9D081
:10ED1800F8E700BF44D70020DCBE020018D7002067
:10ED280003D30200D0BB020020D3020034D7002056
:10ED38006DEA01003BD30200D1EA0100A8CF002010
:10ED48005EE2002040D7002003280A4610B503D908
:10ED5800BDE81040FFF7C8BD074B03EBC0010979B8
:10ED680053F830000AF0ACF9044618B103490448D6
:10ED78000AF0B6F9204610BDBCBE020066D20200F9
:10ED8800D0BB020008B5064803F0DAFC034620B100
:10ED98000121044A044808F025FD002008BD00BFF1
:10EDA800B5ED010063D30200B8BB02002DE9F843BA
:10EDB80004460026244DDFF8949000AF4D4521D33A
:10EDC800EEB12046FAF75EF90022411D00232048E3
:10EDD8000BF037FE054650BB6E4688B06A461D4BA1
:10EDE800C2E905344FF4007393831B4B42F8103F7C
:10EDF8004FF4E45103461948FCF72AFBB546BD46D3
:10EE0800BDE8F88395F8088018F0010F0BD1296840
:10EE180019B120460CF020FB28B118F0020F04D0DD
:10EE280020466B6898470C35C8E70126FBE7214662
:10EE380004300CF0D8FA294609480BF0B3FE09480B
:10EE480005F09EFEDBE700BF84C70020D8C700207E
:10EE58003CC8002090D3020003000001B8BB0200A8
:10EE680050C90020BCC500202DE9F843134E144FAB
:10EE7800DFF8508000220023304605F0CDFC05461F
:10EE8800B8B9BDE8F883237ADA070AD49B0708D40F
:10EE9800216819B148460CF0DFFA10B1484663689A
:10EEA80098470C34BC42EED3294640460BF0D3FDBC
:10EEB800E0E7054C05F10409F4E700BF50C900205C
:10EEC800D8C700203CC8002084C70020094B1B5C21
:10EED80003F00303022B08BF2038C0B2A0F141039E
:10EEE800192B04D9A0F15F035842584170470120FB
:10EEF800704700BFD0E80200A0F12C03DBB2112B51
:10EF08009DBF0348D84000F001000020704700BFB3
:10EF180001400200F8B505460024094E56F8047B66
:10EF28003846FAF7AFF83946024628460CF063FA35
:10EF380020B10134042CF1D10020F8BD0120FCE7F8
:10EF4800FCBE02002DE9F0430468A3B02378804694
:10EF58000E4615460094002B00F0CF80684B1B78B6
:10EF6800062B13D10020621C00921146074612F8A6
:10EF7800010BFFF7ABFF0028F7D107B100910B1B7E
:10EF88002246314628460AF05FF946E0013B082B45
:10EF980043D8DFE803F064495AA20D421C3F05003C
:10EFA80022460021134612F8010B60B10121F9E74E
:10EFB80022460021534F134612F8010B385C10F01B
:10EFC800440F40F0988001B100931B1BD8E76846B6
:10EFD8000AF0A5F80022009B4A481F4613F8011BB7
:10EFE800415C490710D102B100973B1B22463146CC
:10EFF80028460AF029F93B783D2B07D17B783F2B2F
:10F008000BD10237009708E00122E6E73F2B04D135
:10F018000137F7E728460AF0EDF80020009BC8F80A
:10F02800003023B0BDE8F08327463A7810460AF04E
:10F038006DF83B46013708B9002AF6D12246314619
:10F0480028461B1B0AF000F9DCE727463A783B46BE
:10F05800222A07F10107F1D0002AF7D1EEE720466E
:10F068000A2201A906F01CFF0124019B02900093CB
:10F07800009B1878292825D020B303F10109FFF750
:10F088003BFFCDF8009008B9274619E00A2201A9EC
:10F09800484606F005FF22AB671C03EB840444F8DE
:10F0A800800C4846F9F7EEFFDDF804900446484620
:10F0B800F9F7E8FF844206D0202FCDF8009002D05F
:10F0C8003C46D5E72746BB003146284602AA0AF047
:10F0D800DEF8009B013300939FE70A22204602A92D
:10F0E80006F062FE0B460299024600912846314618
:10F0F8000AF095F891E701215DE74FF0FF3090E7BE
:10F1080060E20020D0E8020010B50446F9F7BAFF23
:10F11800012821D923781249CA5C02F00302022A85
:10F1280008BF203B412B17D16378CA5C02F0030269
:10F13800022A08BF203B542B0ED1A27802F0F70315
:10F14800232B0BD0252A09D0104609F0DFFF10B970
:10F15800B2FA82F0400910BD0020FCE70120FAE76E
:10F16800D0E802002DE9F04107460468DFF89081F5
:10F1780000293DD1207809F0BDFF624E054660B3F5
:10F18800062305222046604933700CF034F9F8B1A3
:10F19800052220465D490CF02EF9C8B10B22204605
:10F1A8005B490CF028F998B10A22204659490CF01D
:10F1B80022F968B10B22204657490CF01CF938B1E6
:10F1C8000722204655490CF016F9B0FA80F56D096A
:10F1D80088F8005000203C604EE098F8003053B9A1
:10F1E8002046FFF791FF002848D007233370F1E746
:10F1F80098F800301BB10222424B1A70EAE7002946
:10F2080043DD2246157816462846013209F07EFF6E
:10F218000028F7D13046F9F735FF032830D92B46B7
:10F228003F4A515D01F00301022908BFA5F12003FF
:10F23800412B25D17378D15C01F00301022908BF65
:10F24800203B542B1CD1B378D15C01F00301022977
:10F2580008BF203B2B2B0AD0252B11D1F378D25C89
:10F2680002F00302022A08BF203B582B08D00922CB
:10F278006FF00100234B1A70BDE8F0810223B5E757
:10F28800207809F037FF002836D12278244B9B5C80
:10F298005B070AD42D2A08D02B2A06D0222A07D1A8
:10F2A8000322184B01341A7094E70422154BA4E783
:10F2B800282A04D10122134B14441A708AE71046F5
:10F2C80009F024FF88B10F490B78042B0AD1224694
:10F2D800144612F8010B09F019FF0028F8D105238C
:10F2E8000B7077E7082B3FF475AF1046FFF704FE65
:10F2F80010B10822034B80E74FF0FF30BCE700BF96
:10F308005FE2002060E20020C7D30200CDD30200F4
:10F31800D3D30200DFD30200EAD30200F6D30200FF
:10F32800D0E802002DE9F74F894616461F46804669
:10F33800002800F09980002A00F096805368002B7E
:10F3480000F092800024104609F02FFF42463368EF
:10F35800CDF804809F4228BF1F46454B1C70454B83
:10F368001C701146087809F0D1FE25460132044682
:10F378000028F6D105B101910025DFF8FCB0019B0A
:10F388001A78002A50D0AF424ED91BF802202946DD
:10F39800120748BF013301A848BF0193FFF7E2FEF7
:10F3A800431C41D0023008BF00253246294601A837
:10F3B80008BFCDF80480FFF7C5FD013034D0019AAD
:10F3C8001078FFF799FDB0B1507809F09FFE78B139
:10F3D8000135BD4241D0294601A8FFF7C3FE0130DF
:10F3E80022D03246294601A8FFF7ACFD01301BD0D8
:10F3F800019B01330193019A107809F087FE38B315
:10F408000132117892460846013209F07FFE002841
:10F41800F7D139B1084609F06DFE18B95046FFF723
:10F4280079FDA8B1CDF804A0019DC4B92B78CBB162
:10F438002846FFF76FFD002814BF00206FF00A0070
:10F44800B9F1000F01D0C9F8005003B0BDE8F08F42
:10F458000135BD4208BF012491E70446E4E76FF097
:10F468000600EDE72046EBE76FF01500EDE700BF7B
:10F4780060E200205FE20020D0E8020010B50446F8
:10F4880092B04822002168460BF096FF0D4B216888
:10F498001A6891421A4603D161685B6899420ED096
:10F4A80094E80300012382E803008DF8003002ABE2
:10F4B80094E8030083E80300684600F0EDFD12B00D
:10F4C80010BD00BF4CD700202DE9F74F05230422BB
:10F4D8006E460025CDE90023154FDFF85880DFF888
:10F4E800589056F804BB154BBBF1040F14BF3C46AB
:10F4F8004446204614BFCA469A46F9F7C3FD042875
:10F5080010D121465046F9F7B3FD58B12246594665
:10F518000B4803F021F9034620B10121094A0A48A2
:10F5280009F072FF15B103B0BDE8F08F0125D8E7E7
:10F5380018E300201DE3002004E3002009E3002075
:10F5480021D4020032D40200F0BB020008B50B48F7
:10F5580003F002F9034638B10121094A094809F0C4
:10F5680053FF6FF00D0008BD074803F0F5F80028B9
:10F57800F9D003460221054AF0E700BF5CD4020037
:10F5880067D40200F0BB020021DB02009DD4020018
:10F5980010B5044692B04822002168460BF00CFFD3
:10F5A8000122204602A900F049FE034630B101219C
:10F5B800064A074809F028FF12B010BD0323684621
:10F5C8008DF8003000F068FDF6E700BFD3D40200E4
:10F5D800F0BB02000023064A13601371054A13604A
:10F5E8001371054A13601371044A1360137170474D
:10F5F80013E3002009E300200EE3002004E30020C9
:10F6080010B5044692B04822002168460BF0D4FE9B
:10F61800204602A900F07AFF034630B101210A4AC8
:10F628000A4809F0F1FE12B010BD029B039AA3F537
:10F638009C53083B1343F6D1062368468DF80030E7
:10F6480000F02AFDEFE700BFFAD40200F0BB020089
:10F6580010B5044692B04822002168460BF0ACFE73
:10F66800204602A901F0A0FB034630B10121104A4F
:10F67800104809F0C9FE12B010BD9DF808305A1E96
:10F68800032A01D9072BF6D1DDE90421A2F59C5301
:10F69800083B0B4308D00A4308D00A2368468DF874
:10F6A800003000F0F9FCE6E70823F7E70923F5E75F
:10F6B8002ED50200F0BB020010B5044692B04822D5
:10F6C800002168460BF078FE204602A901F0CAFB2B
:10F6D800034630B10121064A064809F095FE12B0EA
:10F6E80010BD0B2368468DF8003000F0D5FCF6E716
:10F6F8006AD50200F0BB02001FB50024074B4FF487
:10F708008062029302AB009305490E2305480394D7
:10F7180005F03CFA204604B010BD00BF9AD502009F
:10F7280038E7002008D00020072810B5144605D077
:10F7380009280CD0BDE81040FFF74CBF07480BF074
:10F7480052FE21460648BDE810400BF04CBE054865
:10F758000BF049FE21460448F5E700BF13E30020FB
:10F7680009E300200EE3002004E3002010B596B062
:10F7780004464822002104A80BF01EFE00236A4616
:10F7880000938DF8043002938DF80C30204602ABBC
:10F7980006A9F9F781FC034630B101210C4A0D484E
:10F7A80009F032FE16B010BD69469DF8180002AA8D
:10F7B800FFF7BAFF9DF818301BB1074907480BF04F
:10F7C8005EFA022304A88DF8103000F065FCE9E722
:10F7D800A8D50200F0BB0200DCC5002008D000203C
:10F7E80008B550B9054B1B783BB1FFF7F3FEBDE8F0
:10F7F8000840034903480BF042BA08BD22E3002041
:10F80800CCC5002008D0002008B50121034A0448CF
:10F8180009F0F8FD6FF0150008BD00BFC4D502005F
:10F82800F0BB02002DE9F0410025A4B002AF044668
:10F838004822002107F140000BF0BEFD3022294686
:10F8480007F11000BD710BF0B7FD4FF0FF3307F162
:10F858000808C7E90233FB1D009301212046CDF8B3
:10F86800048007F11003BA1D00F034FDB8B16E46EC
:10F878008AB002AA3D4BD461C2E9053040F2013397
:10F8880013843B4B42F8103F4FF411512B46394833
:10F89800FBF7DEFDB5468837BD46BDE8F081BB798C
:10F8A80003F0FB03012B04D1BB69013356D10423B8
:10F8B800BB7100F0BDFB0028EDD12F4ABB79117850
:10F8C800994208D087F8400007F14000137087F884
:10F8D800483000F0E1FB294BB9699A68914203D19D
:10F8E800DB68FA699A421DD00423244D07F11004FD
:10F8F80087F840300FCC0FC50FCC0FC594E80F0028
:10F9080085E80F0007F1480607F110050FCD0FC66F
:10F918000FCD0FC694E80F0086E80F0007F14000EE
:10F9280000F0BAFB164AFB791178994209D0137096
:10F93800052207F1400087F8402087F8483000F09A
:10F94800ABFBBB7903F0FB03012BA4D1BB680133EC
:10F9580008D10C490C480BF092F99CE70B4804F0CD
:10F968008DFFA6E74046FFF789FD94E7DAD5020048
:10F9780004000001F0BB020001E30020D8CF002002
:10F9880023E30020ECC5002008D00020F0C80020A8
:10F9980030B5A5B000214822054668460BF00CFD9D
:10F9A80000F046FB0146A0B9374C2378032B3AD91F
:10F9B80048220DEB02000BF0FFFC607870B130219B
:10F9C8000BF0BEFC044650B9304A0121304809F01A
:10F9D80019FD304804F052FF25B030BD04462946D1
:10F9E800294814AA239400F061FFC11D034607D0DB
:10F9F80001280BD90121284A254809F005FD0BE00B
:10FA08000A230221254A224809F0FEFC072312A8EE
:10FA18008DF8483000F040FB20460BF086FC21981A
:10FA28000BF083FCD5E7284600F0C4FD044630B14E
:10FA380010210BF085FC044608B9194AC5E7284689
:10FA480002A90F9400F0D6FDC21D034607D0012875
:10FA580010D90121104A0E4809F0D6FC10E0022105
:10FA6800104A0B4809F0CEFC0A2302210E4A084826
:10FA780009F0CAFC072368468DF8003000F00CFB3B
:10FA8800002CA6D02046CBE702E3002006D60200D1
:10FA9800F0BB020038C9002094D6020032D602001A
:10FAA800BED60200EBD602005AD6020038B50C4684
:10FAB800054640B931B30846F9F7E4FA082816D0E4
:10FAC8006FF0150012E0F9F7DDFA0828F8D18CB1CB
:10FAD8002046F9F7D7FA0828F2D129460B480BF047
:10FAE80082FC21460A480BF07EFC002038BD074BFB
:10FAF8001D70F6E7294605480BF075FC0022044BFB
:10FB08001A70F2E7014B1970F8E700BF67C70020C9
:10FB180070C7002010B538B31448F9F7B3FA044693
:10FB28001348F9F7AFFA082C15D108280ED1104A56
:10FB38000E49104802F010FE38B1034601210E4864
:10FB48000E4A09F061FC6FF00D0010BD07490C4822
:10FB580002F002FEF0E7082802D105490948F7E754
:10FB6800094802F0F9FDE7E70848FAE767C7002007
:10FB780070C7002012D70200F0BB020059D702005C
:10FB880029D702003BD702004ED702002CDB020027
:10FB98000023F0B58DB00D460646CDE90333CDE917
:10FBA8000633CDE909338DF814308DF820308DF8FF
:10FBB8002C3000285ED000295CD0304CA021204693
:10FBC8002F4A237002F02CFE034648B101212D4A2A
:10FBD8002D4809F019FC6FF00D0420460DB0F0BD5A
:10FBE80020462C210BF0F2FB044648B96FF04C0478
:10FBF800F3E734B90121254A234809F003FCF5E766
:10FC08000C27601C2C210BF0E1FB013F0446F0D1CE
:10FC18000028EFD0811C082203A80BF0FEFB601C13
:10FC28002C210BF0D3FB04460028E3D0811C0822CA
:10FC380006A80BF0F2FB2C21601C0BF0C7FB002878
:10FC4800D8D0811C082209A80BF0E7FB01AB09AA50
:10FC580006A903A800F064FA044630B1034601215E
:10FC68000B4A094809F0D0FBB7E7019B3360029BB8
:10FC78002B60B2E76FF01504AFE700BF61E2002028
:10FC880088D7020095D70200F0BB0200B2D7020065
:10FC9800CCD702004FF0FF3307B5684601A9CDE97C
:10FCA8000033FFF775FF48B14D300AD00121064AED
:10FCB800064803B05DF804EB09F0A4BB6846FFF7FB
:10FCC800DDFB03B05DF804FBF9D70200F0BB0200CE
:10FCD800002208B511460346034802F03DFD0028FE
:10FCE80018BF6FF00D0008BD17D802002DE9F74FB7
:10FCF80005230422CDE90023224B187090B922482D
:10FD080002F02AFD034648B1204A2148012109F0A2
:10FD18007BFB6FF00D0003B0BDE8F08FFFF75AFCD6
:10FD28000020F8E76D4600241A4E1B4FDFF86C8060
:10FD380055F8049B1A4BB9F1040F14BFB246BA46E2
:10FD4800504614BFC3469B46F9F79CF9042813D1C3
:10FD580051465846F9F78CF940B152464946114880
:10FD680002F0FAFC034618B10F4ACEE7FFF7ACFBE6
:10FD7800002CD5D10124DBE749460C4802F0ECFC05
:10FD8800F0E700BF22E300202CD8020038D8020098
:10FD9800F0BB020079C700207EC700200EE30020D8
:10FDA80013E3002063D8020086D8020077D8020047
:10FDB800014B1878FFF79ABF22E30020002313B500
:10FDC80004460193D0B101AB0E490F480DF1020270
:10FDD80002F0ECFD031E08DC0C4801210C4A09F076
:10FDE80013FB6FF00D0002B010BD019B0020013322
:10FDF8000CBF04239DF802302370F4E76FF0150060
:10FE0800F1E700BFB0D80200CDD80200F0BB020075
:10FE1800D7D8020038B5431E062B05460C4608D92C
:10FE28000346124A1248012109F0EEFA6FF0150054
:10FE380038BD042902D90B460E4AF3E70E4B5A5C2B
:10FE48000E4B53F820100E4802F086FC40B10346D2
:10FE5800012107480B4A09F0D7FA6FF00D00E7E7D0
:10FE6800094B1D70094B1C70E2E700BF04D9020062
:10FE7800F0BB020026D902001CDB02000CBF020006
:10FE88004BD9020061D9020066C7002065C700206F
:10FE980013B50446B0B10D490D480DF1060202F044
:10FEA80085FD0128034608D00A4801210A4A09F0BD
:10FEB800ABFA6FF00D0002B010BDBDF8063000209F
:10FEC8002370F8E76FF01500F5E700BF86D9020048
:10FED80091D90200F0BB02009AD90200042838B573
:10FEE800044619D804281CD8DFE800F0240A241B8B
:10FEF80024000123154AAB4013421BD1012D10D118
:10FF0800FFF724FB0346A8B10121114A114809F063
:10FF18007BFA6FF00D0038BDA0F11405EDB2182D75
:10FF2800E7D90C48234601210B4A09F06DFA6FF016
:10FF38001500F0E72146094802F00EFC0028EAD037
:10FF48000121074A034809F05DFAE2E7010C300194
:10FF5800D5D90200F0BB0200FFD902001BDA02006B
:10FF680026DA0200F7B507460124294ED6E8EF3F06
:10FF7800C6E8E24F002AF9D1002B46D10DF107005F
:10FF8800FFF71CFF054660B12146224A224809F0C6
:10FF980039FA6FF00D049DF80600FFF79FFF25461C
:10FFA80029E09DF8073003F0FB03012B23D00DF166
:10FFB8000600FFF76DFF0028EBD1184804F0A8FCF5
:10FFC8002046FFF78BFF04460028E4D19FB14FF08D
:10FFD80096720023114804F075FC10F10B0F0446CB
:10FFE80007D103210E4A0C4809F00CFA6FF073048C
:08FFF800D1E70028CFD100235E
:020000022000DC
:10000000D6E8EF2FC6E8E13F0029F9D1284603B032
:10001000F0BD6FF07605F9E748D700205FDA0200FF
:10002000F0BB0200F0C8002089DA0200014804F0A9
:10003000BBBB00BFA0C80020024B1868B0FA80F01C
:100040004009704754D7002070B50646124D4FF056
:10005000FF324FF0FF33114804F02EFB2C6844B9F7
:1000600008200BF06DF948B9FFF7E0FF6FF068006A
:100070000DE063689E4207D02468F0E704604660A4
:100080006B682BB9C5E90000FFF7D0FF002070BDF9
:1000900018606860F8E700BF54D70020A0C80020AF
:1000A00038B50F4C05462368C3B14FF0FF334FF00E
:1000B000FF320C4804F000FB23680BB11C681BB92D
:1000C000BDE83840FFF7B2BF28465B6898471CB1CF
:1000D000226823461446F2E72246FAE738BD00BFFD
:1000E00054D70020A0C8002070B50E46144605461F
:1000F00000B132B901210A4A0A4809F0A5F90020E5
:1001000070BD1046F8F7C2FFB042F8D8324621461B
:1001100028460BF038F9B0FA80F04009F0E700BF4C
:1001200036DB0200F0BB02002DE9F3411D4600233F
:1001300007460E4614460193F8F7A8FF08281CD17D
:100140003046F8F7A3FF082817D124B12046F8F766
:100150009DFF082811D13288B378ADF80420002122
:10016000022201A88DF8063005F09EFE072809D965
:100170002C4A01212C4809F067F96FF0150002B0F4
:10018000BDE8F081294B022253F820800021F01CA9
:1001900005F08AFEB8F1000F12D14FF0FF332B604B
:1001A0009CB12288A378ADF804200021022201A886
:1001B0008DF8063005F078FE072815D91C4AD8E7D7
:1001C00008FB00F028600130EAD03A88BB78ADF82F
:1001D00004200021022201A88DF8063005F064FEFB
:1001E00007280FD9134AC4E7134B53F820600EB900
:1001F000124ABEE702220021E01C05F055FE7043C2
:100200002860E2E70E4B022253F820400021F81C40
:1002100005F04AFE1CB1444300206C60AFE74FF08C
:10022000FF34F9E75BDC0200F0BB020054BF0200C0
:1002300090DC0200DCDC020074BF0200BCDC0200C7
:1002400074BF02000023F0B585B007460D4602A832
:1002500004211646CDE9023308F098FF044640B168
:1002600003460121184A194809F0F0F8204605B064
:10027000F0BD014602AA384608F063FF044648B1C3
:100280000346134A0121114809F0E0F802A808F0DA
:10029000A7FFEBE7314601AA02A809F053F804468C
:1002A00010B103460B4AEDE7019B1BB1012B03D1B3
:1002B0002B70EBE70346FBE70121074A034809F0EF
:1002C000C5F86FF01504E1E74FDB0200F0BB020058
:1002D000FFDC02002ADD020053DD02002DE9F047B9
:1002E0001D46002390B00393ADF810308DF8123006
:1002F0001646DDE918980722092382460F4605A80D
:100300000B21CDE9002308F041FF044648B1034624
:100310000121784A784809F099F8204610B0BDE8E4
:10032000F087014605AA504608F00BFF044648B185
:100330000346724A0121704809F088F805A808F0C0
:100340004FFFEAE701466B4603AA05A809F026F825
:10035000044610B103466A4AECE76A4A009903A8CA
:10036000FFF7C2FE00284BD00DAAC7F1020105A875
:1003700008F0E8FF041E6AD10D9C052C44DC002C1B
:100380005ADB002E3ED1002D68D125460024B9F15C
:10039000000F43D125F00405012DCFD1B8F1000F96
:1003A000CCD000230825CDE90733CDE90A338DF8F9
:1003B00024308DF830304FF0FF330295C8E9003318
:1003C000002F40F08D8029460DEB050307AA05A8F4
:1003D00008F0E4FF092104460AAA02AB05A808F0C8
:1003E000DDFF50EA04020BD143460AA907A8FFF734
:1003F0009BFE034620B10121434A3F4809F026F8FD
:1004000000249BE73470BEE75A2C15D106B1347036
:10041000002D5AD1B9F1000FF2D05A250AAAC7F11E
:10042000050105A808F08EFF002857D19DF8283057
:10043000002489F80030ADE723460121334A2E48D5
:1004400009F004F86FF015042346314A72E7FBDB2C
:1004500006B13470002D98D05A2C36D005A808F07B
:10046000C0FF032836D9C7F1030101AB0DAA05A8C7
:1004700008F094FF0146D0B9019B102240336B4431
:1004800003F80C0C0DA805F00FFD0923E86001939B
:10049000C7F1040101AB0DAA05A808F07FFF0146D2
:1004A00040B14FF0FF33AB60254604466FE74FF095
:1004B000FF30EAE7019B102240336B4403F80C0C39
:1004C0000DA805F0F1FCA8605FE74FF0FF33C5E928
:1004D00002339FE74FF0FF30E860F4E70023A7E71F
:1004E000072102AB07AA05A808F058FF29460446D1
:1004F00072E700BF4FDB0200F0BB02006FDD0200BD
:100500009CDD0200E4DA0200CCD70200C5DD020067
:10051000D7D80200002373B506460D46CDE9003357
:1005200000293BD0002839D00421684608F02EFE6F
:10053000044640B1034601211A4A1B4808F086FFD1
:10054000204602B070BD01466A46304608F0F9FD0B
:10055000044648B10346154A0121134808F076FFC6
:10056000684608F03DFEEBE72A460221684608F09F
:1005700001FF044610B103460D4AEDE70D49D5E9E8
:10058000003299424FF008039341E9D202210A4A0E
:10059000054808F059FF6FF01504E1E76FF0150406
:1005A000CEE700BF4FDB0200F0BB0200EDDD020032
:1005B0001ADE020000E0995047DE020008B530B9AB
:1005C00001210C4A0C4808F03FFF002008BD002321
:1005D000013810F8012F2C2A01D10133F9E7002A44
:1005E000F7D10A2BF1D9A3F109000523B0FBF3F0F1
:1005F000ECE700BF74DE0200F0BB02002DE9F0431F
:100600000B230D46002107468DB0CDE90911049357
:10061000CDF82B10421E12F8013F2C2B01D10131D5
:10062000F9E7002BF7D185F830304FF0FF33033175
:10063000AB6007A808F0AAFD044648B103460121B3
:10064000974A984808F002FF20460DB0BDE8F083B5
:10065000014607AA384608F074FD044658B1C31D88
:1006600015D00346904A01218E4808F0EFFE07A8F6
:1006700008F0B6FDE8E70646002104AB09AA07A882
:1006800008F08CFE044620B10346884AEBE70126B9
:10069000F2E7874A049909A8FFF726FD002800F031
:1006A000A580012101AA07A808F04CFE04460028F5
:1006B000DDD1019B002B40F0F080022102AA07A8A7
:1006C00008F0ECFE04460028D1D1029B4FF0070849
:1006D000B3F1805FA4BF4FF0FF330293029B03216D
:1006E000AB6005AA03AB07A8CDF80C8008F056FE56
:1006F00004460028BBD1039B0A2130336B4403F826
:100700001C0C2A1D0DF1170008F0A2FE044600285B
:10071000ADD18DF817002A460A2105A808F098FEE9
:1007200004460028A3D1042102AA07A808F0B6FEB7
:10073000044600289BD1029B0521EB6002AA07A872
:1007400008F000FE0446002891D1029B0621AB82EE
:1007500005F1100207A808F0F5FD0446002886D12F
:10076000414605F1280207A808F0B8FD0446002814
:100770007FF47DAF082102AA07A808F0E3FD044634
:1007800000287FF474AF029B09216B8502AA07A899
:1007900008F0D8FD044600287FF469AF029B0A21C7
:1007A000AB8505F1200207A808F0E4FD0446002807
:1007B0007FF45DAF3846FFF701FF85F83000C0B227
:1007C00000EB800000F10B0407A808F00AFE844249
:1007D0000ED2214605F1180207A808F0CBFD044609
:1007E00000287FF444AF95F8303033B900243EE759
:1007F00000220023C5E90623F5E76B6B002BF5D03B
:100800000F274FF0000895F83030984504D3002E9C
:10081000ECD06FF006042AE76A6B391F02EB08126E
:1008200007A808F08FFD4FEA0819044600287FF456
:100830001EAF6A6BF91E4A44083207A808F04EFD45
:10084000044600287FF413AF02AAB91E07A808F0D7
:1008500079FD044600287FF40AAF6B6B029A4B4483
:100860005A81791E02AA07A808F06CFD04460028E8
:100870007FF4FDAE6B6B029A4B449A816A6B3946EA
:100880004A44043207A808F05DFD053704460028F5
:100890007FF4EDAE08F10108B5E70124E7E600BFFB
:1008A0004FDB0200F0BB02009EDE02009CDD020076
:1008B000C2DA020000232DE9F04F16460B220D4646
:1008C0009946A1B002AFC7E90F33BA62F860C7F822
:1008D00043304A1E12F8013F2C2B02D109F10109C5
:1008E000F8E7002BF6D14FF0FF32302409F103086E
:1008F00086F8383086F83030B260F9684978994225
:1009000015D8414607F1340008F040FC0446C0B158
:100910000346AF4A0121AF4808F098FD07F13400C3
:1009200008F05EFC20467C37BD46BDE8F08F04FB36
:1009300003F0F16B013301448A60F16B01448A8258
:10094000DBE7014607F13402284608F0FAFB0446CB
:1009500048B3C31D02D003469F4ADBE7EA468AB08C
:1009600002AA9E4BC2E90705C2E9053840F20243DC
:1009700093849B4B42F8103F00234FF4325195482B
:10098000FAF76AFD0123D5467B61002107F12803B0
:1009900007F13C0207F1340008F000FD044620B1E5
:1009A0000346904AB6E77861EFE78F4AB96A07F1E4
:1009B0003C00FFF799FB386130B901218B4A85482B
:1009C00008F042FD0024A9E7012107F11C0207F10C
:1009D000340008F0B7FC044600289FD1FC69012CC4
:1009E0009CD0022C04D12146814A7A4808F02CFD83
:1009F0004FF0000A0125D046A9F10A037B607B680D
:100A0000AB4203D9FB685B7843450CD87B69002B6C
:100A1000D8D06FF006030121764A6E4808F016FD23
:100A20006FF006047AE705F10109494607F1200253
:100A300007F1340008F032FD044690B16D468AB0EB
:100A400002AA6D4BC2E90780C2E90539052342F8C5
:100A5000103F00234FF421515E48FAF7FDFCAD46EC
:100A60005CE73B6AB3F1805F07DB0221634A5948C8
:100A700008F0ECFC4FF0FF333B623B6A07F12C02BD
:100A80003B650723A91C7B6207F1340007F12403AF
:100A900008F084FC044610B10346594A3AE77B6AE1
:100AA00007F118026033134403F84C0C0A2107F1D4
:100AB0004C0207F12F0008F0CBFC044610B123468E
:100AC000504A27E787F82F000A2107F1480207F16B
:100AD0002C0008F0BDFC04460028F0D107F12002EC
:100AE000E91C07F1340008F0D9FC044638B10121B3
:100AF00000904346444A374806F082FE0EE73B6AC0
:100B000007F12002291D07F134007B6508F01AFC6B
:100B1000044610B103463D4AFCE63B6A07F1600219
:100B2000691D07F13400A7F85C3008F023FC044687
:100B300010B10346364AEDE607F15802A91D07F148
:100B4000340008F0FFFB044610B10346314AE1E6E9
:100B500007F17002E91D07F1340008F0BFFB0446FD
:100B600010B103462C4AD5E607F1720205F10801DF
:100B700007F1340008F0B2FB044610B10346274ADF
:100B8000C8E607F1740205F1090107F1340008F025
:100B9000A5FB044610B10346214ABBE607F16802F3
:100BA00005F10A0107F1340008F0E4FB044610B136
:100BB00003461C4AAEE607F11A0205F10B0107F1E4
:100BC000340008F08BFB044680B30346164AA1E6C6
:100BD000D0DE0200F0BB02009EDE020007DF020052
:100BE000050000019CDD0200C2DA020044DF0200C1
:100BF00063DF02001BE302009ADF0200CCDF020089
:100C00000FE002002FE0020048E002007EE0020058
:100C1000A8E00200DCE00200FEE0020026E10200A3
:100C200046E1020066E102008BE102000C35294634
:100C300007F11A0207F13400B7F91A9008F04EFBD9
:100C4000044610B10346514A64E6B9F1000F00F0C2
:100C50008580B44607F1480EBEE80F00ACE80F00EF
:100C6000BEE80F00ACE80F009EE80F0097F81A905E
:100C70008CE80F00B9F1000F1DD0B9F10A0F15D99A
:100C80000A240A230221424A424808F0DFFB3B695A
:100C90007B61102120460AF057FB48B902213E4AE9
:100CA0003C4808F0D1FB08F10108A8E64C46F0E703
:100CB000706386F830404FF00009BC60BB684B455C
:100CC000F1D0726B691C02EB091207F1340008F0D5
:100CD00039FB4FEA091B044610B103462F4A19E6B7
:100CE000726BA91C5A44083207F1340008F0F6FA76
:100CF000044610B103462A4A0CE607F12002E91C1B
:100D000007F1340008F01EFB044610B10346254AE3
:100D100000E6736B3A6A5B445A81291D07F1200291
:100D200007F1340008F00EFB044610B103461E4ADA
:100D3000F0E5736B3A6A5B449A81726B05355A44ED
:100D40002946043207F1340008F0FCFA044610B1D9
:100D50000346164ADEE509F10109AFE73023F46BDB
:100D600007F1480C03FB0A44BCE80F000FC4BCE8C1
:100D70000F000FC49CE80F0084E80F0096F838308D
:100D80000AF1010A013386F838308CE7AEE102003F
:100D9000D8E10200F0BB020030E2020064E202008F
:100DA00088E20200B2E20200D4E20200F6E20200AF
:100DB0007FB5002306460D46CDE90233002947D012
:100DC000002845D0042102A808F0E0F9044640B10B
:100DD00003460121204A214808F038FB204604B090
:100DE00070BD014602AA304608F0ABF9044630B1A6
:100DF00003461B4A0121194808F028FB18E001218D
:100E00000DF1060202A808F085FA044610B1034667
:100E1000144AEFE7BDF8063002A82B7008F0E1FA9B
:100E2000022809D84FF0FF324FF0FF33C5E9022303
:100E300002A808F0D5F9D1E7022105F1080202A8BD
:100E400008F098FA04460028F2D00346064AD1E793
:100E50006FF01504C2E700BF4FDB0200F0BB0200D9
:100E600047E3020079E30200A2E30200F8B50E4670
:100E70000446F0B1E9B108210F4AFFF735F938B956
:100E80000E4801210E4A08F0DFFA6FF00400F8BDA9
:100E900000250C4F0834214657F8040BF8F7ECF8FE
:100EA00008B93570F3E701350A2DF4D16FF03C0035
:100EB000EDE76FF01500EAE7D7E30200F0BB0200B0
:100EC000E0E302002CBF020070B5064C064EC5B22E
:100ED000B44200D370BDD4E90031284698470834A5
:100EE000F6E700BF1CEA02001CEA020010B5154933
:100EF0001548FEF7DFFD034630B1144A0121BDE875
:100F00001040134806F072BCFEF708FE044610B10C
:100F1000104A0346F2E7FEF7DFFE01210E4801F01A
:100F20001FFC2046FEF7E6FE034608B10B4AE5E744
:100F300001460B4801F014FC034608B1094ADDE7FD
:100F400010BD00BF9FE40200A8E40200B1E402006B
:100F5000F0BB0200D2E40200F2E4020005E5020068
:100F600026E5020031E50200034610B530B10A4A19
:100F70000121BDE81040094806F038BC084B19783B
:100F8000084B1878FEF74AFF034608B1064AEFE718
:100F9000BDE81040FFF7AABF51E50200F0BB020018
:100FA00065C7002066C7002086E50200014610B52F
:100FB000064801F0D5FB034630B1BDE810400121E1
:100FC000034A044806F012BC10BD00BF03D602005D
:100FD000BCE50200F8BB020008B5B0B90B4808F048
:100FE00080FA0B4808F07DFA084808F07AFA0748BA
:100FF00008F077FA054808F074FA044808F071FA26
:10100000BDE80840014808F06CBA08BD65E402007C
:10101000E2E5020010B50749074808F06BFA0446FC
:1010200028B101210346054A054806F0DFFB2046AA
:1010300010BD00BF911202005CD7002008E602003C
:1010400028BC02002DE9F041DFF8D4810D46D8F824
:10105000704000AF072C00F008065BD0132C00F0A6
:10106000A080052C40F0B980D8F854806D496E48B6
:1010700008F03CFA18F4805F41D06C496A4808F0E7
:1010800035FA172418F4006F04D06949664808F04F
:101090002DFA182418F4007F0ED06649624808F033
:1010A00025FA654B18F4004F9B6B04D00121634A6D
:1010B0005D4806F09BFB192418F4806F04D060494A
:1010C000594808F013FA1A2418F4807F19D05D49A2
:1010D000554808F00BFA1B24EB69002E40F09B806A
:1010E000C3F3080222B96FEA53236FEA4323EB618B
:1010F00029462046FAF77CFCBD46BDE8F08116245F
:10110000C0E718F4005FE7D04F49474808F0EEF910
:101110001C24E1E7D8F85C4043484C4908F0E6F964
:10112000600606D5D8F868300121494A3E4806F0E5
:101130005DFBE10705D547493B4808F0D7F9262470
:10114000CAE7A20705D54449374808F0CFF9272454
:10115000C2E7630705D54149334808F0C7F9282499
:10116000BAE7200705D53E492F4808F0BFF92924E2
:10117000B2E7E10605D53B492B4808F0B7F92A2428
:10118000AAE7A20605D53849274808F0AFF92B246D
:10119000A2E723063DD53549234808F0A7F92C24BA
:1011A0009AE7D8F86C8032491F4808F09FF918F088
:1011B000020F03D02F491C4808F098F918F0010FCE
:1011C00003D02D49184808F091F918F0040F83D086
:1011D0002A49154808F08AF97EE7294A294BE8464A
:1011E0008AB00F2CC8BF13466A462749103CC2E993
:1011F00005134FF400731384244BD46142F8103F5D
:1012000000234FF411510848FAF726F90024C54687
:1012100062E7252460E723F4FF7323F0010366E708
:101220005CD7002008CF020028BC02001ECF0200BD
:1012300082CD02002FCF020000ED00E048CF020077
:101240005DCF020078CF0200E2CD020042E602004C
:101250005BE602006BE6020081E602009FE6020008
:10126000BAE60200D7E60200ECE6020006E702005A
:1012700019E7020033E7020063E7020091E702008A
:10128000A5CF020090CF020086D00200040000012A
:1012900000B5104B89B05A6AD86C00929A6A20F057
:1012A00005000192DA6A694602921A6B03925A6B40
:1012B00004929A6B0592DA6B06921A6C1B6D079278
:1012C0009B0748BF40F00400FFF7BCFE09B05DF883
:1012D00004FB00BF5CD700202DE9F0411F46164BF0
:1012E000044693F800800D461646A2B0B8F1000FF0
:1012F00015D1684606F043FB3A4631462846289BFE
:10130000A0470446684606F03BFBB8F1000F02D048
:101310000A4803F049FA204622B0BDE8F0814FF0B8
:10132000FF324FF0FF33054803F0C6F90028E0D044
:101330006FF08304EFE700BF30E30020DCC800203B
:10134000002300B589B0CDE9063303AB0493042331
:1013500003900593A9B10B6806934B68079302238A
:10136000111E18BF01210848CDE9002140F2F531D6
:1013700004AA00F02BF80028B8BF012009B05DF8DE
:1013800004FB0123ECE700BF0501004070B53826DF
:1013900094B006AB05460C463246002118460AF0CA
:1013A0000FF8CDE90454CDE9020654B1012304AA93
:1013B000009200210448019302AA00F007F814B03B
:1013C00070BD2046FBE700BF0001004010B4B1F53E
:1013D000004F029C0ED2042B0CD8042C0AD82404F3
:1013E00044EA0364134644EA0102014610BC034880
:1013F000FFF772BF6FF0800010BC7047217C0100C6
:1014000030B50468ACB1B4FA84F30122C3F11F0310
:10141000DBB29A4024EA0202D0E8EF5FA54204D191
:10142000C0E8EC2FBCF1000FF6D1EAD102480B70F6
:1014300030BD0248FCE700BF0000AD0B0200AD0B61
:1014400010B50368CB40DB0710D401238B40026842
:1014500043EA0201D0E8EF4F944204D1C0E8EC1F08
:10146000BCF1000FF6D1F2D1014810BD0148FCE7F4
:101470000000AD0B0400AD0B014BC3F80405704731
:1014800000700140F7B5044618B1012822D003B01E
:10149000F0BD0222264B0646C3F808230122DA607B
:1014A000C3F80401D3F80431012342F21075204F30
:1014B0008DF80730D4B1012CE9D1D7F80C3403F4FE
:1014C000803386BB002BE2D0012008F040F8013DBC
:1014D000F3D1DCE70022164B0DF10706C3F8080331
:1014E0005860C3F80021D3F80031DDE7D7F818348D
:1014F00003F480333EB9002BC9D0012008F027F84F
:10150000013DF3D1C3E7D7F8182402F0030232708B
:10151000002BBCD09DF807000128B8D108F017F8BF
:10152000013DC7D1B3E7D7F80C2402F00102EEE782
:1015300000500040044B1A7922B9012218601A7138
:101540000248704702487047D0D700200000AD0B1A
:101550000C00AD0B08B5074B1B6833B10520FAF73B
:10156000FDFD10B90520FAF7D7FD0122024BC3F8A3
:10157000182508BDD0D700200050004010B510B18C
:10158000012848D010BD294BD3F81814D3F81824DB
:10159000C90324D502F00303022B05D0012B02D08E
:1015A0000020FFF76FFF0123204A0220C2F8183500
:1015B00008224FF48273002103F1804303F5A04316
:1015C00019601C68012402F1804202F5A0421460F7
:1015D000174A12681AB3154BC3F80403D2E7D3F8BD
:1015E0001424D207DFD5D3F81C2402F00302013AF9
:1015F000012AD5D80E4A12681AB10222C3F8042370
:10160000C0E7D3F80421002AFBD00022C3F804214C
:10161000D3F80431B6E700224FF48073CBE71A68A1
:10162000002AFCD019601B68ACE700BF00500040E6
:10163000D0D7002010B5164BD3F8002152B10020AE
:10164000C3F80001D3F800210122C3F80823114B8D
:101650001B6898470E4BD3F8042182B10022C3F8CF
:101660000421D3F80421D3F81824D3F81824022134
:1016700002F00302012A03D1C3F818159A6010BDC5
:10168000C3F80813034B0120BDE810401B6818473E
:1016900000500040D0D7002001460148FFF7B0BEFF
:1016A000FCC50020036803F01F025B0902600248CA
:1016B00018BF0020704700BF0025844070B432245A
:1016C0000279184B624352FA81F2083233F8124021
:1016D000E10524D5C4F3432124F4F85423F812403F
:1016E00064240026027904FB02340E3434F8025FCD
:1016F00015F4807F03D0C5F34325A9420FD00136EE
:10170000202EF3D164240025624302EBC1029D50D8
:10171000027904FB023070BC5830FFF791BE70BCF8
:10172000704700BF00C6002032235843034B50FAD5
:1017300081F1083133F81100400B704700C60020DA
:1017400032235843054B50FA81F1083133F8110028
:1017500080F00200C0F34000704700BF00C60020C8
:1017600032235843044B50FA81F1083133F8110009
:10177000C0F34010704700BF00C60020024611F0C1
:10178000010004D003490B6A13600B6203B9002007
:10179000704700BF00258440F0B5054600200126B3
:1017A000044607468C420BD1114BD3F87C2132B151
:1017B0000022C3F87C21D3F87C3140F00040F0BD1A
:1017C000E3B29B0003F580729B0806FA03F31D4207
:1017D0000BD002F1804202F54432D2F800C0BCF1D5
:1017E000000F02D01760126818430134DAE700BF17
:1017F000001003402DE9F3470546544B296DD3F8FB
:101800000403C0B240F00040FFF7C6FF061E18DA1E
:1018100000236846E96D00934FF00108FFF7AEFF23
:1018200095F85C30DA0758D4296D4FF00040FFF787
:10183000B3FF6846E96DFFF7A1FF0028F0D126F05D
:1018400000460124002E68D102B0BDE8F08794FA6A
:10185000A4F4B4FA84F4E00804F1080335F8139012
:1018600004F007021DF8003008FA02F223EA02032E
:101870000DF8003001A80194FFF714FF019B4FEA17
:101880009901803350F82370C9F3820A4B07D1467F
:10189000C7F3014725D552462846214607F0BAFE30
:1018A00001A80194FFF7FEFE019BFFB2803350F8C0
:1018B0002330C3F301439F4207D10021204607F0A4
:1018C0009AFE3946204607F096FE01A80194FFF7DC
:1018D000E9FE019B08FA03F30362009C002CB6D1D9
:1018E000A2E7022F0DD10321204607F084FE0AF063
:1018F0000503012BE9D14A462146284607F08AFE16
:10190000E3E70221204607F076FEBAF1030FF2D09A
:10191000032FDAD1BAF1020FECE796FAA6F3B3FA85
:1019200083F304FA03F29B0003F1804303F544338D
:10193000D3F8101526EA0206D3F810252846C2F37C
:101940000142C1F3042107F065FE7BE7001003406C
:1019500032222DE9F3410379214F534353FA81F3A6
:10196000083337F813300546DB070C46CEB234D5C2
:1019700007F06DFE95F8048021464046FFF7F0FE23
:1019800060B121464046FFF7CFFE2A6800B202EB65
:1019900080030022C3F81025C3F8102528462146ED
:1019A000FFF78CFE32222B7901A802FB036600238D
:1019B000083627F816300194FFF774FE019B00EB00
:1019C0008300D0F80022074B134043F00203C0F815
:1019D0000032054802B0BDE8F0810448FAE700BFD4
:1019E00000C60020F0F8FCFF0000AD0B0400AD0BBA
:1019F0002DE9F043D2F8009004460D46164685B016
:101A0000B9F1000F34D032220079DFF8D08142439F
:101A100052FA81F2083238F81230CFB29B0703D560
:101A2000FFF79EFE00283BD100230DF10F02CDE908
:101A300000338DF80E308DF80F300DF10E014B464E
:101A4000284607F08FFD3221237901FB0373083309
:101A500038F8132022F0020228F81320237901FB22
:101A60000377083738F8173043F0010328F81730A8
:101A70007368002B43D04FF0320C22791F780CFB97
:101A800002F2D3F804E052FA85F2544B083233F8EC
:101A90001200E9B210F0020F04D0BEF1000F18D00E
:101AA0004F482FE020F4604020F0200023F812007F
:101AB000BEF1000F0DD0032FF2D872685068226873
:101AC00090F800E002EB8E02FFB9C2F81075C2F880
:101AD00010754FF0320C22790CFB0212083233F8E9
:101AE000120020F01C0023F8120022790CFB0211D6
:101AF000083133F8112042EA870223F81120B36835
:101B000063BB384805B0BDE8F083D2F8108528F0F3
:101B10000308C2F81085226802EB8E00D0F8102569
:101B200022F4473222F44072C0F810252A02D0F87D
:101B3000108502F4F85242EA074242EA0802C0F86D
:101B4000102522790CFB0212083233F8120040EA09
:101B50004E3040F0200023F81200BAE72946D3E9BE
:101B600000872046FFF7AAFDB8F1000FC9D0642313
:101B700020791A4E4343F218F358984504D153681C
:101B80009F4201D100210CE0642303FB00600DF1B2
:101B90000F015830FFF734FC124B9842B2D19DF838
:101BA0000F1064222379534303EBC10346F80380EB
:101BB00023795343322203EBC10333445F6023791B
:101BC000534353FA85F3083336F8132042EA41228F
:101BD00042F4807226F8132093E700BF00C600206D
:101BE0000400AD0B0000AD0B2DE9F04305460C469B
:101BF0001F4685B09AB306793046FFF7A1FD20B1A4
:101C000021463046FFF7ACFD80BB32235E43DFF850
:101C1000FC9056FA84F6083639F816305FFA84F8E4
:101C200013F01C0F02D05378012B1FD001238DF825
:101C30000F3000232046CDE900230DF10F01931C46
:101C4000013207F08FFC32222B7902FB038808F166
:101C5000080839F8183043F0030329F81830002F2A
:101C600051D021462879FFF76BFD18B1284805B0FF
:101C7000BDE8F0833E782B68244903EB8603C3F864
:101C80001005C3F8100532202B794FEA860C434328
:101C900053FA84F3083331F813E0E2B22EF4604EC5
:101CA0002EF0200E21F813E097F801E0BEF1000FAE
:101CB00029D02B68BF789C44DCF810354FEA0E4ED3
:101CC00023F4981323F4F853CCF81035230203F4CB
:101CD000F8530EF4403E3F05DCF8108543EA0E034E
:101CE00007F480173B4343EA0803CCF810352B79FF
:101CF00000FB0322083231F8123043EA463343F046
:101D0000200321F812300348B1E700BF00C60020CD
:101D10000400AD0B0000AD0B30B564250479044B15
:101D200005FB0434A160017905FB0133DA6030BDA5
:101D300000C6002038B505790C462846FFF710FD8F
:101D400058B132235D43064B55FA84F4083433F816
:101D5000143004485B0B137038BD0348FCE700BF28
:101D600000C600200000AD0B0400AD0B2DE9F041D2
:101D7000064607796420184D00FB075898F8604024
:101D800044BB404621464022103009F019FB214651
:101D90003068D8F850608E4212D10023C0F87C31F0
:101DA000D0F87C3140F30730FAF7B6F9642303FB2F
:101DB00007550123094885F86030AB65BDE8F0811F
:101DC000CBB29B0003F580727C2B04BF84508358F8
:101DD0000131E0E70248F1E700C600200000AD0B4A
:101DE0000C00AD0B64210279044B01FB023393F824
:101DF0006000003818BF0120704700BF00C60020F7
:101E000064235422007913FB002302481844FFF78F
:101E100017BB00BF00C6002064235422007913FBC7
:101E2000002302481844FFF7EBBA00BF00C60020A9
:101E300073B503680D46D3F8041306460029A4BF02
:101E40004FF00041C3F80413047929462046FFF7F8
:101E500087FC00B329462046FFF772FCD8B129461B
:101E60002046FFF761FC002501B23468890001F5C6
:101E70008073E550E35833680B44D3F8101541F0F4
:101E80000101C3F8101522B1012332688340C2F862
:101E9000043302B070BD32235C43104B54FA85F416
:101EA000083433F81430C3F38203042B11D0052B0C
:101EB00011D001A80195FFF7F5FB019A0369D34002
:101EC00003F00103991C284602B0BDE8704007F0FA
:101ED00092BB0321F7E70221F5E700BF00C600200F
:101EE0000148FFF787BC00BF64C6002070B5084CEE
:101EF0000E462379154643B92A20FAF70DF9012336
:101F0000044823712660A56070BD0348FCE700BF4C
:101F1000D8D700200000AD0B0C00AD0B002330B56E
:101F20000D4A50F8234003F5A2710133082B42F803
:101F30002140F6D10023084A00F11C0103F5B274D8
:101F400051F8045F0133082B42F82450F6D1036C9A
:101F5000C2F8043330BD00BF00A0024038B50024F1
:101F6000154D2A20C5F81045C5F81445C5F8184583
:101F7000C5F81C45C5F82045C5F82445C5F82845D1
:101F8000C5F82C45C5F89045C5F89445C5F8984561
:101F9000C5F89C45C5F8A045C5F8A445C5F8A845B1
:101FA000C5F8AC45FAF7C6F84FF0FF33C5F808336B
:101FB000024B1C7138BD00BF00A00240D8D70020E2
:101FC0000123024A8340C2F80433704700A0024054
:101FD0000123024A8340C2F80833704700A0024040
:101FE000F8B5012600270B4B0B4DD3F80C4304B971
:101FF000F8BD94FAA4F0B0FA80F006FA00F324EAEF
:102000000304064B82009F502B68002BEFD0A96879
:102010009847ECE700A00240D8D7002000A102407A
:1020200070B503680446033BDBB2052B03D8094AAD
:1020300052F823502DB9A06858B1BDE8704000F0A7
:102040001DB807F07FFB21682B46BDE87040090CE6
:10205000184770BD94BF0200014B5B69184700BF71
:10206000C8C60020014B1B68184700BFC8C6002027
:10207000014B5B68184700BFC8C60020014B1B69B5
:10208000184700BFC8C60020014B9B68184700BF17
:10209000C8C60020014B1B6A184700BFC8C60020F5
:1020A000014B5B6A184700BFC8C60020014B1B6884
:1020B000D8687047E4D70020002230B50B4B196870
:1020C0000C6894420FD001EBC2039D68A8420BD16B
:1020D0004FF003020433D3E8CF1F002903D1C3E834
:1020E000C02F0028F7D130BD0132EAE7FCD700202D
:1020F0002DE9F041002406460F462046DFF85480C3
:102100003368A34201D8BDE8F08106EBC4056B68D3
:10211000DBB2012B16D16A68B8F80030B3EB124F6E
:1021200010D1022FA8680FD1FFF77AFF01206B684A
:1021300023F0FF0343F003036B60B8F80030013372
:10214000A8F800300134DBE70168090C07F0AAFAAF
:10215000ECE700BF38DC002010B5074C02216068B6
:10216000FFF7C6FF0028F9D101212068FFF7C0FF63
:102170000028F3D110BD00BF04D8002070B5072897
:1021800060D8DFE800F00B5F475F435F3C0402F07C
:1021900075F80320BDE87040FBF78CBF03202A4B85
:1021A000D3F81446D3F81866284B1D781870EDB292
:1021B00002F032F8012D10D1254B264A9C4212D054
:1021C000230C1B04B3F1886F0DD0A4F58033203BA2
:1021D000022B0FD96FF0040313603146C4F30B00D8
:1021E00002F00EF800E014601B4B186806F027FDA3
:1021F0000020CFE7194931F913301360F4E70024C8
:10220000124B20461C7002F007F8EDE7FFF7A4FF21
:102210000220BFE70D4B1A78012AD0B20ED1104A26
:102220001168104A8C6854604968116002221A7063
:1022300001F0F2FF084B186806F001FDFFF78CFF74
:102240000120A7E770BD00BF00A0024025E30020E9
:102250000100500500D80020ECD7002038C3020050
:10226000E8D7002004D800200A23F7B54FF47A7588
:102270000C4E0D4F01933168386807F03EFA044662
:1022800040B906F0DAFC40B9012001A9FBF716FEBF
:102290006E30F0D1204603B0F0BD0198684306F0DF
:1022A000C4FCE8E7F0D70020F8D70020054B1B78E6
:1022B0002BB9054B1968054B186807F01EBA0020AA
:1022C000704700BF24E30020F4D70020FCD7002093
:1022D00070B5164B42681B6822F0FF0242F0020202
:1022E000C31A42601248134A0168C3F38913D2E843
:1022F000DF4F651CC2E8D65F002EF8D101EBC301A9
:102300004A6892B242EA04424A600268032002EB41
:10231000C302536823F0FF0343F00103536006F048
:1023200084FC0122044BDA6070BD00BFF4D70020AA
:10233000FCD700203ADC002000A002402DE9F04F3D
:1023400095B038220021064603A809F039F8022387
:102350000493082306932023089304230D9310234A
:1023600040250F9380230122CDE91153D52300216D
:1023700057480B921393FBF761FE0546002840F087
:10238000A380024653493079FFF7B0FD03A8FFF759
:10239000C5FD34686268B2F59D6F40F09280616956
:1023A000E3680B44E16903F59D630B44B3F5003F1B
:1023B00000F287802068294609F002F833681C681B
:1023C000D3F81C9004F53A72019204F16007424A76
:1023D00004F1A40804F1200BB9F1000F5BD1C2F89D
:1023E00000B000254FF0010A2570657084F802A046
:1023F000E570336840461B69636033685B69C4F805
:1024000014B0A360354BC4F81890C3F80080344B67
:10241000E7601F600823C4F8108084F8A43088F8AF
:10242000015088F8025088F8035084F860307D70BD
:10243000BD70FD7007F044F9384607F041F9294BAB
:1024400004F53A721A60284B04F1E80231681A6008
:10245000264B274E1960274B2749C3F81046C3F86F
:102460001456264B264C1D80264B86F800A01D8056
:10247000254B029525601D611B690293029B144B3D
:10248000186806F0DEFB98B103236FF07304337015
:10249000FFF764FD11E09B6904F140096364336850
:1024A0004846DB69C2F800B0236401F0C3FE98E738
:1024B0002468002CECD1154B1C70204615B0BDE8EB
:1024C000F08F6FF01504E3E76FF02D04F5E700BF20
:1024D000ECD700207D210200E8D70020FCD70020A7
:1024E000F8D70020F4D70020F0D70020E4D7002050
:1024F00025E3002000A00240F04902003ADC002061
:1025000000D8002038DC00200056004024E30020E2
:1025100070B5164B42681B6822F0FF0242F00102C0
:10252000C31A42601248134A0168C3F38913D2E800
:10253000DF4F651CC2E8D65F002EF8D101EBC30166
:102540004A6892B242EA04424A600268032002EBFF
:10255000C302536823F0FF0343F00103536006F006
:1025600064FB0122044B5A6070BD00BFF0D700200D
:10257000F8D700203ADC002000A0024010B5FFF799
:1025800073FE012400220321047081704270C27026
:10259000FFF7BEFF054B1C7007F0A5F8BDE8104023
:1025A000034B47F23051186806F04BBB24E3002080
:1025B000ECD7002038B50A4B04461B78022BDDB25D
:1025C0000DD1FFF751FE50B100220121846001704E
:1025D00042708570C270BDE83840FFF799BF38BDC2
:1025E00025E30020034A126812B1002800DB1047DF
:1025F000704700BF18D800202DE9F7430025814619
:102600000F461048294690461E46019303F056FC9B
:10261000041E11DB0134204607F0BDF8C9F80000A4
:1026200068B1334642462146019603F047FC2846EE
:102630003C6003B0BDE8F0836FF01500F9E76FF080
:102640000B00F6E798BC020010B50E4B04461B6861
:10265000A3B1F6F71BFD082810D9237A3F2B0DD024
:1026600009490822204603F065FA014630B904F111
:1026700008000A22BDE8104003F016BC4FF0FF30FE
:1026800010BD00BF18D80020C5E702002DE9F341B6
:1026900005460020174688461E4607F055F80246B4
:1026A00040B915B1284607F078F86FF00B0002B07A
:1026B000BDE8F0816FF05803002403730423056024
:1026C0000E4D037244738473C47344728472C47273
:1026D000C0F80480394603202C7007F051F84FF001
:1026E000FF3301932B78B34201D10020DFE70220B2
:1026F00001A9FBF7E3FB0028F4D0D8E726E300208C
:10270000F8B5054600240F4F57F8046B28463146AC
:1027100008F0A6FE28B90134042CF5D14FF480301E
:102720000DE06CB1A31E012BF8D83046F6F7AEFCD5
:102730000A220021284403F09DFA40EA0440F8BD33
:102740002046FCE7ACBF0200014B18600020704738
:102750001CD80020014B1860704700BF18D800201B
:102760000FB42DE9FF410A9C01F05CFD00284AD01E
:10277000002C4BD0284E294F3168386806F083FA78
:10278000002846D1264D3168286806F05AFA0028FC
:1027900036D122460BAB03A902A80193FFF72CFF09
:1027A000044658B1286806F04AFA386806F069FA13
:1027B000204604B0BDE8F04104B07047029C2046BA
:1027C000FFF742FF02230646012220460399FFF746
:1027D0005DFF04460028E5D1DFF84880D8F8000006
:1027E000FFF78EFF0446D8F8000006F0D0FF2868F7
:1027F00006F025FA002CD8D13046FFF7F3FED4E7D7
:102800006FF00A04D1E74FF0FF34D1E76FF00D0409
:10281000CEE76FF00A04CBE730D8002028D800209C
:102820002CD8002020D800200CB42DE9F04F89B01E
:1028300080460F46129C01F0F5FC002800F0A280B3
:10284000B8F1000F00F0A180002C00F09E80002F56
:1028500000F09E80514DDFF848B12968DBF8000098
:1028600006F011FA002840F096804E4E2968306834
:1028700006F0E7F9002840F08280224613AB07A952
:1028800006A80593FFF7B8FE044618B1306806F0B5
:10289000D6F923E0DDE906930193434B1D68002D33
:1028A00039D00C228246414B1B6802FB0353029332
:1028B000029B9D421CD1BAF1000F2CD0306806F06B
:1028C000BEF94A4639464046D047044618B9404604
:1028D000FFF716FF0446484606F05FFFDBF80000EE
:1028E00006F0CFF9204609B0BDE8F04F02B07047BE
:1028F000AB68A3420DD9019A48469A4228BF1A46AE
:102900002968039303F016F918B9039BD5F804A0BE
:102910001C460C35CCE74846FFF796FE02230546D9
:10292000012248460199FFF7B1FE04460028ADD1C7
:10293000DFF87C904046D9E9004ABA455246214624
:1029400028BF3A4608F02FFDBA45204607D906F0C1
:102950001EFF306806F073F96FF00604BEE7FFF75C
:10296000CFFE0446D9F8000006F011FF306806F0EB
:1029700066F9002CB2D12846FFF734FEAEE76FF0BF
:102980000A04ABE74FF0FF34ACE76FF00D04A9E7A2
:102990006FF01504A6E76FF00A04A3E730D8002013
:1029A00028D800202CD8002010D800200CD80020D7
:1029B00020D800200EB42DE9F343DDF824808146B1
:1029C00001F030FC00285DD0B9F1000F5DD0B8F106
:1029D000000F5AD0304C314F2168386806F053F957
:1029E000002855D12E4E2168306806F02AF90028BB
:1029F00045D14846F6F74AFB451C284606F0CBFE73
:102A0000044668B9306806F01AF96FF00B043868AC
:102A100006F037F9204602B0BDE8F04303B0704736
:102A200049462A4608F0FDFC2046FFF70DFE02232A
:102A30008146012220462946FFF728FE04463068D9
:102A400014B106F0FCF8E2E706F0F9F8B9F1000F6E
:102A5000144D06DB2868FFF753FE10B94846FFF710
:102A6000C1FD0AAA41462868019203F059FA041EE2
:102A7000286808BF6FF04C0406F089FEC7E76FF0C6
:102A80000A04C4E74FF0FF34C4E76FF00D04C1E758
:102A90006FF00A04BEE700BF30D8002028D800201D
:102AA0002CD8002020D8002038B5C3680446A72BB6
:102AB00001D0206810E0032907D0042926D002297C
:102AC00002D10122154B1A7038BD144B00681A78D8
:102AD000022A05D10028F7D0BDE8384006F057BEDD
:102AE0000F4D2A6862B12B689847002320682B603D
:102AF00006F04DFE0B4B1868BDE8384006F09FB855
:102B0000094A1060616851600222DCE7074B1B68CC
:102B1000002BCED000689847CBE700BF26E300200B
:102B200014D800202CD8002020D800201CD8002049
:102B3000012210B511460B48FBF780FA70B90A481C
:102B4000FBF79EFA014648B94FF0FF32074B1A6077
:102B5000BDE8104001230522FFF798BD6FF02D005E
:102B600010BD00BF2CD8002028D8002030D800206D
:102B700010B400F11C03D3E8EF2F511EC3E8E41F8B
:102B8000002CF8D1012A0CDC074BD0E8EF2FC0E86D
:102B9000E13F0029F9D16422002110BC043008F083
:102BA0000FBC10BC704700BF1EF1010010B500241F
:102BB0000A4B4FF45072214609481C7008F000FC83
:102BC00021462246064B074801310829C3E9000285
:102BD0009A6003F16803F7D110BD00BF27E300201E
:102BE00034D800201EF10100164830B500220346FB
:102BF0004FF0FF34144DD0E8EF1FA94204D1C0E8D4
:102C0000EC4FBCF1000FF6D10CBF0121002112D115
:102C1000682101FB023301220C49DA61097893F83B
:102C2000202061F3451283F820200222A3F84820D7
:102C300083F84A2030BD0132082A00F16800DAD159
:102C40000846F7E734D800201EF1010027E30020F2
:102C500030B5024600236825054905FB03F46018DA
:102C60000C59944203D00133082BF6D1002030BD1B
:102C700034D8002010B50446043006F082FF606CA2
:102C800008B1FBF73BFA064BD4E8EF2FC4E8E13F6D
:102C90000029F9D12046BDE81040FFF769BF00BF09
:102CA0001EF1ADDE70B50825064C074E2368B34211
:102CB00002D02046FFF7DEFF013D04F16804F5D1A4
:102CC00070BD00BF34D800201EF101002DE9F8438B
:102CD0000F4C06460025A0464FF068090D4B0E4FDD
:102CE00018702368BB420CD009FB058393F82020A1
:102CF00066F3451283F82020A36B13B1204606F03B
:102D0000AEFD0135082D04F16804EAD1BDE8F88371
:102D100034D8002027E300201EF10100112806DC32
:102D200000280DDB084BC34003F001007047B0F5ED
:102D3000817F07D040F21113C31A5842584170479F
:102D4000002070470120704741000200034B0268D9
:102D50005A6082699A6042691A60704774DB002089
:102D6000012208B511460448FBF768F9002818BF8E
:102D70006FF02D0008BD00BF80DB00202DE9F04F73
:102D800085B082460F4616461D4601F04BFA28B91B
:102D9000012005F04CFF6FF00A041CE05AEA07031B
:102DA00000F051811EB3336823F4A05323F00203D3
:102DB000002B40F04B81706838B9B06878B106F0EC
:102DC00083FE60B96FF0060405E006F077FE002888
:102DD000F3D16FF00504204605B0BDE8F08FF06830
:102DE00028B1B16806F084FE08B96B20D1E79A4B90
:102DF0004FF47A61186805F024FF0446002840F07B
:102E00002881002F64D0F6B1336803F4A053B3F5E2
:102E1000805F18D13368DB0445D44FF0FF3770680A
:102E200008B100F093FD8D4B8D4A1860B368002BFC
:102E300008BF01231360F3688A4A002B08BF0623EA
:102E4000136033681CE00A220021384603F02CF896
:102E50004FF6FE73421E9A4200F2F280824A03024B
:102E600043EA10231380002ED4D1002301217B4A92
:102E70004FF0FF3713607A4A11600621794A1160DA
:102E8000DFF8E8815046C8F80030BAF1000F65D18C
:102E900006F05AFC064600BB6FF009046E4B18683A
:102EA00005F0CDFE97E73A21384608F093FA00B1D5
:102EB000471C38466E4908F0D3FA0A2228B100218F
:102EC000033002F0D7FE0746A9E701463846F8E787
:102ED000654B1880002EC8D09FE707615F4BDFF875
:102EE00080B11B68DFF87CA1B361DBF800303246AB
:102EF000F361DAF8003047F20D013362D8F80030A0
:102F00000420736106F03CFC4FF0FF33594F5A4EDA
:102F100003933E603868B04231D0002840F08C8086
:102F20002020D7F80490FBF7E1F8286070B109F190
:102F300018034D4A019318461288B9F8141006F088
:102F400034FC064638BB2868FBF7D8F86FF0090454
:102F500078680028A2D006F01AFC9FE7F6F796F8EA
:102F600006F0F2FB0646002896D007615046F6F7B9
:102F70008DF851460246306808F015FAAEE7022097
:102F800003A9FAF79BFF0028C4D06E2005F04FFE7E
:102F90006FF00A0482E7D9F808102A6801290AD0DC
:102FA00002291FD01046FBF7A9F83046FBF7A6F818
:102FB0006FF00504CCE708211161D8F8001011F07A
:102FC000020137D00192B9F816000130FBF78EF8F4
:102FD000019A90612A68906930B91046FBF78EF823
:102FE0003046B1E71621E7E7B9F8141009F11803E4
:102FF0000B441946B9F8162008F0D5F900202968C5
:10300000B9F81620896988542A680192D9F808000D
:1030100007F07FFA019A2B685060DBF800205E61B0
:103020009A60DAF80020DA60D8F800201A600022EE
:10303000DA618DE79161E7E707F0B1FA044687E7C7
:103040006FF007042AE76FF00104C4E64FF0FF3485
:10305000C1E66FF00204BEE680DB00208CDB0020BE
:1030600088DB002084DB00203CDC002090DB00209B
:10307000E6E7020074DB0020EEC100BCF8B548F2C0
:103080000F03994205460E4640D022D848F20D0360
:10309000994233D048F20E03994233D00069FFF7CA
:1030A000D7FD044610B3B6F5004F1FD9A6F500466C
:1030B000013E0B2E1AD8DFE816F0AE00E800B6008D
:1030C000B600B6003A013A01B600C4001900190072
:1030D0000B0149F2040399421CD0B1F5104F3FD9BE
:1030E000C068FFF7B5FD0446002848D128680028CD
:1030F00000F02D81BDE8F84006F049BBBDE8F8407E
:10310000FFF724BEBDE8F84006F05CBDBDE8F8401E
:1031100006F045BD0369082B00F21981DFE813F0C2
:103120001000160009000E00160017011701180004
:103130001E000020BDE8F840FFF7C8BD0120F9E7F8
:103140000021E868BDE8F84006F07CBC0121F8E702
:103150000021E868BDE8F84006F080BC0121F8E7EE
:103160000069FFF775FD04460028BFD048F28103CF
:103170009E42BBD10146284600F038FB56E049F29A
:1031800002039E4200F0CD8037D806F0E3FB0746ED
:10319000E0B91020FAF7AAFF0646B8B13946102266
:1031A00008F00EF92B6873606B683381698A002917
:1031B00000F0C8802A8A05F1140006F0F6FAF060E3
:1031C000002840F0BF803046FAF798FF286806F0E4
:1031D000DEFA204606F080FB58B1204606F0BAFB26
:1031E00038B994F8203043F0800384F820300C2361
:1031F000A361204606F075FB18E049F203039E42E6
:103200003DD049F282039E427FF470AF01462846CA
:1032100000F004FB0AE06B692BB9284607F0D9F9E6
:10322000AA6943681A60284607F0D5F9204606F0D7
:10323000A1FB002800F08B802046BDE8F84006F096
:103240000EBB90F8203043F0010380F8203006F0E8
:1032500068FB18B13E4B186805F0F1FC94F820307B
:10326000204623F00A0384F8203006F083FB10B1D7
:10327000204606F0F4FA2046FFF7FCFCD3E7286965
:1032800069280BD16823A361D0E790F82030EE685D
:103290006FF3410380F82030686918B100F06AFBD1
:1032A000A061C3E7204606F026FB28B994F8203039
:1032B00043F0040384F82030204606F01CFB00286D
:1032C000B4D0002EB2D00021204600F0C5FAADE700
:1032D0006B69F3B9284607F07CF9AA6943681A605C
:1032E000426892F8203043F0040382F820304368AB
:1032F00022691A61436862695A6183684BB105F1BA
:10330000180205F1300152F8040B8A4243F8040B0D
:10331000F9D194F82230002B85D0013B84F822307B
:1033200081E790F82230013380F822307EE728468A
:1033300007F04FF96B6913B9AB69436073E74FF05E
:10334000FF33FAE73146204606F0A6FA6EE7F8BDED
:1033500094DB002030B585B00546FFF779FC0446C4
:1033600028B9092005F063FC4FF0FF300EE000F0B3
:1033700059FF68B9204606F0D4FA18B10D4B186809
:1033800005F05DFC2046FFF775FC002005B030BD60
:10339000002006F0D9F9014608B96920E2E7056185
:1033A00001AA47F2090000F0FDFA0028EDD0162826
:1033B000EBD0D7E794DB00202DE9F04385B08146C0
:1033C000884615461C460C9FFFF742FC40B9092071
:1033D00005F02DFC4FF0FF33184605B0BDE8F08333
:1033E00014B90FB11620F3E7B8F1290F00F0ED8002
:1033F0000CDCB8F1010F12D0B8F1060F00F0E1803B
:10340000B8F1000F00F0DF806D20E1E7B8F58D7FA7
:1034100000F08880B8F5007FF6D11E2D08E03D2D24
:10342000F2DC202D0EDC142D4ED0152D53D0022DA4
:10343000EAD1384606F088F90646002840F0C780F1
:103440006920C5E7A5F121031C2BDDD801A252F8A4
:1034500023F000BF33340200333402000934020089
:103460000934020009340200093402000934020060
:103470003334020009340200093402000934020026
:103480000934020009340200093402000934020040
:103490000934020009340200F3340200FB34020054
:1034A000FF34020003350200133502000934020024
:1034B0000934020009340200093402000934020010
:1034C000E5340200173502003A46214605B0BDE852
:1034D000F04307F084B83A46214605B0BDE8F04312
:1034E00007F08BB83A46214605B0BDE8F04307F037
:1034F00092B801230422019305E00223FAE7032393
:10350000F8E7042201920DEB020107F0A4F803464C
:1035100062E70523EEE73A46214605B0BDE8F043F1
:1035200007F099B86B1E112B3FF66EAF01A252F84F
:1035300023F000BF8B350200B535020033340200A2
:1035400009340200A73502007D350200093402006B
:10355000093402000934020009340200093402006F
:103560009935020033340200333402003334020050
:103570000934020033340200333402003A46214653
:1035800005B0BDE8F04307F089B83A46214605B0DA
:10359000BDE8F04307F096B83A46214605B0BDE8CD
:1035A000F04307F0A4B83A46214605B0BDE8F04321
:1035B00007F0AFB83A46214605B0BDE8F04307F042
:1035C000B7B8372D34E71F2D32E7202D30E7002321
:1035D0000822437202728372C372C0F81090404690
:1035E00006F0C0FF7061284600F0B8F9B06124B160
:1035F0003A462146306807F0D6FE314647F20300CE
:10360000776001AA00F0CEF9034600283FF4E4AE4B
:10361000DEE600BF2DE9F04385B0814688461746B7
:103620001D460C9EFFF714FB40B9092005F0FFFA78
:103630004FF0FF37384605B0BDE8F08305B10EB94D
:103640000E20F3E7B8F1290F00F08F800CDCB8F101
:10365000010F11D0B8F1060F00F08380B8F1000F10
:1036600000F081806D20E1E7B8F58D7F2AD0B8F5B4
:10367000007FF7D11E2F0EE0152F1CD00ADC042F7F
:1036800012D0142FEED13246294605B0BDE8F043E2
:1036900007F085B8212FE5D1306806F055F80446CB
:1036A000002864D16920C1E73246294605B0BDE84B
:1036B000F04307F064B83246294605B0BDE8F04350
:1036C00007F07CB87A1E122ACCD801A151F822F05A
:1036D000473702005537020099360200993602003A
:1036E000393702001D3702006536020065360200D8
:1036F0006536020065360200653602002B3702008F
:1037000065360200993602009936020099360200A9
:1037100065360200653602009936020032462946B7
:1037200005B0BDE8F04307F058B83246294605B069
:10373000BDE8F04307F063B83246294605B0BDE85E
:10374000F04307F06EB83246294605B0BDE8F043B5
:1037500007F079B83246294605B0BDE8F04307F0D6
:1037600084B8372F97E71F2F95E7202F93E7002383
:103770000822437202728372C372C0F810904046EE
:1037800006F0F0FE6061384600F0E8F82146A061DE
:1037900001AA47F20400D4F8008000F003F90746BC
:1037A00020B1404605F0F9FF38463FE762683368CC
:1037B00041469A4228BF1A462846326007F0F3FD78
:1037C000404605F0EAFF35E708B5FFF7EFF9FFF7E8
:1037D000C7FA40B9012204481146FAF72FFC002825
:1037E00018BF6FF02D0008BD94DB002010B54369B1
:1037F0000C467BB191F820306FF3C30381F8203081
:10380000406900F0B7F8044BA061BDE810401868AB
:1038100005F015BA10BD00BF94DB002010B591F87B
:1038200020300C466FF3C30381F82030006960B983
:10383000DBB223F0140343F0140381F82030054B6E
:10384000BDE81040186805F0FAB900F093F8A061DF
:10385000F5E700BF94DB00202DE9F341DFF8E880B5
:103860000546D8F80000019105F0EBF9074650B184
:10387000019B002B65D11023AB614FF0FF37384619
:1038800002B0BDE8F081686CA8B1F5F7FFFB461CFB
:10389000304605F059FF044678B9284606F046F848
:1038A00008B16923AB61D8F8000005F0C8F96920B8
:1038B00005F0BDF9E1E73E46EAE72B680422036123
:1038C0000023027243728372C37295F84B2005F194
:1038D0004801013292008260143007F064FDF6B1B5
:1038E0003246696C206807F09CFD666095F82030D0
:1038F000042043F00803224647F2810185F8203076
:1039000005F03EFF284606F011F80028B7D12846FA
:1039100006F007F840B9A8690028B0D0C8E72670BB
:103920006670A670E670E0E7022001A9FAF7C6FA11
:1039300010F10B0F05D00028E9D00028B8BF404295
:10394000B6E77420B4E700BF94DB002003289CBFD7
:10395000014B1856704700BFEAE7020002383528CD
:103960009ABF034B53F820004FF0FF30704700BF61
:1039700094C1020070289ABF024B53F820000248FD
:10398000704700BFD0BF0200ADBAADBA01380428FD
:103990009ABF034B53F820004FF0FF30704700BF31
:1039A000BCBF02004FF0FF3337B50D4DCA6014465F
:1039B00015600A4601460420019305F0E1FE2068E7
:1039C000A84202D0FFF7D6FF08E0022001A9FAF7CB
:1039D00075FA0028F3D00028B8BF404203B030BDCC
:1039E000EEC100BC431C07D0064B984207D83C23CD
:1039F000B0FBF3F080B270474FF6FF7070474FF6A0
:103A0000FE70704787FF3B002DE9F34105460E46E7
:103A1000144600F007FC002800F0C1800023614F2D
:103A20003246294607207B6005F0AAFE4FF0FF339F
:103A30000193022001A9FAF741FAD7F8048006465B
:103A4000B8F1000F06D110F16E0FF2D1304602B07E
:103A5000BDE8F08110F16E0FF8D0D8F80450022DB7
:103A600000F0948047F6FF739D4200F09280002D95
:103A700040F0928044B142F209023B88934209D05F
:103A800042F20912934240D078680028DED005F057
:103A90007EFEDBE74FF443722946204607F090FC98
:103AA000B8F8083001222360D8F80A01FFF79AFF1E
:103AB000A080D8F80E01FFF795FFE080D8F812013A
:103AC000FFF790FF2081D8F81601FFF78BFF608188
:103AD000D8F81A01FFF786FF20231546A081A373AB
:103AE000511E2274657408EB8101D1F80A00FFF7BA
:103AF00079FF6082D1F88A00FFF774FF0132212A32
:103B0000A08204F10604EBD1BEE7294620464FF41B
:103B1000437207F055FC0621B8F80830103444F819
:103B2000103CB8F80A3024F80C3CB8F80C3024F8F3
:103B30000A3CB8F80E3024F8083CB8F8103024F8E5
:103B4000063CB8F8123024F8043C98F8143004F815
:103B5000023C08F1150398F814200633954204F14D
:103B6000060491DA13F8062C04F8062C13F8052C39
:103B700004F8052C01FB0582B2F81700013524F882
:103B8000040CB2F8192024F8022CE4E76FF00C06BC
:103B90007AE76FF05E0677E76FF0150674E74FF08F
:103BA000FF3653E7A8DB002070B50446002800F07C
:103BB0000881022A00F0B980032A00F0C480012A9B
:103BC00040F0FF80E72940F2FF80824D2B68002BF8
:103BD00000F0FD80FEF75EFAE8220021204607F0A3
:103BE000EFFB7D4B1B78032B2B6858689968C4E961
:103BF0000001D8681969C4E902015A6922619A6909
:103C00006261DA69A2611A6AE2615A6A22629A6A98
:103C10006262DA6AA2621A6BE2625A6B226393F8FA
:103C2000512084F85020D3F841202264D3F8452055
:103C30006264D3F84920A264D3F84D20E2641A8F5D
:103C4000A28693F83A2084F8362093F83B2084F833
:103C5000372093F83C2084F8382093F83D2084F8EE
:103C6000392093F83E2084F83A20B3F83F20A28709
:103C700032D1D3F852200A25C4F8E420002252346D
:103C800003F1590193F85600824205DA0C2A04F137
:103C90000C0401F10A0103D1FEF702FA002070BD05
:103CA00005FB0230B0F85760013224F80C6C11F8B3
:103CB0000A6C04F80A6CB0F85A6024F8086CB0F981
:103CC0005C6024F8066CB0F95E0024F8040C11F86E
:103CD000030C04F8020CD5E7D3F8CA201946C4F83F
:103CE000E4200A26002206FB0230B0F852500132CE
:103CF000A4F8525091F854500C2A84F85450B0F85B
:103D0000555004F10C04A4F84A50B0F9575001F191
:103D10000A01A4F84C50B0F95900A4F84E0091F8EB
:103D2000510084F85000DED1B6E752294CD92B4D12
:103D30002B68002B4BD0FEF7ADF9532220462968A3
:103D400007F031FBA8E767293ED9254D2B68002BEA
:103D50003DD0FEF79FF9234B1B78012B23D168221E
:103D60000021204607F02CFB0022296808340B882C
:103D7000C81C44F8083C8B7804F8043C8B78183451
:103D80009A4289DA02EB0213C55C0B4404F8185C12
:103D90005E6853F8085F013244E904655D689B681A
:103DA00044E90253EAE72B681A8922600122227152
:103DB000227200221968C4E904125B68C4E9063261
:103DC0006AE76FF015006AE76FF0790067E76FF058
:103DD000220064E7A4DB002029E30020A0DB002010
:103DE0009CDB002028E300202DE9F04100F01AFAC6
:103DF000054600285FD0314E4FF0FF31306804F0A7
:103E000020FF044600284DD12D4C2378B3BB00F091
:103E100009FA002849D100F005FAA8B14FF00208CC
:103E20004746152006F03DFD014650B105220368C6
:103E300041F204001A71C3F805700022FFF7E4FD97
:103E400018B1B8F1020FE6D1002500F0EBF9A8B1E6
:103E5000152006F026FD014680B1036800226FF0B0
:103E60007F00012718715A7141F203209A71DA71AB
:103E70009F74FFF7C9FD0DB100B92770152006F03A
:103E800010FD0146A0B101250368002241F20400A3
:103E90001D71FFF7B9FD044608B90A4B1D70306863
:103EA00004F0CDFE2046BDE8F0810327B846B8E710
:103EB0006FF00B04F3E74FF0FF34F3E7B0DB0020C3
:103EC0002BE300202CE30020014B186000207047FA
:103ED00098DB00202DE9F041056807460C463DB10E
:103EE00001F47043B3F5005F04D1404BC3E9001502
:103EF000BDE8F0813E4E336863B144F20402914262
:103F000064D00CD844F2020399424ED044F2030329
:103F1000994253D03868BDE8F04105F038BC44F20E
:103F2000012221F4807393420FD044F2031399428B
:103F3000F0D1304C206808B105F029FC01222E4B4D
:103F40001A7025600420336826E0DFF8B080D8F8C6
:103F5000000008B105F01BFC44F201339C420CBF89
:103F60000322022295F85170254B264C1A70C8F88E
:103F7000005017F008053368227810D01AB90520D0
:103F800098470123237007F04107012F02D1022037
:103F90003368984701203368BDE8F0411847002A8C
:103FA000F1D0062098472570EDE7174C206808B13E
:103FB00005F0EDFB032033682560EDE70D4C20682C
:103FC00008B105F0E4FB00220B4BB9E72A78032A7D
:103FD000A0D8DFE802F0020507090720984799E713
:103FE0000820FBE70920F9E70A20F7E7A8DB002013
:103FF00098DB00209CDB002028E30020A4DB0020CD
:1040000029E300202AE30020A0DB002008B50023DC
:10401000094A0A4813700A4A13700A4A13700A4A76
:1040200013700A4A136001221146FAF707F80028B4
:1040300018BF6FF02D0008BD2AE30020B0DB002080
:104040002CE300202BE3002029E3002098DB002054
:1040500010B50B4C206818B105F099FB00232360C4
:10406000084C206818B105F092FB00232360064C31
:10407000206818B105F08BFB00232360002010BDE1
:10408000A4DB0020A0DB00209CDB002030B4074B29
:104090001C6844B143688589A4460268C1899BB203
:1040A000E8B230BC604730BC704700BFB4DB0020D2
:1040B00037B50125074C4FF4FA70656104F0B5FD82
:1040C000002363610193256123690193019B03B080
:1040D00030BD00BF0056004030B50D4D89B0036AB9
:1040E00003AC01908DF808300FCD0FC42B6801A8E8
:1040F000236005F0E3FA40B9044603AD55F8043BEC
:10410000984710B90134052CF8D109B030BD00BF73
:104110005CBC0200034BD3E8EF2FC3E8E10F00299A
:10412000F9D17047B8DB002038B50546002850D0DB
:10413000436A002B50D0836A002B4DD00124294BB9
:10414000D3E8EF2F002A03D1C3E8E14F0029F7D1CC
:1041500045D1686A00F04EF8F9F7E4FF224BC82019
:104160009C6604F062FD2846FFF7B6FF044640B99E
:1041700001221D4B0220DA66FFF7CCFF0024204607
:1041800038BDFFF795FF002C11DBAB6A204698473E
:10419000164B9C421AD013DCA4F18864033C012C1A
:1041A00011D82846FFF798FF04460028E0D00122E6
:1041B0000D4BDA66F9F7CEFF0020FFF7ABFFDEE725
:1041C0000B4B9C42EDD06FF00404F0E76FF00A0453
:1041D000EDE76FF00D04D2E76FF01504CFE74FF075
:1041E000FF34CCE7B8DB002000500040050040045D
:1041F00001005005014B1860704700BFBCDB002078
:1042000007B5044BCDE900011B686846984703B029
:104210005DF804FBBCDB0020014B1870704700BF49
:104220002DE30020024B1878431E58425841704736
:104230002DE300200021074B01221970064B197055
:10424000064B1960064B1960064B18600648F9F7D3
:10425000F5BE00BF2EE300202FE30020C4DB0020CA
:10426000C8DB0020D8DB0020C0DB0020024B186830
:1042700008B104F0E4BC7047C0DB002070B4284BE8
:104280001B68196958691A7C00221A745C7C5A747C
:104290009C7C9A74DC7CDA741C7D1A755C7D5A7582
:1042A0009C7D03299A75DC7DDA7529D0042929D0F3
:1042B00001290FD185681B4E954210D11A7A012130
:1042C00000221972597A5A72997A9A72DA7A6FF0D0
:1042D0005F02DA72144B70BC186804F0B0BC911C19
:1042E00000EB81014C682178622907D0633918BF3F
:1042F0000121490046F821400132DDE70121F9E7BB
:10430000187ADEE7187A1972597A5A72997A9A727B
:10431000DA7A6FF05F02DA720122044B1A70D9E781
:10432000D8DB0020CCDB0020C0DB00202FE3002006
:10433000014B986864307047DCDB002010B5044600
:10434000F6F7AAFF03480121034A03F046FA204684
:1043500006F00EFB28BC0200EEE702002DE9F84350
:1043600004460D4600AFEFF31188202383F3128833
:10437000BFF36F8F0428294A98BF294BE9468AB0BA
:104380009668117C98BF53F820306A4688BF254B49
:10439000C2E9073140F2013323489384234BC2E939
:1043A000050442F8103F00234FF431512048F7F73D
:1043B00053F8CD4645B1EB69C3F3080323B101219E
:1043C0001C4A1B4803F009FA2EB1304606F084FC63
:1043D00008B1037803B91848E9468AB06A46174B12
:1043E000D061C2E9053640F201331384144B42F820
:1043F000103F00234FF411510D48F7F72DF82946CF
:10440000CD462046FFF79AFF88F31188BFF36F8FE0
:104410003046F7F7FDFDBD46BDE8F883DCDB002044
:104420006CC20200FDE7020013E802000500000173
:1044300028BC02003BE802000BE802005CE8020036
:104440000400000138B5094B53F82040013053F8FF
:104450002050A54200D838BD636823B1204606F03D
:104460008FFA0834F5E723689847FAE780C202001C
:10447000012270B5294B032086B01A70FFF7E2FFC6
:10448000F7F7A8FA0420FFF7DDFF254C254D264657
:10449000AE4204F1300410D300F040FE204C224E16
:1044A000AC4226D300F04EFEF5F794FA1F4A137B78
:1044B00023F00103137306B070BD54F80C3C059350
:1044C00054F8103C049354F8143C039354F8183CEB
:1044D000029354F81C3C019354F8203C009354E997
:1044E0000A2354E90C0100F0F7FB54F8303C5E65F8
:1044F000CDE7D4E90A23B3F1FF3F08BFB2F1FF3F94
:1045000005D052EA0301206803D106F0E7FB3034FE
:10451000C6E73146183000F0DBFFF8E730E3002053
:10452000A8BB0200A8BB02001DAE020038D10020CB
:1045300008B50348034A0021121A06F039FA08BDEB
:10454000D8C9002034E30020882370B5134E01221F
:1045500003FB0066002386B0CDE904230F220193FC
:10456000CDE9023214234FF4A0720D4D0D4903FB27
:104570000055044602FB00110B4B3046009500F03D
:10458000ABFB737B2C7423F004037373074B013470
:1045900003EBC423EE606B6006B070BDB0D00020AA
:1045A000DCDB002038F3002097AA020038EB002063
:1045B000BFB50020FFF746FF2E4B03F5006282F3E4
:1045C000088883F30A880024E0232B4D2B4E85F8BE
:1045D0002230EC772C766C76AC7685F820406B6ACE
:1045E000274F43F4E0236B6285F82340F7F792FCF2
:1045F000F7F732FE4FF0FF33AB62EB62F7F7D0FF15
:10460000F7F74EFEF6F7B8FD40F201131D4D2846B0
:10461000AB81C5E91A4401F087F9B56006F09CF951
:104620000120FFF70FFF0220174DFFF70BFF00F0EF
:10463000A9FD164B75610593012315494FF480526E
:10464000CDE9034328463B46CDE90144009400F000
:1046500043FB06466A7B284622F004026A7306F092
:1046600082FB2046FFF770FF3A4631462846F7F7AF
:10467000D5FD00BF38EB002000ED00E0DCDB0020C2
:104680007144020068D2002038D10020BEE8020048
:1046900078F4002038B5064C064DAC4201D300201A
:1046A00038BD2046D4E9011206F086F91434F4E747
:1046B00028C8002050C800202DE9F34104461746C1
:1046C0001E46EFF31188202383F31288BFF36F8F08
:1046D000C368334A7BB180689168884219D057EA31
:1046E000060318D188F31188BFF36F8F6FF00F00A6
:1046F00002B0BDE8F081916891F90E100133E360DA
:1047000093682161A36088F31188BFF36F8F002045
:10471000EEE72169F2E791F90E1090F90E306FF093
:104720007E029942A8BF19469142B8BF11468B42FA
:104730002DDD06F0BBF9054622464146CDE900765F
:10474000184800F037FC0028E1D0EFF31186202351
:1047500083F31288BFF36F8FA068D0B123682169FB
:104760009C420AD04BB193F90E309942A8BF19462A
:104770006FF07E039942B8BF194606F097F940B131
:104780003146084800F086FC6FF00A00B0E70025CB
:10479000D2E7002DF4D186F31188BFF36F8FF3E7D2
:1047A000DCDB002031E3002038B58368044663B3C6
:1047B000194A926893422BD1C368012B03D9013B5C
:1047C000C360002038BDEFF31185202383F31288E6
:1047D000BFF36F8F0169806806F068F9204606F024
:1047E00037FBA06058B190F90E2022610022C26709
:1047F00006F0B9FA2946094800F04CFCE1E7E06010
:1048000085F31188BFF36F8FDBE76FF01500D9E7F1
:104810004FF0FF30D6E700BFDCDB002031E30020A3
:1048200037B51146EFF31185202282F31288BFF3CA
:104830006F8F04689CB12368426823F0030394429D
:10484000036008BF43600121204606F0A3F9044637
:1048500085F31188BFF36F8F204603B030BD51EA56
:104860000302F5D000F10802CDE9001310462946F5
:1048700000F0A0FB0028EFD1014B9B685C69EBE7DF
:10488000DCDB002038B50446EFF31185202383F3E9
:104890001288BFF36F8F06F0DBFA48B10022C267BF
:1048A00006F061FA2946BDE83840074800F0F2BB3F
:1048B000D4E902329A4218BF01330221A36004F105
:1048C000100006F0FFFCEDE731E3002013B5EFF335
:1048D0001181202484F31288BFF36F8F846844B160
:1048E000013C846081F31188BFF36F8F002002B018
:1048F00010BD52EA030406D181F31188BFF36F8F14
:104900006FF00F00F3E7CDE900230246014800F005
:1049100051FBECE731E3002070B50446EFF311855D
:10492000202383F31288BFF36F8F6FF00A062046AF
:1049300006F08EFA18B1C66706F015FAF7E7A06020
:10494000022104F1100006F0BDFC2946BDE87040CC
:10495000014800F09FBB00BF31E300201FB5094AAA
:1049600002AB92E803004FF4906283E803000093E7
:1049700005494FF0FF33054800F00CF9002005B061
:104980005DF804FB84BC020078040120C0D1002043
:104990002DE9F04305464FF0FF364FF0FF37DFF8C3
:1049A0002C8185B0EFF31189202383F31288BFF3A4
:1049B0006F8FD5F888408CB9022105F1A00006F070
:1049C00010F9002860D100234946CDE90067029321
:1049D00005F190023E4800F083FCE3E7D5F88C2017
:1049E00023689442C5F8883008BFC5F88C30D5F8E4
:1049F000A03043F00203C5F8A030E36823F00403BD
:104A000043F00103E360636889F31188BFF36F8F9C
:104A100020469847EFF31189202383F31288BFF3D0
:104A20006F8FE368D90623F0010237D4E260E368B0
:104A30009A071AD5D8F8000023F00203E360A0B16A
:104A40000021026888B143689C4237D1036869BB82
:104A5000D8F80420C8F80030824201D1C8F80430E8
:104A6000002340F8083BFFF70DFFD5F8A03023F0F6
:104A70000203C5F8A03089F31188BFF36F8FDB05FF
:104A800090D400F087FB8DE705F198040022012106
:104A9000204606F041FA0028F8D194E723F01103EC
:104AA000E36004F11000FFF7EDFEC0E70B60D8F8FB
:104AB0000430834208BFC8F80410D1E722B113685C
:104AC000014610461A46BDE71346F9E7FCDB002015
:104AD00031E30020F8B5C36804469A070F46C3F3D4
:104AE00040062CD45B071AD40B680BB983680B60A3
:104AF000E368DD0742BFA36802263B603D6858BFFC
:104B00000126002D3AD01F4B9B68AB420AD0D5F846
:104B1000A030D807C3F3800214D46FF0120600232C
:104B20003B6025E006F0CFF8D5F8A0300028F0D1A2
:104B3000D907C3F3C002F0D552B15B0708D46FF0B8
:104B40000F06ECE7002AFAD1C3F3C003002BF6D11D
:104B500000232360D5F88C3063B9C5E92244284688
:104B600006F059F8E36843F00403E3603B68A36090
:104B70003046F8BD1C60C5F88C40F0E76FF01506B4
:104B8000CDE700BFDCDB00200146014806F07BB822
:104B9000C0D10020F0B50446002089B0C4E922004D
:104BA0000E9D04F19000C4E9240004F19800C4E9CA
:104BB00026004DB32879002840F2011008BF0120DB
:104BC000C4F8A00000204FF0FF364FF0FF37CDE9CA
:104BD0000330CDE90100CDE9066720460B4B009478
:104BE00000F0AAF855B1296811B1204606F071F815
:104BF0006B791BB1237B43F001032373204609B07B
:104C0000BDE8F04006F06AB80120D9E791490200FA
:104C100037B501900846EFF31184202181F3128803
:104C2000BFF36F8FC16811F01E0F16D153EA020552
:104C300008D101A9FFF74EFF84F31188BFF36F8FEE
:104C400003B030BD41F00801C160019910308161AD
:104C5000034900F03DFC0120EEE70020ECE700BF37
:104C600025AC020001460148FFF7D2BFC0D10020A9
:104C7000F7B50C4616461D460190EFF31187202329
:104C800083F31288BFF36F8F084605F0B5FF55EA2E
:104C9000060309D1204601A9FFF71CFF87F31188FD
:104CA000BFF36F8F03B0F0BDE36804F1100043F071
:104CB0000803E360019B3246A36203492B4600F0E0
:104CC00007FC0120EAE700BF25AC020001460148CD
:104CD000FFF7CEBFC0D100202DE9FF410E9E00F1AD
:104CE000580506730426C0E9165500250446467388
:104CF0000D9EC0E906558673D61D0C9A26F0070650
:104D0000C0E91A168560C573056702920B9A01EB1C
:104D1000060801920A9A00924246F7F75FFA054B9D
:104D200065659B6803B15B6F4046636704B0BDE88F
:104D3000F08100BFDCDB0020F0B5002587B00595D1
:104D4000109DDDE9127604950F9D044603950E9D96
:104D500002950D9D01950C9D0095FFF7BDFFB6F1E5
:104D6000FF3F08BFB7F1FF3F05D056EA070305D163
:104D7000204600F0A1F9204607B0F0BD3A46334680
:104D8000024904F1180000F0A3FBF4E71DAE020095
:104D900038B50D4D2B4653F8184F9C4200D004B93E
:104DA000EC68AB6838B95A7BD20604D1A26912B953
:104DB000DA897F2A05D89C4202D0204600F0D0FA3A
:104DC00023466B6138BD00BFDCDB002008B590F9DD
:104DD0000D200146002A437B04DA03F07F0343736E
:104DE00005F07EFF044B9868431A58425841BDE8CD
:104DF0000840FFF7CDBF00BFDCDB002070B490F9A6
:104E00000D30427B002B29DBD30627D183692BBBD6
:104E1000134962F07F0242730A4652F8184F9442D7
:104E200018BF2346CC6923B9C0E900242060C861BB
:104E30000CE090F90E5093F90E60B5420AD0AE42E4
:104E400008DD5A68C0E9003210605860002070BC6C
:104E5000FFF79EBF9C42E7D01B68E4E770BC704739
:104E6000DCDB0020002A2DE9F0410E460CBF1021AA
:104E70000821427B044611420FD141EA0203D209C4
:104E800018D1437308291BD00120FFF781FFBFF31E
:104E90005F8F637B23F060036373274B9B68A342A0
:104EA00043D1EFF30583002B3FD13046BDE8F041FD
:104EB000F7F7C4B803F07F03437305F011FFE1E790
:104EC000A36813B1204605F013FF04F1180006F0A3
:104ED00045F84FF0000804F15807A56DBD4200D019
:104EE000B5B9154FBB689C42CED1EFF30583002BBB
:104EF000CAD00120FFF74CFF40F201130F4DAB81E8
:104F000000232846C5E91A3300F00EFDBD60BEE758
:104F1000284605F0EDFE05F1180006F01FF82846BA
:104F2000C5F87C80FFF76AFFD7E786F31188BFF3E7
:104F30006F8FBDE8F08100BFDCDB002068D200206D
:104F400070B590F90D200146002A437B04DA03F086
:104F50007F03437305F0C4FE154A4B7B104663F094
:104F60007F034B7350F8183FD469834208BF002376
:104F700023B9C1E900042160D1610CE091F90E5020
:104F800093F90E60B5420ED0AE420CDD5868C1E90F
:104F90000030016059609068BDE87040431A584283
:104FA0005841FFF7F5BE9C42E3D01B68E0E700BF25
:104FB000DCDB0020F8B5124B0C46DDE90676114625
:104FC0009868104A1060EFF31182202282F3128851
:104FD000BFF36F8F9D68284605F094FEB6F1FF3F42
:104FE00008BFB7F1FF3F06D03A463346064905F100
:104FF000180000F06DFA2046BDE8F840F7F71EB83B
:10500000DCDB002004DC00201DAE0200F8B5044605
:10501000EFF31186202383F31288BFF36F8F437B56
:1050200049B2DA0619D18569BDB903F07F0343732C
:1050300005F056FE437B164A63F07F034373134625
:10504000817353F8180F984218BF0546D0695DB9AF
:10505000C4E900300460D46111E00020A17386F33C
:105060001188BFF36F8FF8BD95F90E70B9420BD060
:105070008F4209DD6B68C4E900531C606C6001203D
:10508000FFF786FE0120EAE7A842E1D02D68DEE7BF
:10509000DCDB002049B9EFF3058030B9054B5A69D4
:1050A0009B689A4201D0F6F7C9BF81F31188BFF31C
:1050B0006F8F7047DCDB002010B5EFF311842022E6
:1050C00082F31288BFF36F8F427B510704D484F3BD
:1050D0001188BFF36F8F10BD22F004024273FFF7F7
:1050E0008DFE2146BDE810400148FFF7D3BF00BF49
:1050F00031E30020034648B9EFF3058232B9064A8E
:1051000051699268914201D0F6F798BF83F31188F4
:10511000BFF36F8F704700BFDCDB0020EFF311811E
:10512000202383F31288BFF36F8F054B9A68D37BDC
:10513000013BD37381F31188BFF36F8F704700BFBA
:10514000DCDB002038B5EFF31185202484F31288CE
:10515000BFF36F8F0A4B00209A68D37B0133D37360
:10516000FFF716FE85F31188BFF36F8FEFF3118001
:1051700084F31288BFF36F8FBDE83840FFF7BABFE2
:10518000DCDB0020024B03F11802C3E90622704762
:10519000DCDB0020F8B5EFF31185202383F31288C0
:1051A000BFF36F8F19498868437B03F07F03437314
:1051B00005F096FD08468B685A7B62F07F025A73B1
:1051C00050F8182FCC69824208BF002222B9C3E9E7
:1051D00000042360CB610CE093F90E6092F90E702D
:1051E000BE420ED0B7420CDD5168C3E900210B600E
:1051F00053600120FFF7CCFD2846BDE8F840F6F7E4
:105200001DBFA242E3D01268E0E700BFDCDB002054
:1052100050EA01032DE9F04105460E4603D1FFF7A0
:10522000B9FF00202BE0831C71F1FF3329DB05F06F
:10523000AAFE2C18EFF31188202383F31288BFF302
:105240006F8F124F124BB8681860FFF7BFFDB86838
:1052500010492A463346183000F03AF9BA684046F9
:10526000537B43F010035373F6F7E8FE05F08BFE13
:10527000201A63EB0303012873F10003D1DBBDE8BF
:10528000F0816FF00104241AD4E700BFDCDB0020BA
:1052900004DC00201DAE0200B1F1FF3F08BFB0F1F9
:1052A000FF3F08B506D10A4B986805F06BFD4FF03B
:1052B000FF3008BDFFF7ACFF4FF47A7147F6FF737C
:1052C0000022C0FB0132D80B40EA4240F1E700BFA8
:1052D000DCDB0020014B9868704700BFDCDB00205E
:1052E000D3B5DDE90667089CCDE90067FFF762FEEC
:1052F0001CB1034B9B685B69236002B0D0BD00BF4B
:10530000DCDB00200122044BC01A044BC0105843C0
:10531000034B1A54704700BFF0D20020ABAAAAAAD0
:1053200031E30020C3897F2B12D80A4B1B6863B17D
:10533000094B90F90E201B689A4209DB437BDB0680
:1053400006D1064BC31A18BF012303F001007047B2
:105350000023FAE70CDC002008DC0020B0D000209D
:1053600070B50E4B0E4C1E7C054606EB460304EB57
:10537000C304204605F0F2FD00220A4B28469A5548
:10538000FFF7D0FF48B1084B2046BDE870401A68CF
:105390000649013AD31700F09BB870BDDCDB002052
:1053A000F0D2002031E300200CDC00200553020085
:1053B00038B5EFF31185202383F31288BFF36F8F85
:1053C000104B114A9C681068A04206D1FFF7C8FF35
:1053D00085F31188BFF36F8F38BD00211B7C1160EE
:1053E0000A4AD35C002BF3D02046FFF79BFF00282E
:1053F000EED0637BDB0602D12046FFF7A1FD2046FD
:10540000E4E700BFDCDB002004DC002031E3002007
:1054100008B50648064A0749121A05F0CBFABDE856
:105420000840054A0549064805F0C4BA80C5002071
:10543000D8C9002064EA0200000000004CEA020023
:1054400080C50020034B1B680BB9F8F7BFBC0020D8
:10545000704700BF10DC002030B570B10B4B5B68AB
:1054600098420AD0036843B1D3E90421D0E9044546
:10547000121941EB0501C3E90421D0E900321360A0
:105480005A600023C0E9003330BD00BFF0C60020E1
:1054900010B50E4B1C689C4204D1FFF7D3FF6FF090
:1054A000004010BDFFF7CEFF002CF8D0D4E9043245
:1054B0001B1A62EBE072B3F1004F72F10001EEDAF9
:1054C000002AACBF18460020EBE700BFF0C6002062
:1054D000B3F1FF3F08BFB2F1FF3FF8B504461D46E8
:1054E00016465ED08160EFF31187202383F3128884
:1054F000BFF36F8F013275F1FF3324DA6FF00103D0
:105500002D49D1E900209B1A4FF0FF3262EB0000D9
:105510009E1B60EB0500012E70F1000301DA0126ED
:105520000020C4E90460254ED6F800C07568B44573
:1055300008BF4FF0000CBCF1000F0DD1C4E90065AD
:105540002C6074601CE0FFF77DFF013645F100051B
:10555000361845EBE070E4E7DCE90420D4E90431D7
:10556000934271EB000E1DDAD21ADCF8043060EBC6
:105570000100CCE90420C4E900C31C60CCF804405D
:105580003368B34209D09C4207D10D4B1C6824B943
:10559000FFF77EFF2146F8F7EBFB87F31188BFF397
:1055A0006F8FF8BD9B1A61EB0001AC45C4E9043173
:1055B000C4D0DCF800C0BEE708D30020F0C600204D
:1055C00010DC00202DE9F84FEFF3118C202383F33A
:1055D0001288BFF36F8FDFF8B0A0DFF8B09000241F
:1055E000C9F80000DAF800000025504508BF002087
:1055F000274FE046D7E90021D9F8003078B3D0E949
:10560000046C4FEAE37EB3427EEB0C0B05DAF61A2C
:105610006CEB0E04C0E9046421E0B21841EBE671C2
:10562000C0E90445C7E90021FFF716FF88F3118898
:10563000BFF36F8F83689847EFF31188202383F3BC
:105640001288BFF36F8FD9F80030DAF800009B1B87
:105650005045C446C9F80030CBD1D7E90021002419
:105660009A1841EBE373C7E90023C9F80040FFF73C
:105670000FFF2146F8F77CFB88F31188BFF36F8F8B
:10568000BDE8F84FFFF794BEF0C6002010DC002004
:1056900008D3002010B5EFF31184202383F3128880
:1056A000BFF36F8FFFF7CEFE0346054AD2E9000134
:1056B000181841EBE37184F31188BFF36F8F10BDAD
:1056C00008D30020F8B50446EFF31187202383F3B5
:1056D0001288BFF36F8F026822B187F31188BFF37E
:1056E0006F8FF8BDD0E90A36581C46F10001022838
:1056F00071F1000127D3012B76F10001BCBF01231A
:1057000016465D1E46F1FF3605F041FC013041F1C1
:105710000001401946EB0101012871F1000139DB5C
:1057200005F035FC013041F100016FF00102401934
:1057300046EB01034FF0FF31121A61EB03032046E1
:105740001749FFF7C5FE236B01332363236A6BB14F
:1057500087F31188BFF36F8F2046236A9847EFF3D2
:105760001187202383F31288BFF36F8F54F8185FDB
:10577000A542B2D0002DB0D0284605F01DFB002375
:10578000EB6787F31188BFF36F8F2846BDE8F840B9
:1057900005F0E9BA6FF001024FF0FF33CFE700BF29
:1057A000C55602002DE9F04105461C4690461F46AD
:1057B000EFF31186202383F31288BFF36F8FB4F1C8
:1057C000FF3F08BFB2F1FF3F05D186F31188BFF359
:1057D0006F8FBDE8F081531C74F1FF3309DB012AA0
:1057E00074F10003BCBF0122002412F1FF3844F120
:1057F000FF37284605F0B2FBDDE906010023C5E9C5
:105800000A012B6342463B4628460249FFF760FEE9
:10581000DBE700BFC55602002DE9F74F1D46274BB9
:1058200016469F68012387F8603087F8613052EA96
:1058300005030CBF0123002307F16002804605F039
:1058400074FC8146EFF3118B4FF0200A8AF3128823
:10585000BFF36F8F97F860404CB901465A464046F7
:1058600005F004FC8BF31188BFF36F8F0BE000236E
:1058700087F8603056EA050309D18BF31188BFF32E
:105880006F8F6FF00A04204603B0BDE8F08F5946D1
:10589000CDE900650A4A0B48FFF78CFB0446EFF39D
:1058A00011858AF31288BFF36F8F2A464946404616
:1058B00005F0DCFB85F31188D6E700BFDCDB0020B8
:1058C000F8C6002032E3002038B50346EFF3118517
:1058D000202282F31288BFF36F8FC16001218160A3
:1058E0000068834206D185F31188BFF36F8F0024CF
:1058F000204638BDD0E9003213605A600023C0E969
:10590000003305F08AFC294604460248FFF7C2FB33
:10591000EEE700BF32E300200A460146014805F0E9
:10592000F5BC00BF28C80020014B4367704700BF8B
:1059300028C8002038B504460D4605F0C4F920B942
:10594000064B9B685B6F0BB938BD054B2A46214659
:105950001846BDE8384005F0D9BC00BFDCDB0020AC
:1059600028C8002038B50546002941D051F8043C2C
:105970000C1F002BB8BFE41800F0DCFA1D4A1368B6
:1059800033B9636014602846BDE8384000F0D8BAE7
:10599000A34208D9206821188B4201BF19685B68AF
:1059A00009182160EDE71A465B680BB1A342FAD9EA
:1059B00011685018A0420BD12068014450181160A2
:1059C0008342E0D118685B68084453601060DAE7EE
:1059D00002D90C232B60D6E7206821188B4202BF26
:1059E00019685B680918636008BF21605460CAE7E2
:1059F00038BD00BF18DC0020F8B5CD1C064625F0E8
:105A0000030508350C2D38BF0C25002D01DBA942FC
:105A100003D90C2333600020F8BD00F08BFA214934
:105A20000A6814469CB9204F3B6823B9214630468A
:105A300000F03CF838602946304600F037F8431C47
:105A400023D10C233046336000F07AFAE3E7236871
:105A50005B1B17D40B2B03D923601C44256004E087
:105A60006368A2420CBF0B605360304600F068FAD6
:105A700004F10B00231D20F00700C21A1CBF1B1AE3
:105A8000A350C9E722466468CCE7C41C24F0030491
:105A9000A042E3D0211A304600F008F80130DDD1F1
:105AA000CFE700BF18DC002014DC002038B500234D
:105AB000054D044608462B60F6F706FE431C02D14E
:105AC0002B6803B1236038BD1CDC00200CB4184BDC
:105AD00030B50C1E9DB01D6808DA8B234FF0FF30E7
:105AE0002B601DB0BDE8304002B070474FF4027328
:105AF0000290069002A9ADF8143014BF04F1FF33F0
:105B00002346209A2846049307934FF6FF73ADF877
:105B1000163021AB019300F019FA431CBCBF8B2354
:105B20002B60002CDDD0029B00221A70D9E700BF49
:105B300000C7002070B50A4405460E4E914201D1BF
:105B4000002011E015F8013B11F8014BF05C00F06A
:105B500003000128305D00F0030008BF2033012856
:105B600003D12034181BE9D070BD181BFCD1002CC8
:105B7000E4D1F9E7D0E80200242B2DE9F04786466E
:105B8000904601D8012B06D101F055FF1623036082
:105B90000020BDE8F0870D4635482A4615F8014B30
:105BA000065D16F00806F8D12D2C24D12C7801269C
:105BB000951C2BBB302C30D00A2306F1004C002260
:105BC0000CF1FF3C1046BCFBF3F903FB19CAA4F12E
:105BD0003007092F28D83C46A34234DD571C07D094
:105BE00081452DD301D1A2452ADB00FB03400122D0
:105BF00015F8014BEBE72B2C04BF2C78951CD8E74C
:105C0000102BDAD1302CD8D12A7802F0DF02582AB2
:105C1000D3D16C7810230235CFE72B7803F0DF0364
:105C2000582BF6D00823C8E7A4F14107192F01D853
:105C3000373CD1E7A4F16107192F04D8573CCBE7D3
:105C40004FF0FF32D4E7531C08D122236046CEF830
:105C50000030B8F1000F9CD0691E06E006B140424A
:105C6000B8F1000F95D0002AF6D1C8F8001090E7DF
:105C7000D0E8020013460A46014602480068FFF7D2
:105C80007BBF00BF00C700202DE9F04F904685B0D4
:105C900089461E460D46454A02902B4615F8014B93
:105CA000175D17F00807F8D12D2C41D12C7801276A
:105CB0009D1C002E41D1302C4CD00A2607F1004A01
:105CC00007F1FF3BF31732460AF1FF3A58460393B8
:105CD0005146F3F769F8019200228E468446114638
:105CE0001046A4F13003092B05D9A4F14103192B67
:105CF00037D8A4F137039E423DDD541C15D08445AE
:105D00007EEB010234D38E4508BF844502D1019A4F
:105D10009A422DDB039A714300FB0211A6FB00029D
:105D20000A44181842EBE371012215F8014BD8E739
:105D30002B2C04BF2C789D1CBBE7102EBED1302C21
:105D4000BCD12B7803F0DF03582BB7D16C78102629
:105D50000235B3E72B7803F0DF03582BF6D0082683
:105D6000ACE7A4F16103192B05D8A4F15703C2E7EE
:105D70004FF0FF32D9E7531C0AD12223029A58462A
:105D800051461360B8F1000F0AD105B0BDE8F08F9D
:105D900017B1404261EB4101B8F1000FF5D00AB1F3
:105DA00005F1FF39C8F80090EFE700BFD0E8020026
:105DB00013460A46014602480068FFF765BF00BF68
:105DC00000C700202DE9F04386460D46354E284693
:105DD00015F8014B375D17F00807F8D12D2C26D1A7
:105DE0002C780127851C3BBB302C32D00A234FF086
:105DF000FF380026B8FBF3F803FB08F930466FEADA
:105E00000909A4F1300CBCF1090F29D86446A3425A
:105E100037DDB6F1FF3F07D080452FD301D1A14533
:105E20002CDB00FB0340012615F8014BE9E72B2C86
:105E300004BF2C78851CD6E7102BD8D1302CD6D1B6
:105E4000287800F0DF005828D1D16C781023023573
:105E5000CDE72B7803F0DF03582BF6D00823C6E7F5
:105E6000A4F1410CBCF1190F01D8373CCFE7A4F1E4
:105E7000610CBCF1190F04D8573CC8E74FF0FF364E
:105E8000D2E7731C06D122233046CEF8003032B957
:105E9000BDE8F08307B14042002AF9D006B1691E7F
:105EA0001160F5E7D0E8020013460A4601460248B1
:105EB0000068FFF787BF00BF00C7002007B5009349
:105EC00013460A4601460348006805F0E3FA03B0AA
:105ED0005DF804FB00C7002070B51E469AB04FF471
:105EE0000173044608461546ADF80C300091049144
:105EF000F3F7CCF8094B2A46694601900993002331
:105F0000059020460D9312934FF6FF73ADF80E30B7
:105F1000334600F017F91AB070BD00BFD1B30200CC
:105F200013460A46014602480068FFF7D5BF00BF86
:105F300000C70020014801F076BD00BF50C8002016
:105F4000014801F076BD00BF50C800202DE9F04F98
:105F500098468B899DB007461B060D46144610D502
:105F60000B6973B94021FFF747FD2860286130B9FC
:105F70000C233B604FF0FF301DB0BDE8F08F402395
:105F80006B610023CDF80C804FF00109DFF8A08190
:105F9000099320238DF8293030238DF82A302346A9
:105FA0009A4613F8012B0AB1252AF9D1BAEB040B52
:105FB0000BD05B4622462946384605F096FA01305A
:105FC00000F0A780099A5A4409929AF80030002BF1
:105FD00000F09F8000234FF0FF320AF1010A049382
:105FE00007938DF853301A93CDE9052354460522C3
:105FF0004F4814F8011B05F0B8F9049AD8B9D00637
:1060000044BF20238DF85330110744BF2B238DF854
:1060100053309AF800302A2B15D0079A54460020A6
:106020004FF00A0C214611F8013B303B092B4BD9AC
:10603000B0B1079214E0A0EB0803A24609FA03F3FB
:1060400013430493D2E7039B191D1B68002B039194
:10605000BBBF5B4242F0020207930793B8BF0492B2
:1060600023782E2B0AD163782A2B32D1039B02345A
:106070001A1D1B6843EAE37303920593DFF8B4A08B
:1060800003222178504605F070F938B1A0EB0A00E0
:106090004022049B013482401343049314F8011BF3
:1060A000062225488DF8281005F05FF9002836D023
:1060B000224B1BBB039B073323F0070308330393D7
:1060C000099B334409936AE70CFB02320C4601201A
:1060D000A8E7002301344FF00A0C19460593204627
:1060E00010F8012B303A092A03D9002BC6D00591AC
:1060F000C4E70CFB012104460123F0E703AB2A4669
:1061000004A9384600930E4BAFF30080421C0646AC
:10611000D6D1AB895B063FF52DAF09982CE703ABD1
:106120002A4604A938460093054B00F083F9EDE7B1
:10613000D0E90200D6E90200DAE90200000000001E
:10614000EBB402002DE9F0470C46ADF5227D0021AD
:1061500006460DF10408A74F0093CDF81881CDE94C
:106160004411A549A091A549A1911378002B00F0F5
:106170005C81F95C551C11F0080119D06368002B93
:106180000FDD23681A78BA5C120701D42A46ECE7BF
:10619000459A01330132236045926268013A626098
:1061A000ECE7A19B2146304698470028E9D0EDE76F
:1061B000252B12D099466368002B40F39480226807
:1061C00013784B4540F0318163680132013B226016
:1061D0006360459B01334593D8E7419143915378E0
:1061E0002A2B04BF1023951C4FF00A0208BF4193CD
:1061F000A94619F8011BA1F13003092B1ED9DFF8BC
:1062000000A20322504605F0B0F838B1A0EB0A0016
:106210000123419A4D4683401343419315F8013BB6
:10622000782B06D8572B10D8252BC3D056D8002B47
:1062300064D0032347930A2342936AE0439B4D466D
:1062400002FB031130394391D2E7A3F15802202A0F
:10625000EFD801A151F822F0476302003362020037
:10626000336202006963020033620200336202009B
:1062700033620200336202003362020033620200C2
:10628000336202007F63020065630200E362020082
:10629000E3620200E362020033620200596302001B
:1062A0003362020033620200336202003362020092
:1062B0008F63020061630200036302003362020025
:1062C000336202008B6302003362020065630200E6
:1062D000336202003362020047630200453B022B37
:1062E000A7D8052314E0A19B2146304698470028F3
:1062F0003FF465AF4498002840F08F804FF0FF30A6
:106300008FE0419B43F4087341931023429304238D
:1063100047936368002B4ADD419B590604D42368E8
:106320001A78BA5C120749D4479B022B58DC6B469B
:10633000224641A9304600F0ABF9012875D0022869
:106340007FF424AFD6E7419A42F4007241921022C2
:106350006E2B429202D9DAE7002342930323D7E758
:106360000823D3E70A22F3E72946404605F0E2F97D
:10637000419B054643F0400341930123C8E7419BFD
:1063800043F0400341930023C2E70223C0E7419852
:10639000C3063FF5FBAE009B10F0010F459A03F1D9
:1063A000040100911B6814BF1A801A60EEE6A19BDD
:1063B0002146304698470028AED09BE7459A0132E7
:1063C00045926268013A002A626002DD013323606F
:1063D000A5E7A19B21463046984700289FD089E732
:1063E000042B0FDC6B46224641A9304600F0AAF987
:1063F000A3E700BFD0E80200A1B5020017B6020073
:10640000D6E902000A4B002B3FF4C0AE6B46224691
:1064100041A93046AFF300808FE7A3895B063FF5C3
:106420006DAF0DF5227DBDE8F0874498F9E700BF18
:10643000000000002DE9FF470F7E914680460C4684
:10644000782F9A460C9D01F1430207D8622F0AD893
:10645000002F00F0E080582F00F0BB8004F14206CE
:1064600084F842703AE0A7F16303152BF6D801A136
:1064700051F823F0CD640200E16402005D64020083
:106480005D6402005D6402005D640200E16402007C
:106490005D6402005D6402005D6402005D640200F0
:1064A000FD65020071650200B36502005D640200D3
:1064B0005D6402001F6602005D64020071650200F7
:1064C0005D6402005D640200BB6502002B6804F19C
:1064D00042061A1D1B682A6084F842300123ABE093
:1064E000236829681F0601F10400286001D50D68A2
:1064F00003E05E06FBD5B1F90050002D61687ADA41
:106500002D200029A16084F843002DDA6D425E48F9
:106510000A231646B5FBF3F103FB1157C75D06F8D6
:10652000017D2F460D46BB42F4D9082B0BD12368C1
:10653000DF0708D5236961689942DEBF302306F87A
:10654000013C06F1FF36921B22614B4603AA21460D
:106550004046CDF800A005F07BF8013071D14FF036
:10656000FF3004B0BDE8F08723F004032360CDE7DB
:106570002B682068191D2960050601D51D6802E0F9
:106580004106FBD51D886F2F3F4814BF0A230823FF
:10659000002184F843106668002EA660B9DB2168EC
:1065A00021F004012160002DB3D1002EB1D1164697
:1065B000BBE7236843F0200323607827334884F83F
:1065C0004570296823680E1D2E601E0603D50D68D0
:1065D00004E02D48F3E75D06F9D50D88D90744BFDF
:1065E00043F0200323600DB11023D1E7236823F08B
:1065F00020032360F8E724480A23CCE72B682668A9
:10660000181D6169286035061B6801D5196002E014
:106610007006FBD5198000231646236195E72B6889
:1066200000211A1D2A601E686268304604F09DFE33
:1066300008B1801B606063682361002384F84330E5
:1066400083E72369324649464046D047013086D029
:1066500023689B0714D4E068039B9842B8BF184690
:106660007FE70123324649464046D04701303FF498
:1066700076AF0135E36803995B1AAB42F1DCEAE7D8
:10668000002504F11906F5E7E1E90200F2E902004C
:106690002DE9F84315468A6880460C4632B98A6966
:1066A000002A14BF4FF0FF3201228A6022680027BF
:1066B000DFF88C90D1065FBF1A68111D196016684B
:1066C000A06988B1012807D12B681A7863699B5C9F
:1066D00053B9002F31D022E0022820D12B681B783B
:1066E00019F803301B071AD423680137DA065EBF96
:1066F0002B681B7806F8013B2A686B680132013B66
:106700002A60A2686B60013AA26042B1002BD7DC1C
:10671000D4F880312946404698470028D0D02368D5
:1067200013F0100305D1E2680132E260A26902B100
:106730003370236900203B442361BDE8F88300BF28
:10674000D0E802002DE9F04F984687B0784B0C4610
:106750008246164627464FF0000B93E8070003AB2E
:1067600083E80700734BA169734A032908BF1A46DF
:10677000A36801925A1EB2F5AE7F89BF6FF4AE7561
:106780004FF0000903EB050940F25D1388BFA360D9
:1067900057F81C3B43F450633D462360316803AB1C
:1067A0000222097853F82B0004F0DFFD002840D0C6
:1067B000BBF1010F12D162682AB92268082142F4A4
:1067C000007261602260226822F4A0622260A268E6
:1067D000511EA160DAB94FF0020BDFE7BBF1020FE7
:1067E00006D0A268511EA1608AB94FF0010BD5E70F
:1067F000226802F4C061B1F5007F1FD142F48072BB
:1068000010212260A2686160511EA160B2B132689D
:10681000511C3160127805F8012B7268013A002A88
:10682000726006DCD4F8802131465046904700283B
:1068300074D10BF1010BBBF1030FAFD163680BB93E
:106840000A23636063684FF0000B3C496069C91A12
:1068500004F070FFA368226873B33168606991F82F
:1068600000C010F80C0038B3BCF1300F16D1100581
:1068700014D50BF1010BB9F1000F03D0013309F16D
:10688000FF39A3607368013B002B73600DDD336833
:1068900001333360A368013BA360DBE722F410629D
:1068A00022600B7805F8013BECE7D4F880313146E3
:1068B000504698470028EDD02368D9050DD5BD4234
:1068C00009D905F1FF3915F8011CD4F87C3132469D
:1068D0004D4650469847BD4228D0226812F010021B
:1068E00013D12A70394663685046019EB047D8F8E4
:1068F000003021681A1D11F0200FC8F800201B6815
:106900000FD01860E3680133E360ED1B23690020BA
:106910005D442B44236107B0BDE8F08F4FF0000BBE
:10692000CAE7CA074CBF18801860EBE70120F2E7FE
:106930008CBC02008DB4020091B4020013EA020084
:10694000704700F053BF034690F8240020B99B6ABB
:106950000B6001238B8070476FF08500704700F05B
:106960003CBF00F043BF012903D1C30701D5F2F7B3
:10697000C3BE7047836800EBC101B3F5004F2CBF65
:1069800051F8220031F81200704700EBC101806815
:10699000B0F5004F2CBF41F8223021F8123070477B
:1069A000012208B5FFF7E6FFD04008BD836800EB81
:1069B000C101B3F5004F08D34B681AB143F001038E
:1069C0004B60704723F00103FAE74B881AB143F09C
:1069D00001034B80704723F00103FAE753000122C3
:1069E000FFF7D3BF8368B3F5004F34BF04230823F8
:1069F000C91A081AC0087047B0F5004F34BF042305
:106A00000823481C0833A0EBD300B0FA80F0C0F193
:106A10001F0070472DE9F041174603220E46044639
:106A2000FFF7A8FF8642054607F104080AD10122B4
:106A3000E368BA4023EA0203E360002344F8283005
:106A4000BDE8F081314602222046FFF793FF06465B
:106A50002B4601460322204644F82850FFF795FFB5
:106A6000334629462046BDE8F0410222FFF78DBF9C
:106A700070B50D4686680446FFF792FFB6F5004FE5
:106A8000014601D3012809D03046FFF7B5FF29465A
:106A900002462046BDE87040FFF7BCBF70BD2DE93F
:106AA000F04705468068FFF7A7FF05EB800ADAF894
:106AB000109088460646B9F1000F1BD00327DAF87C
:106AC000104028462146FFF76BFF404507D332466A
:106AD00021462846FFF79EFF2046BDE8F0870322A7
:106AE00021462846FFF746FF013FCAF8100001D0B3
:106AF0008145E4D14FF0FF34EB680136B4401C40CF
:106B0000EAD094FAA4F2B2FA82F2131D55F82340A7
:106B1000DEE72DE9F04114460E460546FFF740FF3B
:106B2000A4EB0608371B0744424631462846FFF7C8
:106B300055FF3A4621462846FFF750FF43460022BC
:106B400021462846FFF721FF21462846FFF728FF68
:106B50003B46211800222846BDE8F041FFF715BF4B
:106B60002DE9F041164604460F46FFF719FF31465E
:106B700005462046FFF714FF05442A4639462046BD
:106B8000FFF72CFF31462046FFF70AFF2B4631184E
:106B900000222046BDE8F041FFF7F7BE2DE9F041A5
:106BA0000D4686680446FFF7FBFEB6F5004F01462A
:106BB00001D3012832D03046FFF71EFF04EB8001DD
:106BC0000E6996B90122E36882401343E360022212
:106BD0000D612B4629462046FFF7D7FE03222946A2
:106BE0002046BDE8F041FFF7D0BE022231462046E4
:106BF000FFF7C0FE0746034629462046FFF7C5FEBD
:106C00000322334629462046FFF7BFFE39462B466E
:106C10002046FFF7BAFE02223146E1E7BDE8F081E7
:106C2000F8B50C460546FFF7BBFE26180122314693
:106C30002846FFF79FFEC3070CD431462846FFF7CE
:106C400017FF21462846FFF7ABFE214622182846AB
:106C5000FFF786FF002221462846FFF78BFE271A02
:106C6000012239462846FFF785FE10EA020613D1B5
:106C700039462846FFF7FCFE214632462846FFF7F4
:106C800079FE2246211A2846FFF76AFF214632463E
:106C90002846FFF76FFE241A21462846BDE8F84033
:106CA000FFF77CBF38B571B1056800222846FFF7B1
:106CB00099FE044601462846FFF778FE2146BDE8C6
:106CC0003840FFF7ADBF38BD70B5066809B9002080
:106CD00070BDB368B3EBD10FF9D9B3F5004F34BF32
:106CE00004230823CC1D1C44E40821463046FFF74A
:106CF000D6FE05460028EAD001463046FFF750FE92
:106D0000A04209D92C44294630462246FFF701FF0C
:106D100021463046FFF742FF304601222946FFF761
:106D200045FEB368B3F5004F34BF0423082303EBDB
:106D3000C5031844CCE72DE9F84306681446B26849
:106D400001F1FF39B2F5004F34BF0423082319EADB
:106D500001090F460BD0494239408B424F4628BFAC
:106D60000B46894654B900252846BDE8F883994268
:106D7000F8D82146BDE8F843FFF7A6BFB2EBD40F21
:106D8000F1D9B2F5004F34BF04220822E11D394485
:106D9000C91A11443046C908FFF781FE8046002811
:106DA000E1D0B36809EBC005B3F5004F34BF04234D
:106DB00008231D4435447B1E1D44B5FBF7F57D4378
:106DC000A5EB090529463046FFF70CFE2C44073495
:106DD00024F00704A41B804507464FEAE40408D2C8
:106DE000024641463046FFF794FE41463046FFF7E3
:106DF000D5FE39463046FFF7D3FD3844844208D2E9
:106E0000394630462246FFF784FE21463046FFF7DA
:106E1000C5FE012239463046FFF7C8FDA4E7B2F5AA
:106E2000802F2CBF082304232DE9F0410026D21A1D
:106E30008C18CD1D25F0070524F00704641BE40819
:106E4000056021462046AC60EE60FFF7D5FD421D8F
:106E50009200013002F107074FEAD7073146A2F14D
:106E6000100205F11000B8BF324604F0A9FA3A4604
:106E700031462846FFF7B2FD3346324631462846B2
:106E8000FFF783FDA4EB0708284631460122FFF7F0
:106E90008DFD42463946FFF7A1FD3B463246394655
:106EA0002846FFF772FD21462846FFF797FD434627
:106EB000324621462846FFF768FD21462846012232
:106EC000FFF774FD3946BDE8F041FFF767BE2DE9D5
:106ED000F04706460D46174698462BB34FF0000A7A
:106EE00098F8004093F80190DB78A40004EB430489
:106EF00098F802301C444444CA4509D33946304608
:106F0000AC46D8F8042008F10803BDE8F047604714
:106F100014F8013B0AF1010A204648F82340F2F731
:106F2000B5F801300444E7E76FF01500BDE8F087DD
:106F300070B5002502462846144614F8013B0BB9EB
:106F4000184609E098B18D4207D1702B04D0A3F107
:106F500040023A2A0BD8002070BDA3F140063A2E19
:106F600005D853780135941C002BE9D00020252B3F
:106F7000224608BF80F00100DEE70020704730B5F0
:106F80008A680C68551C14B14B68934201DC8D6013
:106F900030BD013B934208BF00228D600CBFE2541C
:106FA000A054F5E70FB407B504A951F8040B0191FB
:106FB00000F09AFB03B05DF804EB04B070470CB42A
:106FC00007B504AB53F8042B0193F3F7E7F903B0CB
:106FD0005DF804EB02B07047044608B50846114658
:106FE0001A46A047FEF776F9F5F712F80CB40346F7
:106FF00007B5084605AA40F20511DB6801929847DB
:1070000003B05DF804EB02B070472DE9F04107468C
:10701000884615461E461446B44205D30EB1601B81
:1070200008E02378002BFAD0414614F8010BB8474A
:107030000028F1DABDE8F08110B50369024613F0CB
:10704000080009D11368D4689C429BBF0120126AD2
:10705000E31AD31A0B6010BD00231846FAE713B5E4
:1070600001A90446FFF7E8FF20B1019BE268013B5C
:1070700013440193206A019BC01A013802B010BD6D
:1070800010B5044650182269236AD20702D5013B85
:10709000184010BD984228BFC01AFAE710B5044640
:1070A0000A46C168FFF7ECFF2369E06023F008039C
:1070B000236110BD38B50D46C2698B00016843F0ED
:1070C0000203044642F8213001682A46FFF7D8FF40
:1070D000E3686168984208BF2369206008BF43F0F5
:1070E00008032A46204608BF2361FFF7C9FF6060F6
:1070F00038BD2DE9F74FC768C6699B4616F827309B
:10710000044603F00303022B884691464FF0000328
:1071100006EB870A09D01360CBF800302369990782
:1071200010D4002003B0BDE8F08F56F8271013608C
:107130008908CBF80030F1D0FFF7B0FFE368A36017
:107140000120EFE7A3695046984716F82730054617
:10715000DA07E6D513F002031DD0B8F1000F03D013
:1071600041462046FFF7A6FF61682A462046FFF702
:1071700087FFD4E902319942606004D12A46204653
:10718000FFF77EFFA060A3682360E360236943F0FC
:1071900008032361D4E7014620460193FFF77EFFF1
:1071A000E268A260B8F1000F04D02168E269019B97
:1071B00042F8213005EB0802CBF800202168204678
:1071C000FFF75EFF2369206043F00803236116F890
:1071D00027306FF3000306F82730C9F800A0AFE7A7
:1071E00070B504461546FFF74BFF2368834205D16F
:1071F0002369216023F00803236170BDE269AB00BD
:1072000043F0020342F8213061682A462046FFF726
:1072100037FF6060F1E738B5036904465B0706D5C0
:10722000456AFFF71CFF85422CBF6562606238BD6E
:1072300038B50D4604461C22002104F0C1F8002296
:10724000EB68A361AB6863612B68E3616B686262A2
:1072500023622A6923B1591E194208BF42F0010274
:107260002261012204F128000021BDE8384003F02A
:10727000A8BC2DE9F04F002587B00093036A0446AF
:107280008B420E469246A9460395059539D3EFF3F6
:10729000118B202383F31288BFF36F8F059AD84692
:1072A0002AB129462046FFF79BFF0023059304A936
:1072B0002046FFF7C1FE04990746B1422AD322684F
:1072C000E369204613F8221003EB820921F0030141
:1072D00003F8221021683246FFF7D2FEE3682060EF
:1072E000984212D0002788F31188BFF36F8F03995B
:1072F00029B162690AB12046904700230393002F09
:10730000C5D1484607B0BDE8F08F236943F00803B4
:107310002361E7E718B12046FFF7CCFEE3E7009BC7
:107320005AEA030319D0019103F0CDFC0199A0B9E9
:107330008BF31188BFF36F8F5246009B04F1280036
:10734000FDF7C4FAEFF31188202383F31288BFF30B
:107350006F8FB0FA80F77F09C5E7204605AB03AA17
:107360002568FFF7C6FE0746BDE770B5044683698A
:1073700008460D4698470246EFF31186202383F313
:107380001288BFF36F8F2B78204643F001032B70D8
:107390006168FFF775FE60602046FFF73CFF86F3EB
:1073A0001188BFF36F8F70BD2DE9F041044620278F
:1073B000EFF3118687F31288BFF36F8F236913F001
:1073C000080FA36802D16268934200D9226AD21AD8
:1073D000E16932B986F31188BFF36F8F4FF000086F
:1073E00033E011F8232001EB830812F00300F1D001
:1073F000022803D151F82350AD0805D1D00712D48B
:107400004046A36998470546A1682A462046FFF7EB
:1074100037FE2946A0602046FFF740FE86F311881C
:10742000BFF36F8FC4E742F0020201F82320A36983
:107430004046A5689847294602462046FFF720FEA9
:10744000A06086F31188BFF36F8F4046BDE8F081DE
:10745000F8B50446836908460D4698470646EFF39B
:107460001187202383F31288BFF36F8F2B786FF37C
:1074700000032B7023699B0705D5E268E36903EBE2
:1074800082039D421AD12B786FF341032B70D4E90C
:107490000231994204D132462046FFF7F1FDA06047
:1074A00031462046FFF7FAFD87F31188BFF36F8F4F
:1074B00004F12800BDE8F840FDF7E4B92B6860F35B
:1074C0009F032B60F0E702698368120702D44268C9
:1074D0009A4200D2026AD31A181E18BF01207047C0
:1074E000038B13F0070305D10368002B0CBF0020AA
:1074F00003207047022B05D1408BB0FA80F0400981
:1075000080007047012B05D10368002B0CBF0020C1
:10751000052070470020704710B50C4600B111B926
:107520006FF0150010BD081D00F093F80028F9D188
:10753000A368032BF6D9F3E72DE9F0410D46074682
:107540001946281D90461E4600F097F8044638B1AB
:107550003346424629463846A446BDE8F0416047D6
:10756000BDE8F08110B4EFF31182202484F3128877
:10757000BFF36F8F416110BC0121F3F7D5BB38B564
:107580000C46054658B151B10B6843B14B6833B155
:107590001C22002103F014FF00202C6138BD6FF085
:1075A0001500FBE770B505460E46FFF7B5FF041E54
:1075B00014DBEFF31182202383F31288BFF36F8F64
:1075C0004FF6FF716B8B2C8B8B4204F0070407D1B5
:1075D00082F31188BFF36F8F6FF00A04204670BDED
:1075E000022C0CD101336B8382F31188BFF36F8FB0
:1075F0000023224631462846FFF79EFFEEE7062C81
:1076000014D8DFE804F004131313041A0400002351
:1076100033606B683BB9C5E90066ACB90221284606
:10762000F3F782FBDAE71E606E60F6E782F31188FB
:10763000BFF36F8F6FF00404D0E782F31188BFF3BC
:107640006F8F6FF08504C9E782F31188BFF36F8FE6
:10765000C4E7034640B1426802F00302022A06D0A2
:10766000032A04D0012A05D06FF0150070471A686C
:10767000002AF9D000209860704710B54268034690
:1076800002F00302022A4FF00004816007D0032AAF
:1076900002D05C60002001E018685C6010BD1868D2
:1076A0005C600028F6D0FEF70FF9F3E77047037827
:1076B0005B075FBF03684288C3F34A2303EB1210E2
:1076C0005DBF173020F007008008002070470020C1
:1076D000704701F0A6BA0346D3E8EF0F421CC3E897
:1076E000E12F0029F8D170471FB50023CDE9020131
:1076F0001A4619461846CDE90033F3F731FF05B0B5
:107700005DF804FB0120F3F7EFBC0020704770B573
:10771000D2E901369B1B8B420C4615460AD31368EF
:107720000A460146981903F03EFE2046AB68234402
:10773000AB6070BD6FF01B00FBE770B50E461546E1
:107740001946044618B9BDE87040F3F7CDBC33B113
:10775000C2F34A231030120D184403F024FEC4E98A
:1077600000562046BDE87040F3F742BE2DE9F341D4
:107770005F1C4FEA8708064608F1170020F0070053
:1077800080080C461546F3F711FD00238DF80470B0
:10779000ADF805308DF8073068B10346019AA8F1BD
:1077A000040143F8102F2A46294452F8045B8A4208
:1077B00043F8045FF9D100233146A20102F4E072DC
:1077C00042EA482222F07F4222F4700222F03F0275
:1077D00002B0BDE8F041FFF7B0BF07B50123019249
:1077E00001AAFFF7C3FF03B05DF804FB07B5CDE9BD
:1077F000002302236A46FFF7B9FF03B05DF804FBDC
:107800001FB5CDE90123069B01AA03930323FFF7CC
:10781000ADFF05B05DF804FBF8B506460D4614460D
:107820001F4604B9F8BD214628463A46B047241AF7
:107830000544F6E713B500240094F2F7CBFE02B03E
:1078400010BD10B542680446D2E900238168006883
:10785000FFF7E2FF002263681A6010BD38B54B687D
:1078600005461A68CB680C469A4202D10846FFF7D3
:10787000E8FF6368D3E8EF2F511CC3E8E01F00283E
:10788000F8D1A36800209D5438BD0A2838B50446B5
:107890000D4602D10D20FFF7E1FF29462046FFF7F4
:1078A000DDFF002038BD2DE9F043054687B00846CE
:1078B0000E8891F800900C46D1F808801746F3F72F
:1078C00095FE011EC6F38216C9F3C2091EDB4846A7
:1078D000F3F7A0FD0346214651F8102B6088C2F350
:1078E0004A22002A01EB020408BF00210022C0F353
:1078F0000B10CDE90407CDE9021428464146019654
:107900000092F3F79FFE07B0BDE8F0830023E2E7A3
:10791000436800201B685B689961704743681B6877
:107920001A68526853607047012143681B685A689F
:1079300011771868FFF785BF43681B681868F3F76D
:10794000EFBF70B543680C461D686B689869F3F724
:10795000A7FB214603460F222868BDE87040184760
:1079600001460068F4F744B808B5F4F79DF8BDE89F
:107970000840F4F79DB80A460121FFF72EBF704773
:10798000704700210120F4F733B8836E83F30B882E
:10799000704761B662B680F31188BFF36F8F70478E
:1079A00072B6002383F31188BFF36F8FBFF34F8F3D
:1079B00030BF62B6BFF36F8F704772B6002383F398
:1079C0001188BFF36F8FBFF34F8F20BF80F31188F3
:1079D000BFF36F8F62B6704740E800F313F4803F47
:1079E000D8B208BF6FF01500704730B50C684B680F
:1079F00085B00A894D890094013B24F01F0423447B
:107A000002F01F0242EA451223F01F0369468DF877
:107A100008200393F4F77AFC05B030BD00207047CE
:107A20004FF0FF3070474FF0FF324FF0FF33FCF75D
:107A300043BEFCF7B9BEFCF77BBCF4F7B9BFF4F763
:107A4000C1BF0CB4034607B504AA084652F8041B8C
:107A5000DB680192984703B05DF804EB02B0704711
:107A6000FCF72ABEFCF7A0BE37B5694601AA054659
:107A7000F2F7C0FC044640B9FFF7DDFF09234FF0E1
:107A8000FF340360204603B030BD4FF0FF32019851
:107A90004FF0FF33FFF7E4FF009B20469B689847B9
:107AA00004460198FFF7DEFF2846F2F711FDE9E7EB
:107AB00073B50D461646694601AAF2F79BFC0446CB
:107AC00040B9FFF7B8FF09234FF0FF3403602046A9
:107AD00002B070BD009B9B691BB9FFF7ACFF5F2331
:107AE000F2E701984FF0FF324FF0FF33FFF7B8FF96
:107AF000009B3246294620469B69984704460198D8
:107B0000FFF7B0FFE3E72DE9FF410D46164602A956
:107B100003AA1F46F2F76EFC044648B9FFF78BFF35
:107B200009234FF0FF340360204604B0BDE8F08124
:107B3000029B5B6A1BB9FFF77EFF5F23F1E70398A7
:107B40004FF0FF324FF0FF33FFF78AFF0B9B3246B7
:107B500001930A9B29460093029B2046D3F8248078
:107B60003B46C04704460398FFF77CFFDCE773B54C
:107B70000D461646694601AAF2F73CFC044640B998
:107B8000FFF759FF09234FF0FF340360204602B08E
:107B900070BD009B5B6B1BB9FFF74DFF5F23F2E7E6
:107BA00001984FF0FF324FF0FF33FFF759FF009B72
:107BB0003246294620465B6B984704460198FFF7FA
:107BC00051FFE3E72DE9FF410D46164602A903AA3E
:107BD0001F46F2F70FFC044648B9FFF72CFF0923B4
:107BE0004FF0FF340360204604B0BDE8F081029BF3
:107BF0009B6A1BB9FFF71FFF5F23F1E703984FF064
:107C0000FF324FF0FF33FFF72BFF0B9B3246019300
:107C10000A9B29460093029B2046D3F828803B46C6
:107C2000C04704460398FFF71DFFDCE72DE9F0414C
:107C3000141E05460E4613DB4FF4004740F2E730B2
:107C400000214FF47A720023C4FB0701F1F7ACF86E
:107C500002460B4631462846BDE8F041F4F7A4BD84
:107C60004FF0FF321346F5E703681B689B6813B1BA
:107C70005B6803B118470020704708B5F4F7D8FED9
:107C8000F4F738FF002008BD10B1006800B140686B
:107C9000704701234A0901F01F018B4000EB82006D
:107CA000D0E8EF2F1A43C0E8E12F0029F8D1704740
:107CB00001234A0901F01F018B40DB4300EB8200E6
:107CC000D0E8EF2F1A40C0E8E12F0029F8D1704723
:107CD000FCF7F2BC4FF0FF324FF0FF331030FFF7EC
:107CE000F7BF30B103680C33D3E8AF0F084100F0A1
:107CF0000100704710B50346FFF7C6FF28B1C26800
:107D00001AB1BDE810401846104710BDFCF74CBD35
:107D100038B503680021044693F82050FFF7E1FFCF
:107D200078B90222236883F82020206890F8203058
:107D3000934233D1062D31D108210C30FFF7B8FF23
:107D400024E02368186802F008FE10B903222368B3
:107D5000E9E709212046FFF7C4FF0028E1D00A2106
:107D60002046FFF7BEFF2268C0F10603DBB282F8AF
:107D70002030206890F820209A420FD1062AD9D1CD
:107D8000062D0BD008210C30FFF783FF2368DB6939
:107D900023B92046BDE83840FFF7ACBF38BD38B541
:107DA0000546FFF797FF00212846FFF79AFF10BB13
:107DB0002846FFF769FF2B68044670B1846864B1F8
:107DC000186802F0CAFDC8B12846FFF75DFF01211F
:107DD000836828469847041E07DB286800210C307A
:107DE000FFF757FF2846FFF793FF05F11000FFF755
:107DF0008DFF204638BD6FF07704F6E76FF005047D
:107E0000F3E708B50368D86938B11B689B689868C0
:107E100018B18047C31E5842584108BD10B50446EA
:107E20000809B3B1092812D9A2F10A031844C0B253
:107E300004F8010B002301F00F01092983BF0A3A5E
:107E40008918C9B2303121706370601C10BD3030A8
:107E5000EEE70028E6D1EDE7D0E90032D21A012A98
:107E60000DD95A1C02601B781B020B8003685A1C38
:107E700002601B780A88002013430B8070476FF064
:107E80001500704710B5D0E900349C4220D05C1C2E
:107E900004601B780B7000231360D0E90014A1422A
:107EA00019D20978146801F07F0199400C441460DC
:107EB00001684C1C046091F90010002905DB13686F
:107EC000B3F1805F04D2002004E007331C2BE4D11F
:107ED0006FF0150010BD6FF00A00FBE770B5D1E937
:107EE00000369E4202D16FF0150070BD5D1C0D6022
:107EF000AE421C78F7D09D1C0D60597890F85E302A
:107F00000020042B04BF04F0010313705170ECE750
:107F1000F7B51C461546A27D430003F0020322F08C
:107F20000302C0F3410013430E462072A375284696
:107F30000DF10601FFF790FFD8B9D5E90012BDF8A1
:107F40000630521A9A4212DB636073B12A682260CB
:107F50001A442A60237A67686BB9BB1C9E4206D319
:107F60000020F61AE060266103E02360F2E76FF07C
:107F7000150003B0F0BD284604F11401FFF76CFFB3
:107F80000028F6D13B1DE9E7FFF766BFFFF764BFA6
:107F9000FFF762BFFFF760BF38B50446FFF75CFF2D
:107FA00040B9D4E900239B1A8B6023B122684A6050
:107FB0001A44226038BD4860FCE7FFF74DBFD1E9A5
:107FC0000032D21A012A09D95A1C0A60020A1A7010
:107FD0000B685A1C0A601870002070476FF00B0085
:107FE000704738B50546D1E9002340689B1A821CCA
:107FF00093420C460DD380B2FFF7E1FFD5E90012A2
:10800000206803F0D0F9002023686A6813442360D5
:1080100038BD6FF00B00FBE770B51468641AB4F15B
:10802000805F27D225460026ED09334606F101067A
:10803000FAD102335668DBB25D42CB1AB342136009
:108040001EBF0133136048552046136800F07F01BE
:108050001970C009136805D101331D44234415600C
:10806000536070BD197861F07F0119701368013396
:108070001360EAE76FF07900F3E770B5064614463F
:10808000084669B11568114605351560FFF797FF79
:1080900040B9224629463046BDE87040FFF7BCBFD4
:1080A0006FF0150070BD2DE9F843877D047A07F065
:1080B000010805468946C7F340070CB1838A83B39C
:1080C000D9F80060494605362846C9F80060FFF730
:1080D00088FFB0B92B7AB3B9600000F006002A69B6
:1080E000D9F80030384340EAC800134440F030006B
:1080F0004A463146C9F8003000F03F00FFF78CFFD8
:1081000040B1BDE8F8834946A88AFFF758FF002828
:10811000E2D0F6E7D9F804302A699B1AC9F804308E
:10812000EFE76FF01500ECE70A4601884020FFF703
:10813000A4BF2DE9F843C38806460D463BB30F683C
:1081400005370F60C088FFF73AFF044608BB4FF0C1
:108150000C08B388A34206DC2A463946BDE8F8433A
:108160008220FFF759BF08FB04F9306829464844CC
:10817000FFF737FF80B933684B441A7AD5E90031ED
:1081800099420BD0591C296001341A70E1E76FF055
:1081900015042046BDE8F8830446FAE76FF00B04A7
:1081A000F7E7F8B50D46D1E90031CB1A9342064600
:1081B00001D30020F8BDD41A0F19D0E913231344BA
:1081C0009F4213D8974211D300232246F4F776FE3C
:1081D0000028EFDB0DD0F369A0420344F3616B6824
:1081E00003446B60E5D26FF00A00E3E76FF00B0029
:1081F000E0E76FF07F00DDE770B5C36CC2698CB05B
:1082000002930546134402220393284602A9FFF76E
:10821000C8FF041E2DDBEB6C01AA0DF1030102A8BF
:108220000293FFF72FFE10F10B0F04464FF00102EF
:10823000EBD000283CDB9DF8036006F0F003302B08
:108240001BD10222284602A9FFF7ABFF041E10DB58
:10825000029B16F0060F1A88284652BA92B20CBF3B
:108260000232043202A9FFF79CFF00EAE074002CFE
:108270000ADA14F10B0F1BD119E02846019A02A962
:10828000FFF78FFF0446F2E700229DF803000199F3
:1082900000F0F003602B0B926FD016D8402B62D009
:1082A00009D8202B2FD0302B4BD00023EB6100249A
:1082B00020460CB070BD502BF7D1042305A902A8AD
:1082C0008DF81030FFF762FE54E0B02B65D00BD86C
:1082D000702B5AD0902BE8D1072305A902A88DF85E
:1082E0001030FFF759FE45E0D02BDED195F95F3015
:1082F000002BC4BF03F1FF335AB2092385F85F2076
:108300008DF8103010E08DF81020284605AA02A93B
:10831000FFF7E4FD044670BB9DF815304BB9AB691F
:108320000B9043F00403AB61284604A900F005F963
:10833000BBE7284604A90B936FF06E0400F0FDF82C
:10834000B6E7022302AA8DF8103005ABFFF7E0FD77
:108350000446099B0B902B62284604A900F0EDF817
:10836000002CA2DAA4E7032305A902A88DF8103097
:10837000FFF70AFE04460B94EEE7052305A902A8C1
:108380008DF81030FFF704FEF4E7062305A902A8D4
:108390008DF81030FFF7FEFDECE7082305A90DEB83
:1083A00003008DF81030FFF708FEE3E738B5456BA2
:1083B0000446288806220121F4F7CCF90028A0629F
:1083C00004DAFFF738FB0068404238BD2B88616B48
:1083D000012B0CBF08221822FFF76AFB002803DAE2
:1083E000A06AFFF741FBECE70020EEE72DE9F3413F
:1083F000002406460F461546A046AC4201D3002095
:108400000DE0B06A0023CDE900882A1B3919FFF777
:108410007AFB031E06DAFFF70EFB0068404202B04B
:10842000BDE8F0811C44E8E72DE9F041002507464E
:108430002B460C46C9688B4210D10026B046AE428E
:1084400016D2B86A00222146FFF791FB031E0CDA10
:10845000FFF7F1FA00684042BDE8F081A26802EB44
:10846000C302526801331544E5E71E44B54217D8EC
:108470000020F1E71B1AC1F804800132E168914243
:10848000DDD9A16801EBC20148689842F2D9C01A4F
:108490004860A06850F83210194440F83210CEE716
:1084A0000022EBE713B5806A002483F00103CDE9D5
:1084B00000449B01FFF786FB002803DAFFF7BBFAB5
:1084C0000068404202B010BD08B5806AFFF7CCFAE0
:1084D000002804DAFFF7AFFA0068404208BD002028
:1084E000FCE7FFF7F1BF38B504460D46826D002169
:1084F000406D02F065FF636D2B60A26D13446B60ED
:1085000038BD08B502F043FD4FF47A72A0FB0203B8
:1085100002FB0133C00B40EA434008BD4FF0FF327D
:108520004FF0FF33FCF7C8B810F0040F0CBF6FF02A
:108530007F0000207047FCF737B938B5836C0446DC
:108540000D4653B1FFF7F7FF20462946A36C984725
:108550002046BDE83840FFF7E1BF38BD30B589B0EF
:1085600004460D46FFF7BDFF00211C22C4E905119A
:10857000C4E90711684602F023FF0123694620463B
:108580008DF800300795FFF7D8FF09B030BD2DE911
:10859000F0410F4690461E46054620B3FFF7BEFF4A
:1085A0002C6AB4B144452246334628BF4246394678
:1085B0002846F4F783FC044616B910F10B0F08D0D7
:1085C000002C0CDC08BF6FF07F0428462146FFF723
:1085D000C5FF2846FFF7AFFF2046BDE8F0812B6AB4
:1085E0001B1B2B62F5E76FF01504F5E738B5054660
:1085F000F4F74CFC041E05DA21462846FFF7AEFFCF
:10860000204638BDFFF77DFF00246861F8E710B50C
:10861000044690B16822002102F0D2FE204602F00A
:108620004DFA042384F85E3094F8603043F002037E
:1086300084F860303C23A4F85C3010BD37B50546A3
:1086400000283AD0C36AC3B3FFF768FF6B6D8BB3E2
:10865000EB6C7BB32846F4F70FFC041E24DB694661
:108660002846FFF740FFAB69694643F002032846FE
:10867000AB61F4F75BFB041E13DBDDE90012284657
:10868000521AF4F703FC041E0BDBFFF73AFF002439
:10869000686185F85F402846FFF74DFF204603B02C
:1086A00030BD2846FFF71DFF0023C5E90533C5E9A6
:1086B0000733F0E76FF00B04F6E76FF01504EDE712
:1086C00070B50E4605468EB000283AD0002938D045
:1086D000FFF724FF284601A9FFF705FFA869FFF768
:1086E00023FF041E22DB304601A9FFF7DCFC041E39
:1086F0001CDB019A029B03929B1A1C220493F368D1
:108700000021059333690DEB0200069302F058FE39
:1087100003AB09930223284607A90A93F4F7C2FB87
:10872000041E09DA21462846FFF718FF2846FFF7FE
:1087300002FF20460EB070BDFFF7E3FE0024686123
:10874000F4E76FF01504F4E773B50E460546F0B193
:10875000E9B1FFF7E3FE28466946FFF7C4FEA869C2
:10876000FFF7E2FE041E0CDB69463046FFF7DCFC37
:10877000041E06DBDDE900122846521AFFF736FF19
:1087800004462846FFF7D7FE204602B070BD6FF0C2
:108790001504F9E737B5054608B3FFF7BFFE2846CD
:1087A0006946FFF7A0FEA869FFF7BEFE041E10DBB6
:1087B0006846F4F73DFB041E0BDBDDE9001228469A
:1087C000521AFFF713FF041E03DB00212846FFF7B0
:1087D000C5FE2846FFF7AFFE204603B030BD6FF060
:1087E0001504F9E773B50E460546F0B1E9B1FFF798
:1087F00095FE28466946FFF776FEA869FFF794FEC6
:10880000041E0CDB69463046FFF793FC041E06DBB2
:10881000DDE900122846521AFFF7E8FE0446284612
:10882000FFF789FE204602B070BD6FF01504F9E72E
:1088300037B5054618B3FFF771FE28466946FFF7BE
:1088400052FEA869FFF770FE041E12DB6846F4F7BB
:1088500001FB041E0DDBDDE900122846521AFFF76A
:10886000C5FE044695F95F307F2B1CBF013385F8A8
:108870005F302846FFF75FFE204603B030BD6FF043
:108880001504F9E738B50446F0B1FFF747FE65690E
:10889000FFF737FE401B06D52046FFF74CFE6FF072
:1088A0000A05284638BDB4F85C30002BF4D04FF4EC
:1088B0007A7253438342EFD82046FFF7B9FF05464B
:1088C0002046FFF738FEECE76FF01505E9E738B50D
:1088D00004464569FFF715FE431B4FF47A70B4F860
:1088E0005C2023EAE37350431AB1984204D9C01ABA
:1088F00038BD4FF0FF30FBE70020F9E738B50546FB
:10890000D0B1FFF70BFEAB699B070FD52B6A83B97C
:108910002846FFF771FC041E03DA21462846FFF7BC
:108920001DFE2846FFF707FE204638BD6FF07F0486
:10893000F7E76FF00F04F4E76FF01504F4E7012395
:10894000FFF725BE70B506460C468D18AC4201D324
:10895000002070BD214630462A1BFFF7F0FF00289B
:10896000F7DB01D00444F1E76FF00400F1E70C22DB
:108970000369C9B201FB0233186C00F007007047AD
:1089800070B5C9B20369EFF31185202484F312880E
:10899000BFF36F8F0C2606FB0134246C14F0C00467
:1089A00008D0A24206D085F31188BFF36F8F4FF035
:1089B000FF3070BD012271430B441A6485F31188A6
:1089C000BFF36F8F43680B445B6898470020F0E764
:1089D0008022FFF7D5BFF8B5069F0469C9B2EFF34F
:1089E0001186202585F31288BFF36F8F0C2569430C
:1089F0000C44256C05F0070CBCF1010F0BD127646A
:108A000086F31188BFF36F8FC4E90E2343685B5868
:108A100098470020F8BD05F0C005AF4286F31188E5
:108A2000BFF36F8F0CBF6FF077004FF0FF30F1E7AF
:108A300013B580240094FFF7CEFF02B010BD10B430
:108A40001C240069CBB203FB0400002110BC1047BA
:108A50000020F8F793BD002000F082BD1046FBF720
:108A600011BF084608B51146F8F790FC002818BF5A
:108A70006FF0040008BD08B500F065FD002818BFC0
:108A80006FF0040008BD436800205B681B690B6041
:108A90007047436802EA01005B6821EA02019860BE
:108AA0000020D9607047436800205B689960704778
:108AB000436800205B68D960704743685A68536810
:108AC00021EA03000B4090600020D360704710B58E
:108AD00003695868F8B1884219D19C680868A142B6
:108AE000586000D19860002008602AB15A680A6076
:108AF0009A68596002B99960002010E0814206D15D
:108B00000868206098688142EDD19C60EBE70446DC
:108B100000680028F2D1002AE8D16FF0150010BDDE
:108B200030B543681360057A446804EBC504A3427A
:108B300002D36FF0010030BD5C798C4201D0083364
:108B4000F0E70020F7E743681B68D3F88004C3F818
:108B500080047047436802691B68D3F8100150B164
:108B60000020526912780A70C3F81001D3F810215E
:108B700001221A6070474FF0FF30704702680346C9
:108B8000D2F8580140B95B689B0706D4D2F820019F
:108B9000003818BF012070470120704742681368F1
:108BA000D3F80413C90517D5D3F82011A1B1EFF3F9
:108BB0001181202080F31288BFF36F8FD3F820013A
:108BC00030B10020C3F82001D3F820010120D86083
:108BD00081F31188BFF36F8F5268D20614D5EFF37B
:108BE0001182202181F31288BFF36F8FD3F85811BF
:108BF00011B10021C3F800154FF48001C3F8081328
:108C000082F31188BFF36F8F7047002200F1500389
:108C10009B009BB203F1804303F5A8331A601B68E5
:108C2000704708B5F4F740FF08BD01F091BE10B5DC
:108C30000446FEF700FF046010BD02F044B8FBF7E5
:108C400021BE4B1C70B5054617D021EAE1744FF4E4
:108C5000004640F2E73000214FF47A720023C4FB53
:108C60000601F0F7A1F802460B462846FBF72EFE58
:108C7000002818BF6FF00A0070BD4FF0FF32134696
:108C8000F3E7FBF791BD4B1C70B5054617D021EA01
:108C9000E1744FF4004640F2E73000214FF47A725D
:108CA0000023C4FB0601F0F77FF802460B46284676
:108CB000FBF702FD002818BF6FF00A0070BD4FF0EF
:108CC000FF321346F3E7002070472DE9F0411446C8
:108CD000002286B001290D461E46CDE90422DDF8AA
:108CE000308007680AD1192C13D1FEF7A4FE5F2348
:108CF00003604FF0FF3006B0BDE8F0812146284602
:108D000003AAF5F74BFA00281EDAFEF794FE6D234E
:108D1000EEE72146284603AAF5F740FA0028F4DBDF
:108D2000143C012C07D836B14FF008083268B368FC
:108D30000492059304AE334629463846039ACDF88B
:108D40000080FAF739FBD6E7B5F58D7FF3D10C2C0F
:108D500008BF4FF00408EEE72DE9F0411C46002360
:108D600086B00F461546CDE9043308230668294628
:108D700038460DEB0302DDF830800393F5F70EFA69
:108D8000002809DAFEF757FE6D234FF0FF36036027
:108D9000304606B0BDE8F081012F1CD1A5F11403C7
:108DA000012B18D803AA04AB304600923946029A28
:108DB000FAF730FC06460028EAD1012FE8D1042D4D
:108DC0000CD120680028E3D0FFF731FFFEF733FE17
:108DD00003682360DCE742462346E5E7143D012DA6
:108DE000D6D8049BC4E90030059BA3601023C8F8C3
:108DF0000030CDE7006801F03EB838B5044604B94C
:108E000038BDE069256802F094FA204602F091FA34
:108E10002C46F4E7FBF750BCFBF7C6BC2DE9F0434A
:108E200089B00546D0E900900E4617469846109C3A
:108E300008B1FFF7F1FFA4B9CDE9004443463A4633
:108E40003146484601F0E2F80446686828B14FF020
:108E5000FF324FF0FF33FFF7DDFF204609B0BDE8DA
:108E6000F0832388012B0BD1ADF80830636862884A
:108E700003930823ADF80A2001936B440093DDE7C8
:108E8000022B18D16288ADF80830ADF80A20231DF6
:108E90000DF10C0C04F1140E624618685968083381
:108EA00003C273459446F7D1237D8DF81C301623F9
:108EB000019302ABE2E7FEF7BEFD6A234FF0FF34F9
:108EC0000360C2E7002307B5CDE90033FFF7A6FF33
:108ED00003B05DF804FB2DE9F04F064640688BB007
:108EE0000C46DDE914579046994608B1FFF794FF08
:108EF000D6F800A005B1AFB900232146CDE9003373
:108F000042464B46504601F0C2F90446706828B10B
:108F10004FF0FF324FF0FF33FFF77CFF20460BB0DE
:108F2000BDE8F08F4FF0160B04AB5A4600211846EF
:108F300002F046FA03AACDE9000221464B4642461A
:108F40005046CDF80CB001F0A2F9041EDEDBBDF8EE
:108F50001020012A0AD1039B082BD7D1BDF812108B
:108F60002A80059A69806A603B60CFE7022ACDD1EA
:108F7000039B162BCAD1BDF812300DF1140C6B8077
:108F80002B460DF1240E23F8042B624603CA7245CA
:108F900018605960944603F10803F6D19DF8243017
:108FA0002B751823E0E7002307B5CDE90033FFF761
:108FB00092FF03B05DF804FB38B505460068FAF788
:108FC000C9F9044610B92846F5F778FA204638BDA5
:108FD000F0B50A880B46012A066887B00DD1ADF8B6
:108FE0000020082249885B68ADF8021001936946A9
:108FF000304600F0F4FE07B0F0BD022A15D14988D2
:10900000ADF80020ADF802101A1D01AD03F11407F0
:109010002C4610685168083203C4BA422546F7D17D
:109020001B7D16228DF81430E1E7FEF704FD6A235C
:1090300003604FF0FF30DEE7F0B5056808880B46A7
:10904000012887B00DD14A884B68ADF8022008226C
:10905000ADF8000001936946284600F01EFE07B0F7
:10906000F0BD022815D14A88ADF80000ADF8022005
:1090700001AE0A1D01F11407344610685168083228
:1090800003C4BA422646F7D11B7D16228DF8143050
:10909000E1E7284607B0BDE8F04000F0FEBD03461A
:1090A00070B40C46DA8800681979224301240569F6
:1090B0008C402B6812F0010F866814BF2343A34332
:1090C0002B60336870BC1847012303FA01F1036970
:1090D0001B68194203D022B183681B6903E0002A90
:1090E000FAD08368DB6818470A460121FEF775BB92
:1090F0000121F5F72DBE0021F5F72ABEA0F12303CB
:10910000DBB2082B9DBF40F20510D84000F00100F3
:10911000002070470D2804D0A0F10A03584258419E
:1091200070470120704710B5016802468B1C036030
:109130008C782046FFF7EEFF10B90CB103311160B7
:1091400010BD1368F6F7F2B803688B4286BF40681B
:1091500000EB0110002070470378012B04D0023B84
:10916000012B03D8406870470820704700207047E3
:1091700010B503780446023B012B02D8806802F048
:10918000D8F800220023C4E9022310BD38B50D46EB
:10919000044640B11021284602F0D6F8606028B19C
:1091A0000020256038BD6FF01500FBE76FF00B0065
:1091B000F8E770B5044628B143681BB10025236861
:1091C0009D4200D370BD666806EB05163046FFF77A
:1091D000CFFF10220021304602F0F2F80135EEE711
:1091E00038B5044648B143683BB10025FFF7E1FFBD
:1091F0006068256002F09DF8656038BD10B578B1F3
:1092000043686BB1FFF7A0FF044648B1FFF7B0FF1A
:1092100004230022237000230020C4E9022310BD90
:109220006FF01500FBE770B516461D4668B1436840
:109230005BB1FFF789FF044638B1FFF799FF0123BF
:109240000020C4E90265237070BD6FF01500FBE7D4
:10925000F8B517461D46C0B14368B3B1AAB1FFF7D0
:1092600073FF044688B1681C02F06AF8064678B1BC
:109270002A46394602F097F82046FFF779FF022385
:10928000002065602370A660F8BD6FF01500FBE755
:109290006FF00B00F8E7F8B517461D46C0B14368FC
:1092A000B3B1AAB1FFF750FF044688B1284602F0D7
:1092B00047F8064678B12A46394602F074F8204647
:1092C000FFF756FF0323002065602370A660F8BDFA
:1092D0006FF01500FBE76FF00B00F8E708B5B0B1D1
:1092E0004368A3B19AB1FFF72FFF80B10378012B38
:1092F0000DD1D0E9023113F5004041F10001B0F584
:10930000803F71F1000102D20020138008BD6FF090
:109310001500FBE708B590B1436883B17AB1FFF758
:1093200013FF60B10378012B09D1D0E90231B3F505
:10933000803F71F1000102D20020138008BD6FF060
:109340001500FBE708B590B1436883B17AB1FFF728
:10935000FBFE60B10378012B09D1D0E9023113F192
:10936000004041F1000111B90020136008BD6FF009
:109370001500FBE708B570B1436863B15AB1FFF758
:10938000E3FE40B10378012B05D1D0E90201C2E927
:109390000001002008BD6FF01500FBE770B5164610
:1093A0001C46C0B14368B3B1AAB1A4B1FFF7CCFE6B
:1093B000014680B10378022B0DD1FFF7CDFE236863
:1093C000054683420AD302468968304601F0EBFF26
:1093D0000020256070BD6FF01500FBE76FF00B00FB
:1093E000F8E7024608B570B1406860B1116819B17C
:1093F000002108B103780BB9084608BD10460131B9
:10940000FFF7A2FEF5E76FF01501F5E7FEF7E5B906
:10941000FEF7ECB908B530B1F6F716FEBDE8084026
:109420000020F6F7A3BDF6F707FE0028F6D0BDE84A
:109430000840F6F7EDB908B50020F6F753FD00280F
:1094400018BF6FF00D0008BDFEF7C7B9FEF7CEB923
:1094500073B50C4605461646FEF7EDFA0023224684
:10946000036001A92846FCF705FC019B0446AB42BA
:1094700003D16FF03C0002B070BD1B78002BF8D117
:1094800000F10043013B033302D800203460F2E7CF
:10949000FEF7D1FA0368222BF7D1EAE730B51025A1
:1094A00087B0144601AB02AA0195FFF777FF68B9B0
:1094B000019B224618336B4403F8100C294602A87E
:1094C000FFF7C6FF002818BF6FF03C0007B030BDA3
:1094D00008B501F03BFA18B1BDE80840FFF7ABBF93
:1094E00008BD03780BB1F7F761BD70470A4601214B
:1094F000FEF773B900B589B006AB02930823039356
:1095000001AB049304230791CDE9053004AA03209D
:1095100002A9F7F715FF0228019B09D003280AD0FA
:1095200060B9181E18BF0120404209B05DF804FB65
:109530006FF01500F9E76FF08500F6E74FF0FF30A8
:10954000F3E700207047002070477047004701F0A4
:10955000FFB940F00040C1F88000C2F880007047B9
:10956000F7F790BFF7B51646DDE90847019001A867
:109570001D46F8F797F8019BB6F1000C18BF4FF0A5
:10958000010C00EB83000B1E18BF0123002D43EAE2
:109590004C0314BF4FF00C0C4FF0000C002C43EAAE
:1095A0000C0314BF4FF4E06C4FF0000C002F43EAA3
:1095B0000C0314BF4FF4403C4FF0000CD0F80022D5
:1095C00043EA0C0322EA030301B109780EB13678AD
:1095D000760019430DB12D78AD0031430CB12478DC
:1095E000240229430FB13F783F040C433C43C0F8A9
:1095F000004203B0F0BD1FB50DF10F03019300232E
:109600008DF80F101A4619460093FFF7ABFF05B00F
:109610005DF804FB70B501F1080330F8133016460D
:10962000DA0504460D4609D5C3F3432300EBC30214
:10963000314650F83330526828469847A3682BB11A
:1096400031462846E268BDE87040184770BD38B51D
:109650000579044628460A46F8F782F8C0B1114653
:109660002846F8F76DF898B111462846F8F75CF8E7
:10967000012322688340C2F80833226803B202EB58
:109680008303D3F8102522F00302C3F8102538BD58
:109690000021BDE838401046FFF7ADBFF8F758B9D4
:1096A000FFF7D5BF022904D0042906D0012900D133
:1096B0007047806808B1F4F72FBD7047F8F7CCBC4D
:1096C000002210B50468944200D110BD00EBC20125
:1096D0004B68013223F0FF0343F003034B60F2E7D2
:1096E0000420F8F76DBC0420F8F772BC08B5F8F751
:1096F00035FCBDE80840FAF7B9BD38B50446002589
:10970000031D2268AA4201D8002319E04FF000028D
:10971000D3E8CF0F032804D1C3E8CC2FBCF1000F4E
:10972000F6D102D008330135EBE701EB851318467B
:109730004022002101F044FE034604EBC504A06072
:10974000184638BD0830704738B5054620B9F8F7D7
:1097500089FC80B9002038BDF4F7D6FC0446002807
:10976000F8D0F8F77FFC38B92046F4F7D5FC012093
:10977000F4F7A0FCEEE72C46C56040F8084FEAE796
:1097800040EA0141104640F8081DF8F77DBCF8F7A3
:1097900075BCF8F76DBCF4F7B7BC08B5F4F7BCFCC2
:1097A000BDE808400120F4F785BC0429F8B505465A
:1097B000174603D0102910D000240CE00820F4F73D
:1097C00095FC04460028F7D000234360012347801E
:1097D00003802B6843602046F8BD1620F4F786FC12
:1097E00004460028E8D0061D12220021304601F070
:1097F000E7FD022323802B46678005F1100253F812
:10980000041B934246F8041BF9D1E4E7134609B957
:10981000116070470A88012A02D0022A07D07047D7
:109820001A68082A28BF08221A6001F0BCBD1A680D
:10983000162A28BF1622F7E708B5F9F709FA40B14A
:1098400000F11C03D3E8EF1F0131C3E8E21F002A37
:10985000F8D108BD006808B1F9F78AB9704737B583
:109860000025036804460093838F6846ADF80650D0
:10987000ADF8043000F0EBFD38B1A36B68469847B3
:1098800094F83E300BB1A563E56303B030BD40688A
:10989000003818BF0120704700230B60836813B99C
:1098A000C0E90111704719608160704738B50546FD
:1098B0000C46F8F7EFFBAA68236894426B6008BF78
:1098C000AB6000232046236000F04DF9BDE838402E
:1098D000F8F7E6BB406870470069431E584258419C
:1098E00070470069831E5842584170470069C31E83
:1098F0005842584170474069B0F5817F05D040F229
:109900001113C31A5842584170470120704790F80C
:109910002000C0F34000704790F82000C0F38000A2
:10992000704790F82000C0F3C0007047006C00F052
:109930000100704790F8200000F0010070470369B3
:10994000012B05D18069A0F180035842584170472E
:109950000020704790F82000C0097047836933F0F9
:10996000800314BF01200020704790F82000C0F34E
:1099700040107047806B003818BF0120704790F886
:109980003400431E58425841704708B590F82030C3
:10999000014613F001020BD1FFF7E0FF28B908469A
:1099A000FFF7CDFF80F00100C2B202F0010008BD58
:1099B0000022FAE770B504460D4616462046FFF72A
:1099C000E4FF70B155B1284600F0BCF848B9314603
:1099D0000220F4F773FA0028F0D070BD6368002B02
:1099E000F5D00020F9E74068003818BF0120704723
:1099F00090F82200003818BF0120704710B50446C7
:109A0000FFF7ACFF94F82010C1F3401340EA0302C3
:109A1000236982F00102012B14BF0123C1F38003EB
:109A2000D2B220461A40FFF766FF48B1C1F30011D9
:109A30002046FFF784FF0A4080F00100104010BD6F
:109A40000121F5E710B50C46F9F702F928B190F8B5
:109A5000203064F3861380F8203010BD10B50C461A
:109A6000F9F7F6F828B190F8213064F3000380F894
:109A7000213010BDD0E9092353EA020109D04FF487
:109A80007A71B3FBF1F001FB02000128B8BF01209D
:109A900070474FF0FF307047D0E90B2353EA0201C3
:109AA00009D04FF47A71B3FBF1F001FB02000128F9
:109AB000B8BF012070474FF0FF30704701380228CF
:109AC0008CBF002001207047013802288CBF002085
:109AD000012070470388012B03D0022B06D0012000
:109AE0007047082914BF0020012070471629F9E7A4
:109AF000032915D011280CD004DC88B106280AD01F
:109B000000207047B0F5817F05D040F211139842D4
:109B1000F6D1022900E0012914BF0020012070477E
:109B200001207047C368012B03D0022B07D001200E
:109B300070470888012814BF00200120704708885A
:109B40000228F8E700B10068003818BF012070470C
:109B500000B1006870474389406818447047028923
:109B60004089101A704710B504464068FFF70FFE91
:109B7000E06808B1F4F7C2FA2046BDE81040F4F7F7
:109B8000BDBA10B50446206800B910BD626803680C
:109B90009042236008BF6360FFF7E5FFF3E700F042
:109BA0001ABD10B5044660B1406908B1F4F7A6FAD1
:109BB000A06908B1F4F7A2FA2046BDE81040F4F716
:109BC0009DBA10BD10B5044600F003FD2368436044
:109BD000A36983602046BDE8104000F0FCBC2DE97D
:109BE000FF4180460F461646FFF768FF38B96A20E6
:109BF000FFF71DF84FF0FF3004B0BDE8F0813046AC
